:100000000C9467280C94A1E90C9476E90C944BE9C4
:100010000C9420E90C94F5E80C94CAE80C949FE841
:100020000C940BC30C9498280C9498280C94982842
:100030000C9498280C940CA70C9498280C9498284D
:100040000C9498280C94AABB0C9498280C9498288B
:100050000C9498280C9498280C943ABA0C94CCE9F7
:100060000C9498280C9451C20C9498280C949828BD
:100070000C9498280C9498280C9498280C94982800
:100080000C9498280C9498280C9498280C949828F0
:100090000C9498280C9498280C9498280C949828E0
:1000A0000C9498280C9498280C9498280C949828D0
:1000B0000C9498280C9498280C9498280C949828C0
:1000C0000C9498280C9498280C9498280C949828B0
:1000D0000C9498280C9498280C9498280C949828A0
:1000E0000C9498282B622B6232623262326239623F
:1000F000396239624662406240624062A868AD6817
:10010000B268BC68C6683F69D068D868E068EA68C9
:10011000F468FE680D6917693F6921692B693569C3
:1001200038763B762A762E76347672763F7643762C
:1001300049764D76517657765B765F767276657640
:1001400069766D7685C28BC29CC2A7C2AFC2C4C29B
:10015000B3C2C4C2B7C2BBC2C4C2C1C2084AD73B41
:100160003BCE016E84BCBFFDC12F3D6C74319ABD86
:1001700056833DDA3D00C77F11BED9E4BB4C3E91AA
:100180006BAAAABE000000803F05A84CCDB2D44E99
:10019000B93836A9020C50B9918688083CA6AAAA9B
:1001A0002ABE000000803F00434F4D4D554E49434D
:1001B0004154494F4E0044525952554E00455252F7
:1001C0004F525300494E464F004543484F0020745C
:1001D0006F6F206C6F6E6720657874727573696FCE
:1001E0006E2070726576656E7465640A0020636FB8
:1001F0006C6420657874727573696F6E20707265B7
:1002000076656E7465640A0047322F473320626159
:100210006420706172616D65746572730A00536C5D
:100220006565702E2E2E004C756C7A426F742054CA
:10023000415A20352072656164792E0052657375CC
:100240006D696E67207072696E7400436C69636BD0
:1002500020746F20726573756D652E2E2E004E6FA3
:10026000206D6F76652E00456E642066696C652092
:100270006C6973740A00426567696E2066696C6513
:10028000206C6973740A004D31323500534420707C
:1002900072696E74696E67206279746520004E6FB2
:1002A00074205344207072696E74696E670A004648
:1002B000696C652064656C657465643A0044656CBE
:1002C0006574696F6E206661696C65642C2046698F
:1002D0006C653A20006F70656E206661696C6564BC
:1002E0002C2046696C653A20002569730025696DEC
:1002F00020256973002569682025696D20256973AB
:1003000000256964202569682025696D20256973A9
:100310000025697920256964202569682025696D93
:1003200020256973005072696E742074696D653A96
:100330002000000125301D0CFF24311C0BFF232F52
:100340001B0AFFFF040308060202222B1A41420384
:100350003809FF3628294527444350726F74656376
:100360007465642050696E0A00457874727564651E
:1003700072202573004C756C7A426F742054415A78
:1003800020352072656164792E00C901C401BD0168
:10039000B601A8016F66660044454255473A006FB2
:1003A0006B00436F6F6C696E6720646F6E652E0023
:1003B00048656174696E6720646F6E652E00205712
:1003C0003A004578747275646572202573004C7527
:1003D0006C7A426F742054415A20352072656164F2
:1003E000792E0042656420646F6E652E0020573AB6
:1003F000004265642068656174696E672E0042651D
:100400006420636F6F6C696E672E004C756C7A4266
:100410006F742054415A2035204F66662E00436188
:10042000703A454D455247454E43595F50415253EE
:1004300045523A310A004361703A434153455F4C9B
:10044000494748545F4252494748544E4553533AEE
:10045000300A004361703A544F47474C455F4C495E
:10046000474854533A300A004361703A534F465458
:10047000574152455F504F5745523A300A00436149
:10048000703A4C4556454C494E475F444154413AB9
:10049000300A004361703A5A5F50524F42453A3039
:1004A0000A004361703A4155544F4C4556454C3A09
:1004B000300A004361703A5052494E545F4A4F42ED
:1004C0003A310A004361703A50524F4752455353F4
:1004D0003A300A004361703A4155544F5245504FEB
:1004E00052545F54454D503A310A004361703A45C9
:1004F0004550524F4D3A310A004649524D574152EC
:10050000455F4E414D453A4D61726C696E20204603
:1005100049524D574152455F56455253494F4E3A05
:10052000312E312E352E3434204558545255444501
:10053000525F545950453A53696E676C65457874FB
:10054000727564657220534F555243455F434F4463
:10055000455F55524C3A68747470733A2F2F636F2D
:1005600064652E616C6570686F626A656374732E72
:10057000636F6D2F646966667573696F6E2F4D4189
:10058000524C494E2050524F544F434F4C5F5645AA
:100590005253494F4E3A312E30204D414348494E37
:1005A000455F545950453A4C756C7A426F742054EB
:1005B000415A20352045585452554445525F434FC7
:1005C000554E543A3120555549443A633332353506
:1005D0006339362D343039372D343838342D386579
:1005E00064302D6465643266663962616536310A4D
:1005F000002F2F20007A5F6D696E3A2000795F6DC1
:10060000696E3A2000785F6D696E3A20005265701D
:100610006F7274696E6720656E6473746F70207397
:1006200074617475730A004D31343520533C696E22
:100630006465783E206F7574206F662072616E6706
:10064000652028302D31290A00000000000000003C
:1006500000000000004F666673657473206170705F
:100660006C696564004572723A20546F6F20666150
:10067000722100546F6F206661722066726F6D2068
:100680007265666572656E636520706F696E740A67
:10069000004E6F2063617365206C696768740A009F
:1006A0004163746976652045787472756465723A41
:1006B0002000556E6B6E6F776E20636F6D6D616E8F
:1006C000643A20220020204E6F7A7A6C653A20002E
:1006D000200066696C616D656E7420756E6C6F616B
:1006E00064005761697420666F72005052494E541D
:1006F000205041555345440020204E6F7A7A6C6556
:100700003A20006368616E6765006F6620746865F3
:100710002066696C616D656E74005761697420664E
:100720006F72207374617274005052494E5420509D
:1007300041555345440020204E6F7A7A6C653A202B
:100740000020004261636B004D696E696D756D201C
:1007500054656D70206973203132302E0048656118
:1007600074696E67206661696C65640025753A2559
:1007700030327500253032753A25303275002575D6
:100780006420253032753A253032750000060900A4
:10079000FE000000000001090008FE000005080836
:1007A00006000040F0C88888987810050808060000
:1007B00000C0F88888888888F805050506000120AB
:1007C00030F830200508080600002070F8202020AE
:1007D00020E00509090600FF2070A8A8B8888870E5
:1007E000200509090600FFE080C0B0A828302828AD
:1007F0000509090600FFF8A88888888888A8F805F0
:100800000A0A0600FE205050505088A8A88870039D
:10081000030306000340A04000060900FE07019202
:10082000032120FFFF08FF07FF0000000600000172
:100830000707060200808080808000800302020695
:100840000105A0A00507070600005050F850F85019
:10085000500507070600002078A07028F020050743
:1008600007060000C0C810204098180507070600BA
:10087000006090A040A89068020303060104C040F5
:100880008003070706010020408080804020030786
:100890000706010080402020204080050505060055
:1008A0000120A870A8200505050600012020F820D9
:1008B000200203030602FFC0408005010106000379
:1008C000F8020202060200C0C00505050600010884
:1008D00010204080050707060000708888888888F7
:1008E0007003070706010040C040404040E0050794
:1008F00007060000708808708080F805070706006A
:1009000000F81020100808F0050707060000103056
:100910005090F81010050707060000F880F008084E
:100920008870050707060000708080F088887005D1
:100930000707060000F808102020202005070706FA
:1009400000007088887088887005070706000070AE
:10095000888878080870020505060200C0C000C03B
:10096000C00206060602FFC0C000C04080040707A0
:1009700006000010204080402010050303060002FE
:10098000F800F8040707060100804020102040808E
:1009900005070706000070880810200020050707DB
:1009A00006000070880868A8A87005070706000000
:1009B000708888F8888888050707060000F088880E
:1009C000F08888F00507070600007088808080881E
:1009D00070050707060000F08888888888F00507FA
:1009E00007060000F88080F08080F8050707060001
:1009F00000F88080F080808005070706000070887E
:100A000080B8888870050707060000888888F888FD
:100A1000888801070706020080808080808080052A
:100A20000707060000381010101090600507070631
:100A300000008890A0C0A0908805070706000080ED
:100A40008080808080F805070706000088D8A88885
:100A50008888880507070600008888C8A8988888BD
:100A600005070706000070888888888870050707D2
:100A7000060000F08888F0808080050707060000E7
:100A800070888888A89068050707060000F08888A5
:100A9000F0A090880507070600007880807008089D
:100AA000F0050707060000F8202020202020050779
:100AB0000706000088888888888870050707060070
:100AC00000888888888850200507070600008888E5
:100AD000888888A85005070706000088885020509D
:100AE0008888050707060000888888502020200590
:100AF0000707060000F80810204080F803070706E3
:100B00000100E08080808080E0050505060001800E
:100B100040201008030707060100E02020202020C5
:100B2000E0050303060004205088050101060000CB
:100B3000F802020206020580400505050600007065
:100B4000087888780507070600008080B0C8888884
:100B5000F00505050600007080808870050707060F
:100B60000000080868988888780505050600007068
:100B700088F880700507070600003048E0404040D4
:100B8000400506060600FF7088887808700507078C
:100B90000600008080B0C888888801070706020028
:100BA000800080808080800308080601FF200020EC
:100BB000202020A040040707060000808090A0C0ED
:100BC000A090030707060100C04040404040E005F8
:100BD0000505060000D0A8A8A8A805050506000080
:100BE000B0C8888888050505060000708888887068
:100BF0000506060600FFF08888F0808005060606D8
:100C000000FF788888780808050505060000B0C848
:100C100080808005050506000070807008F00407DC
:100C2000070600004040E040404030050505060052
:100C3000008888889868050505060000888888501F
:100C4000200505050600008888A8A85005050506AA
:100C5000000088502050880506060600FF88888816
:100C6000780870050505060000F8102040F8030715
:100C7000070601002040408040402001070706028F
:100C8000008080808080808003070706010080400C
:100C900040204040800502020600026890000000EB
:100CA0000600000000000600000000000600000032
:100CB0000000060000000000060000000000060022
:100CC0000000000006000000000006000000000018
:100CD0000600000000000600000000000600000002
:100CE00000000600000000000600000000000600F2
:100CF00000000000060000000000060000000000E8
:100D000006000000000006000000000006000000D1
:100D100000000600000000000600000000000600C1
:100D200000000000060000000000060000000000B7
:100D300006000000000006000000000006000000A1
:100D40000000060000000000060000000000060091
:100D50000000000006000000000006000000000087
:100D600006000000000006000001070706020080E0
:100D70000080808080800507070600002070A8A002
:100D8000A87020050707060000304040E04050A84A
:100D900005050506000088705070880507070600E5
:100DA00000885020F820F820010707060200808004
:100DB00080008080800508080600003048205050E0
:100DC000209060030101060107A005070706000047
:100DD000F888B8B8B888F8050707060001700878E1
:100DE000887800F80505050600012850A050280560
:100DF0000303060001F8080802020206020640800A
:100E0000050707060000F888A88898A8F8050101DA
:100E1000060006F8040404060003609090600507CD
:100E2000070600002020F8202000F8040505060031
:100E30000360902040F0030505060003E020E02059
:100E4000E002020206020640800508080600FF884C
:100E500088888898E88080050707060000789898B9
:100E600078181818020202060202C0C00202020626
:100E700002FF408003050506000340C04040E00536
:100E80000707060001708888887000F805050506C8
:100E90000001A0502850A00507070600008890A870
:100EA00058B808080507070600008890B848982039
:100EB00038050808060000C040C048D838080805B2
:100EC00007070600002000204080887005080806FB
:100ED00000004020007088F8888805080806000097
:100EE0001020007088F88888050808060000205047
:100EF000007088F88888050808060000689000706F
:100F000088F888880508080600005000708888F86E
:100F100088880508080600002050207088F8888816
:100F20000507070600003860A0B8E0A0B80508086B
:100F30000600FF7088808088702060050808060021
:100F400000402000F880F080F8050808060000083E
:100F50001000F880F080F805080806000020500016
:100F6000F880F080F80507070600005000F880F0D0
:100F700080F8030808060100804000E0404040E09F
:100F8000030808060100204000E0404040E003085C
:100F90000806010040A000E0404040E003070706CB
:100FA0000100A000E0404040E00507070600007097
:100FB0004848E8484870050808060000689000881E
:100FC000C8A898880508080600004020708888880E
:100FD00088700508080600001020708888888870CE
:100FE00005080806000020500070888888700508F1
:100FF0000806000068900070888888700508080658
:10100000000050007088888888700505050600017A
:1010100088502050880508080600FF1070A8A8A86E
:10102000A870400508080600004020888888888845
:1010300070050808060000102088888888887005D8
:101040000808060000205000888888887005080875
:101050000600005000888888888870050808060007
:101060000010208850202020200509090600FFC01C
:1010700040704848704040E00408080601FF609056
:1010800090A09090E08005080806000040200070C5
:101090000878887805080806000010200070087895
:1010A00088780508080600002050007008788878C5
:1010B0000508080600006890007008788878050721
:1010C00007060000500070087888780508080600B8
:1010D000002050207008788878050606060000D0A9
:1010E0002878A0A8500506060600FF7080887020AA
:1010F000600508080600004020007088F880700530
:1011000008080600001020007088F88070050808A4
:101110000600002050007088F88070050707060060
:101120000050007088F880700308080601008040B5
:101130000040C04040E00308080601002040004095
:10114000C04040E003080806010040A00040C04045
:1011500040E0030707060100A00040C04040E00552
:101160000707060000A040A0107888700508080650
:101170000000689000B0C88888880508080600004C
:10118000402000708888887005080806000010203C
:1011900000708888887005080806000020500070DC
:1011A00088888870050808060000689000708888A4
:1011B0008870050707060000500070888888700551
:1011C00005050600012000F800200507070600FFBE
:1011D0001070A8A8A870400508080600004020006C
:1011E000888888986805080806000010200088880C
:1011F00088986805080806000020500088888898AC
:101200006805070706000050008888889868050967
:10121000090600FF102000888888F8087004070776
:101220000601FFC04060506040E00508080600FF6E
:1012300050008888887808705A00590058000920A2
:10124000000000000000000000000000007FFFE040
:101250000000000000000000000000007000E0003E
:10126000000000000000000000000061F8600000C5
:101270000000000000000000000041F82000000015
:1012800000000000000000000040F020000000000E
:10129000000000000000000040602000000000008E
:1012A000000000000000005801A07F800000000046
:1012B0000000004104005C63A0FFC00000000000CB
:1012C00000002082005EF7A0FFC0000000000000C8
:1012D000002082005EF7A0FFC000000000000000B8
:1012E0004104005C63A07F800000000000000082D9
:1012F00008005801A07F80000000000000010410D9
:1013000000406020FFC00000000000000104100049
:1013100040F020FFC00000000000000082080041F3
:10132000F820FFC00000000000000041040061F848
:10133000603F00000000000000000000007000E0BE
:101340001E0000000000000001FFFF807FFFE00C96
:101350000000000000000001FFFF8000000000000E
:10136000000000000000000000007FFFE00000001F
:101370000000000000000000007000E0000000001D
:101380000000000000000000630C6000000000008E
:1013900000000000000000470E20000000000000D8
:1013A0000000000000004F0F2000000000000000BF
:1013B00000000000005F0FA000000000000000001F
:1013C000000000005E07A07F800000000000000019
:1013D000410400406020FFC0000000000000002029
:1013E000820040F020FFC0000000000000002082CA
:1013F0000040F020FFC00000000000000041040099
:101400004060207F80000000000000008208005E35
:1014100007A07F80000000000000010410005F0FA3
:10142000A0FFC0000000000000010410004F0F20CA
:10143000FFC000000000000000820800470E20FFEF
:10144000C000000000000000410400630C603F0089
:10145000000000000000000000007000E01E00001E
:10146000000000000001FFFF807FFFE00C00000093
:101470000000000001FFFF80000000534420636172
:101480007264206F6B0A006F70656E526F6F74200C
:101490006661696C65640A00766F6C756D652E69AE
:1014A0006E6974206661696C65640A005344206942
:1014B0006E6974206661696C0A0020643A002069D4
:1014C0003A0020703A0020643A0020693A00207007
:1014D0003A0020440020490020204D333034205071
:1014E0000020440020490020204D3330312050009E
:1014F0005049442073657474696E67733A0A00201A
:10150000460020420020480020204D313435205331
:10151000004D6174657269616C20686561747570F5
:1015200020706172616D65746572733A0A00205AA9
:101530000020590020204D323036205800486F6D71
:1015400065206F66667365743A0A00204500205A6C
:101550000020590020580020420020540020204D37
:10156000323035205300416476616E6365643A2001
:10157000533C6D696E5F66656564726174653E209B
:10158000543C6D696E5F74726176656C5F6665650B
:1015900064726174653E20423C6D696E5F7365677D
:1015A0006D656E745F74696D655F6D733E20583C48
:1015B0006D61785F78795F6A65726B3E205A3C6D29
:1015C00061785F7A5F6A65726B3E20453C6D617839
:1015D0005F655F6A65726B3E0A002054002052000E
:1015E00020204D323034205000416363656C6572B9
:1015F0006174696F6E2028756E6974732F73322958
:101600003A20503C7072696E745F616363656C3E32
:1016100020523C726574726163745F616363656CD0
:101620003E20543C74726176656C5F616363656CE7
:101630003E0A00204500205A0020590020204D324B
:1016400030312058004D6178696D756D20416363BC
:10165000656C65726174696F6E2028756E6974734C
:101660002F7332293A0A00204500205A00205900E1
:1016700020204D3230332058004D6178696D756DF2
:10168000206665656472617465732028756E69747F
:10169000732F73293A0A00204500205A0020590070
:1016A00020204D39322058005374657073207065C6
:1016B0007220756E69743A0A0020204D3230302055
:1016C00044300A0020204D3230302044002044694C
:1016D0007361626C65640A0046696C616D656E7465
:1016E0002073657474696E67733A0020204D31343D
:1016F000392043203B20556E69747320696E204366
:10170000656C736975730A002020473231202020F0
:10171000203B20556E69747320696E206D6D0A0040
:10172000205A3A0020593A0020436F756E742058B1
:101730003A0020453A00205A3A0020593A00583AD7
:1017400000656E7175657565696E6720220045726A
:10175000726F722077726974696E6720746F2045AA
:101760004550524F4D210A00486F6D652025732565
:1017700073257320666972737400206669727374CE
:101780000A005A0059005800486F6D652000000695
:101790000900FE06018902FE20FFFE07FE06FE008C
:1017A0000000060007010606060200808080800017
:1017B00080030303060103A0A0A00507070600FF9E
:1017C0005050F850F850500509090600FE2070A846
:1017D000A07028A870200608080600FF40A848103E
:1017E000204854080507070600FF60909060989015
:1017F000680103030602038080800207070602FFD8
:10180000408080808080400207070602FF804040C1
:10181000404040800505050600008850F8508805C6
:1018200005050600002020F820200204040602FE20
:10183000C0404080050101060002F80202020602D3
:1018400000C0C0040606060100101020408080047D
:10185000060606010060909090906003060606015F
:101860000040C0404040E0040606060100609010C1
:101870002040F0040606060100F020601010E0058C
:10188000060606000010305090F810040606060107
:1018900000F080E01010E00406060601006080E021
:1018A000909060040606060100F0101020404004ED
:1018B000060606010060906090906004060606012E
:1018C00000609090701060020505060200C0C00024
:1018D000C0C00207070602FEC0C000C0404080052D
:1018E0000505060000186080601805030306000166
:1018F000F800F8050505060000C0300830C00407F0
:1019000007060100609010604000400506060600D2
:10191000007090A8B0807005060606000020508870
:10192000F88888050606060000F088F08888F0042C
:10193000060606010060908080906004060606019D
:1019400000E090909090E0040606060100F080E030
:101950008080F0040606060100F080E080808004AC
:101960000606060100609080B0906004060606013D
:10197000009090F0909090030606060100E0404031
:101980004040E00506060600003810101090600484
:10199000060606010090A0C0A0909004060606016D
:1019A000008080808080F005060606000088D8A8A8
:1019B000A8888804060606010090D0B09090900593
:1019C00006060600007088888888700406060601EE
:1019D00000E09090E080800407070601FF6090908F
:1019E000D0B06010040606060100E09090E09090F0
:1019F0000406060601006090402090600506060679
:101A00000000F82020202020040606060100909007
:101A100090909060040606060100909090F060603F
:101A20000506060600008888A8A8D88805060606C8
:101A3000000088502020508805060606000088888F
:101A400050202020040606060100F010204080F0FF
:101A5000030606060100E080808080E0040606069A
:101A60000100808040201010030606060100E020DF
:101A7000202020E005030306000320508805010113
:101A80000600FEF802020206020480400404040676
:101A90000100709090700406060601008080E090BE
:101AA00090E00404040601007080807004060606BD
:101AB000010010107090907004040406010060B0E2
:101AC000C070040606060100205040E040400406B5
:101AD000060601FE60909070106004060606010084
:101AE0008080E09090900306060601004000C04010
:101AF00040E00308080601FE200060202020A040EE
:101B00000406060601008080A0C0A0900306060619
:101B10000100C040404040E0050404060000D0A899
:101B2000A888040404060100E090909004040406D0
:101B30000100609090600406060601FEE09090E0CF
:101B400080800406060601FE709090701010040458
:101B500004060100A0D0808004040406010070C0C7
:101B600030E00406060601004040E0405020040436
:101B70000406010090909070040404060100909007
:101B8000606005040406000088A8A8500404040648
:101B90000100906060900406060601FE909090702F
:101BA0009060040404060100F02040F003070706DB
:101BB0000100204040804040200107070602FF80CE
:101BC00080808080808003070706010080404020DD
:101BD00040408004020206010350A0FFFFFFFFFF08
:101BE000FFFFFFFFFFFFFFFFFFFFFFFFFFFFFFFF05
:101BF000FFFFFFFFFFFFFFFFFFFFFFFF00000006EB
:101C0000000701060606020080008080808004062E
:101C1000060601FF2070A0A070200507070600FF40
:101C2000304840F04040F8050505060000A85088FF
:101C300050A80506060600008850F820F820010785
:101C4000070602FF8080800080808004070706016D
:101C5000FF708060906010E0030101060105A0069E
:101C60000707060000788494A49484780305050689
:101C7000010160A06000E00505050600002850A0F5
:101C80005028040303060100F010100401010601AE
:101C900002F00607070600007884B4A4A484780440
:101CA0000101060105F004030306010260906005CE
:101CB00007070600FF2020F8202000F8030505068E
:101CC000010140A02040E0030505060101C02040BD
:101CD00020C002020206020440800405050601FF3E
:101CE0009090B0D08005060606000078E8E86828E5
:101CF00028010101060202800202020602FE408063
:101D000003050506010140C04040E003050506014A
:101D10000140A04000E0050505060000A050285045
:101D2000A00508080600FF40C0405070307810053C
:101D300008080600FF40C040506808103805080831
:101D40000600FFC0204030F030781004070706017D
:101D500000200020608090600507070600004020FA
:101D6000205070888805070706000010202050705A
:101D700088880507070600002050205070888805D5
:101D800007070600002850205070888805070706BE
:101D900000005000205070888805070706000020CA
:101DA00050205070888805060606000078A0F0A034
:101DB000A0B80408080601FE609080809060204072
:101DC0000407070601004020F080E080F0040707C8
:101DD0000601002040F080E080F0040707060100C3
:101DE0002050F080E080F00407070601005000F06A
:101DF00080E080F00307070601008040E04040409B
:101E0000E00307070601002040E0404040E00307F0
:101E10000706010040A0E0404040E003070706013C
:101E200000A000E0404040E00506060600007048C3
:101E3000E848487004070706010050A090D0B09011
:101E4000900407070601004020609090906004070E
:101E5000070601002040609090906004070706018B
:101E6000002050609090906004070706010050A089
:101E70006090909060040707060100500060909009
:101E80009060050505060000885020508804080869
:101E90000601FF1070B0B0D0D0E080040707060143
:101EA00000402090909090600407070601002040B9
:101EB0009090909060040707060100205090909049
:101EC0009060040707060100500090909090600514
:101ED0000707060000102088502020200406060670
:101EE000010080E09090E08004060606010060900A
:101EF000A0A090A004070706010040200070909069
:101F000070040707060100204000709090700407DD
:101F1000070601002050007090907004070706012A
:101F20000050A0007090907004060606010050005A
:101F30007090907004070706010020502070909068
:101F40007005040406000070A8B0780406060601B7
:101F5000FE708080702040040707060100402000CA
:101F600060B0C07004070706010020400060B0C0E8
:101F70007004070706010020500060B0C07004061E
:101F800006060100500060B0C0700307070601009C
:101F9000804000C04040E0030707060100204000E9
:101FA000C04040E003070706010040A000C04040D9
:101FB000E0030606060100A000C04040E004070759
:101FC0000601003060107090906004070706010061
:101FD00050A000E090909004070706010040200008
:101FE0006090906004070706010020400060909018
:101FF000600407070601002050006090906004070D
:102000000706010050A000609090600406060601DB
:10201000005000609090600505050600002000F863
:10202000002004040406010070B0D0E00407070695
:1020300001004020009090907004070706010020E6
:102040004000909090700407070601002050009017
:102050009090700406060601005000909090700465
:1020600009090601FE2040009090907090600408DD
:10207000080601FE8080E09090E080800408080659
:1020800001FE5000909090709060000022002500AA
:1020900028002B002E003100340002010000050151
:1020A00008010B0100000A0B02090C0D0E080703C2
:1020B000040100000000000000000000000000001B
:1020C0000000000000000000000000000000000010
:1020D00012111000000000000000000000000000CD
:1020E0000000000000000000000043290A006162B7
:1020F0006C656420286D696E2074656D70200043E6
:102100006F6C6420657874727564657320617265A4
:10211000200045313A200045303A20005A3A20004C
:10212000593A2000583A20004D53312C4D5332205B
:1021300050696E730A00506C656173652072657337
:102140006574005052494E5445522048414C544504
:1021500044005072696E7465722068616C746564C5
:102160002E206B696C6C28292063616C6C6564217E
:102170000A006265640A002C2073797374656D200F
:1021800073746F7070656421204865617465725F57
:1021900049443A2000544845524D414C2052554E36
:1021A000415741592042454400546865726D616C45
:1021B0002052756E6177617900544845524D414C0B
:1021C0002052554E415741592045310054484552FF
:1021D0004D414C2052554E41574159204530004801
:1021E000656174696E67206661696C65642042454B
:1021F000440048656174696E67206661696C656456
:102200000048656174696E67206661696C65640089
:1022100048656174696E67206661696C6564204514
:10222000300057726974696E6720746F2066696C3C
:10223000653A20006F70656E206661696C65642C7C
:102240002046696C653A20006F70656E2066616992
:102250006C65642C2046696C653A200046696C65A3
:102260002073656C65637465640A002053697A6540
:102270003A200046696C65206F70656E65643A208F
:10228000006F70656E206661696C65642C2046691C
:102290006C653A20002066696C653A20004E6F77C5
:1022A00020002220706F73002220706172656E74AE
:1022B0003A2200535542524F5554494E452043410E
:1022C0004C4C207461726765743A22004B494C4C47
:1022D00045442E2000747279696E6720746F206304
:1022E000616C6C207375622D67636F64652066692D
:1022F0006C6573207769746820746F6F206D616EF0
:1023000079206C6576656C732E204D4158206C6584
:1023100076656C2069733A000000200023002600D7
:1023200029002C002F0032000001000003010601EB
:102330000901000000000000000000000000000093
:10234000954300008A4300007A437C3C3E5E2B3D6F
:102350003F2F5B5D3B2C2A225C0043616E6E6F74E5
:10236000206F70656E2073756264697220000105CC
:102370000800FF060121023520FFFF07FF06FF09C5
:102380000050221656808080800080153353A0A014
:10239000A00257575050F850F8505002575720702D
:1023A000A07028702013355580A040A02002475708
:1023B00040A0A040A0A05025135380808012265634
:1023C00040808080804012265680404040408002FD
:1023D00045559060F060900255552020F82020115E
:1023E0003353604080044151F011335340E04002C8
:1023F000465610102040808012365640A0A0A0A063
:102400004012365640C0404040E0024656609010B0
:102410006080F0024656F020601090600246562020
:1024200060A0F02020024656F080E0109060024646
:10243000566080E0909060024656F01020204040A8
:102440000246566090609090600246566090907090
:102450001060122555C0C000C0C011365660600023
:10246000604080123656204080804020034353F065
:1024700000F012365680402020408012365640A090
:1024800020400040015858304898A8A89040300299
:102490004656609090F09090024656E090E0909002
:1024A000E0024656609080809060024656E0909030
:1024B0009090E0024656F080E08080F0024656F0B0
:1024C00080E0808080024656609080B09060024636
:1024D000569090F0909090123656E040404040E088
:1024E00002465670202020A04002465690A0C0A070
:1024F000A0900246568080808080F002465690F080
:10250000F090909002465690D0F0B0B090024656AF
:10251000609090909060024656E09090E08080013C
:102520004757609090D0B06010024656E09090E01F
:102530009090024656609040209060123656E040DF
:10254000404040400246569090909090600246561F
:10255000909090906060024656909090F0F09002BB
:102560004656909060609090025656888850202081
:1025700020024656F010204080F0123656E080804F
:102580008080E0024656808040201010123656E0CF
:1025900020202020E016325240A0014151F01622A6
:1025A000528040024454709090700246568080E001
:1025B0009090E01234546080806002465610107093
:1025C00090907002445460B0C06002465620504063
:1025D000E040400145556090701060024656808092
:1025E000E09090901236564000C04040E0113757BE
:1025F0002000202020A040024656808090E090904D
:10260000123656C040404040E0025454D0A8A8A81A
:10261000024454E0909090024454609090600145D0
:1026200055E090E080800145557090701010024494
:1026300054A0D0808012345460C020C0024656405E
:1026400040E040502002445490909070123454A0C6
:10265000A0A04002545488A8A8500244549060603E
:10266000900145559090709060024454F02040F0E5
:10267000024757304020C0204030221656808080CC
:10268000808080024757C02040304020C006425220
:1026900050A0FFFFFFFFFFFFFFFFFFFFFFFFFFFF58
:1026A000FFFFFFFFFFFFFFFFFFFFFFFFFFFFFFFF3A
:1026B000FFFFFF09005022165680008080808001B5
:1026C00046562070A0A070200246562050E0405090
:1026D000A002555588705070880256568850F820D0
:1026E000F820221757808080008080800247577032
:1026F00080E0907010E0173151A002565670A8C8C3
:10270000C8A87014355560A06000E003435350A082
:1027100050123353E02020143151E002565670E835
:10272000D8E8D870173151E015335340A040123526
:102730005540E04000E014355540A02040E01435FD
:1027400055C020C020C016225240800145559090AF
:1027500090E08002565678E8E868282824115180D5
:10276000112252408014355540C04040E014355588
:1027700040A04000E0034353A050A0024757808090
:1027800080A060F0200247578080A0D01020700207
:10279000475780408060A0F02012365640004080AD
:1027A000A04002475740206090F090900247572089
:1027B000406090F0909002475760906090F0909049
:1027C00002475750A06090F09090024757900060E9
:1027D00090F0909002475760906090F09090024681
:1027E0005670A0A0F0A0B001475760908080906024
:1027F000400247574020F080E080F00247572040D9
:10280000F080E080F00247576090F080E080F002B6
:1028100047579000F080E080F01237578040E0404A
:102820004040E01237572040E0404040E012375728
:1028300040A0E0404040E0123757A000E040404058
:10284000E00256567048E848487002475750A0903A
:10285000D0B090900247574020609090906002471F
:102860005720406090909060024757609060909031
:10287000906002475750A060909090600247579038
:10288000006090909060123353A040A002465670B2
:10289000B0B0D0D0E00247574020909090906002B6
:1028A00047572040909090906002475760909090DA
:1028B0009090600247579000909090906002575718
:1028C0001020885020202002465680E09090E08022
:1028D0000246566090A0A090A0024757402000708A
:1028E00090907002475720400070909070024757B8
:1028F0002050007090907002475750A00070909048
:102900007002465650007090907002475760906079
:1029100070909070025454F068B078113555608012
:1029200080604002475740200060B0C060024757B7
:1029300020400060B0C06002475760900060B0C0A7
:1029400060024656500060B0C060123757804000A9
:10295000C04040E0123757204000C04040E01237EE
:102960005740A000C04040E0123656A000C0404092
:10297000E0024757A040A01070906002475750A057
:1029800000E09090900247574020006090906002D5
:102990004757204000609090600247576090006069
:1029A00090906002475750A0006090906002465699
:1029B0009000609090601235554000E00040024465
:1029C0005470B0D0E00247574020009090907002C1
:1029D00047572040009090907002475760900090B9
:1029E0009090700246569000909090700148582048
:1029F000400090907090600147578080E090E080A8
:102A0000800147579000909070906001050700FE8C
:102A10000500FB01F220FFFE05FE05FE020040025C
:102A200015258080800080053242A0A002556550A7
:102A3000F850F8500146562070C030E0200255652D
:102A40009010204048025565608068906805122209
:102A500080800225354080808040022535804040BE
:102A60004080043343A040A003334340E0400122B0
:102A7000324080043141E002112180025565081086
:102A80002040800245556090909060022535C040FE
:102A9000404040024555E0106080F0024555E0108E
:102AA0006010E00245552060A0F020024555F080FE
:102AB000E010E00245556080E09060024555F0105E
:102AC00020404002455560906090600245556090FE
:102AD0007010600313238000800214248000808023
:102AE0000235452040804020033343E000E00235BA
:102AF000458040204080024555E01060004002556E
:102B0000657088B8A870024555609090F0900245B5
:102B100055E090E090E0023545608080806002459D
:102B200055E0909090E0023545E080E080E002358D
:102B300045E080E080800245557080B0907002458D
:102B4000559090F09090023545E0404040E00245BD
:102B500055301010906002455590A0C0A0900235ED
:102B60004580808080E002556588D8A88888024525
:102B70005590D0B09090024555609090906002457D
:102B800055E09090E0800146566090909060100271
:102B90004555E09090E09002455570806010E0024D
:102BA0003545E0404040400245559090909060028D
:102BB00045559090A0A04002556588A8A8A850024D
:102BC000455590906090900245559090701060022D
:102BD0003545E0204080E0022535C0808080C0027D
:102BE00055658040201008022535C0404040C00592
:102BF000324240A0024151F005223280400244544A
:102C00007090907002455580E09090E002344460EE
:102C1000808060024555107090907002445460B0FE
:102C2000C0600235452040E040400046567090901C
:102C300070106002455580E090909002152580004C
:102C4000808080002737400040404040800245554A
:102C50008090A0E0900215258080808080025464DE
:102C6000F0A8A8A8024454E09090900244546090C8
:102C70009060004656E09090E0808000465670904C
:102C800090701010023444A0C0808002445470C080
:102C900030E002354540E04040200244549090909E
:102CA000700244549090A040025464A8A85050026E
:102CB0003444A04040A000465690909070106002AE
:102CC0004454F02040F002354560408040600215D9
:102CD000258080808080023545C0402040C005426C
:102CE0005250A0FFFFFFFFFFFFFFFFFFFFFFFFFFAF
:102CF000FFFFFFFFFFFFFFFFFFFFFFFFFFFFFFFFE4
:102D0000FFFFFFFF020040FFFFFFFFFFFFFFFFFF8E
:102D1000FFFFFFFFFFFFFFFFFFFFFFFFFFFFFFFFC3
:102D2000FFFFFFFFFFFFFFFFFFFFFFFFFFFFFFFFB3
:102D3000FFFFFFFFFFFFFFFFFFFFFFFFFFFFFFFFA3
:102D4000FFFFFFFFFFFFFFFFFFFFFFFFFFFFFFFF93
:102D5000FFFFFFFFFFFFFFFFFFFFFFFFFFFFFFFF83
:102D6000FFFFFFFFFFFF01060D00FE09016602D60F
:102D700020FFFE0BFE0AFE0D006022196980808094
:102D8000808080800080183363A0A0A00357675024
:102D900050F850F850500259692078A0A0702828A7
:102DA000F02002596948A85010204050A8900258BD
:102DB0006840A0A040A0989068281363808080118C
:102DC0003B6B2040408080808080404020113B6BE6
:102DD000804040202020202040408006556520A8CB
:102DE00070A8200455652020F8202011336360402E
:102DF00080065161F811336340E0400259690808C8
:102E000010102040408080025969205088888888AE
:102E10008850200259692060A02020202020F8023C
:102E200059697088880810204080F8025969F808AC
:102E300010207008088870025969101030505090A6
:102E4000F81010025969F88080B0C808088870022C
:102E5000596970888080F088888870025969F808FC
:102E6000101020204040400259697088888870887E
:102E70008888700259697088888878080888701175
:102E8000386840E040000040E04011386840E040D1
:102E900000006040800259690810204080402010E6
:102EA00008045464F80000F80259698040201008B2
:102EB0001020408002596970888808102020002066
:102EC00002596970888898A8A8B08078025969204A
:102ED00050888888F8888888025969F0484848707E
:102EE000484848F0025969708880808080808870E6
:102EF000025969F048484848484848F0025969F87A
:102F0000808080F0808080F8025969F8808080F0AD
:102F1000808080800259697088808080988888705D
:102F200002596988888888F888888888123969E011
:102F300040404040404040E00259693810101010B5
:102F400010109060025969888890A0C0A09088886D
:102F50000259698080808080808080F80259698869
:102F600088D8A8A88888888802596988C8C8A8A865
:102F700098988888025969708888888888888870B5
:102F8000025969F0888888F080808080015A6A70D0
:102F9000888888888888A87008025969F088888895
:102FA000F0A090888802596970888080700808882D
:102FB00070025969F8202020202020202002596921
:102FC000888888888888888870025969888888886D
:102FD000505050202002596988888888A8A8A8A83D
:102FE0005002596988885050205050888802596989
:102FF000888850502020202020025969F80810109D
:1030000020404080F8113B6BE08080808080808091
:103010008080E0025969808040402010100808112B
:103020003B6BE0202020202020202020E00853635C
:10303000205088015161F82A226280400256667051
:103040000878889868025969808080F08888888824
:10305000F0025666708880808870025969080808F6
:103060007888888888780256667088F88088700228
:10307000596930484040F0404040400058687088EE
:10308000888878088870025969808080B0C88888EC
:1030900088881238684000C040404040E0004A6ADA
:1030A00010003010101010909060025969808080DC
:1030B00090A0C0A09088123969C040404040404074
:1030C00040E0025666D0A8A8A8A888025666B0C8F4
:1030D0008888888802566670888888887000586852
:1030E000F0888888F08080800058687888888878A0
:1030F000080808025666B0C8808080800256667054
:1031000088601088700258684040F0404040483065
:10311000025666888888889868025666888888502B
:1031200050200256668888A8A8A850025666885083
:10313000202050880058688888889868088870021D
:103140005666F810204080F8015B6B182020202084
:10315000C0202020201822196980808080808080F3
:103160008080015B6BC0202020201820202020C000
:1031700008536348A890FFFFFFFFFFFFFFFFFFFF1B
:10318000FFFFFFFFFFFFFFFFFFFFFFFFFFFFFFFF4F
:10319000FFFFFFFFFFFFFF0D006022196980008025
:1031A0008080808080800358682070A8A0A0A870CC
:1031B0002002596930484040E0404048B00356661C
:1031C00088705050708802596988885050F820F8EB
:1031D0002020221969808080800080808080124AAF
:1031E0006A609080609090601090601A3262A0A037
:1031F0000359697088A8D8C8D8A888700457677020
:103200000878887800F80356662850A0A050280453
:103210005363F80808163161E00359697088E8D8EB
:10322000D8E8D888700A5161F817446460909060BB
:103230000357672020F8202000F807356540A020BC
:1032400040E007356540A04020C02A22624080004F
:1032500058688888888898E8808002596978E8E802
:10326000E8E868282828262161C0202262408007DB
:10327000356540C04040E00457677088888870001A
:10328000F8035666A050282850A0025A6A40C04051
:1032900040E00818283808025A6A40C04040E01050
:1032A00028081038025A6A40A04020A04818283840
:1032B00008025969200020204080888870025A6ADC
:1032C00040200020508888F88888025A6A10200020
:1032D00020508888F88888025A6A30480020508830
:1032E00088F88888025A6A28500020508888F88810
:1032F00088025A6A50500020508888F88888025AFC
:103300006A20502020508888F8888802596958A07F
:10331000A0A0B0E0A0A0B8005B6B70888080808027
:103320008088702040025A6A402000F88080F08037
:1033300080F8025A6A102000F88080F08080F8023D
:103340005A6A304800F88080F08080F8025A6A504B
:103350005000F88080F08080F8123A6A804000E0E7
:103360004040404040E0123A6A204000E040404087
:103370004040E0124A6A609000E04040404040E037
:10338000123A6AA0A000E04040404040E002596983
:10339000F0484848E8484848F0025A6A28500088EF
:1033A00088C8A8988888025A6A402000708888884F
:1033B000888870025A6A102000708888888888700F
:1033C000025A6A30480070888888888870025A6A71
:1033D00028500070888888888870025A6A50500087
:1033E00070888888888870035565885020508801C7
:1033F0005B6B08709898A8A8A8C8C87080025A6A21
:1034000040200088888888888870025A6A102000C6
:1034100088888888888870025A6A30480088888836
:1034200088888870025A6A505000888888888888FE
:1034300070025A6A102000888850202020200259EB
:103440006980F0888888F080808002596960909057
:10345000A0A0908888B00259694020007008788840
:103460009868025969102000700878889868025995
:1034700069304800700878889868025969285000B7
:1034800070087888986802596950500070087888E8
:103490009868025A6A304830007008788898680244
:1034A0005666702870A0A850005868708880808880
:1034B0007020400259694020007088F880887002AE
:1034C00059691020007088F8808870025969304866
:1034D000007088F88088700259695050007088F830
:1034E000808870123969804000C040404040E0123E
:1034F0003969204000C040404040E0124969609076
:1035000000C040404040E0123969A0A000C04040E7
:103510004040E0025A6A50206010708888888870A5
:10352000025969285000B0C88888888802596940C3
:10353000200070888888887002596910200070887F
:103540008888887002596930480070888888887037
:10355000025969285000708888888870025969501B
:103560005000708888888870035767202000F80012
:103570002020015868087098A8A8C870800259696E
:10358000402000888888889868025969102000883F
:10359000888888986802596930480088888888989F
:1035A00068025969505000888888889868005B6B69
:1035B0001020008888889868088870005A6A80807F
:1035C000B0C88888C8B08080005B6B505000888885
:1035D0008898680888700000000000000000000063
:1035E00000000000000000000000000000000000DB
:1035F0000000000000000000000C000000000000BF
:10360000000C00000000000000120000000000009C
:103610000023000000000000002100000000000066
:10362000004C800000000000005E800000000000F0
:10363000009240000000000000A1400000000000D7
:103640000121200000000000027F90000000000027
:10365000020010000000000007FFF800000000005A
:103660000400080000000000080004000000000042
:10367000080006000000000010000200000000002A
:10368000301E010000000000207F810000000000CB
:1036900041FFE0800000000043FCF08000000000DB
:1036A000873B7840000000018EDBFC6000000001D9
:1036B0000FEBCC20000000021FEDB610000000024E
:1036C0001FDEB6100000000439CD7F0800000004A2
:1036D00036E0FF08000000087EC0BB840000001830
:1036E0007F005D86000000107FC0ED82000000209A
:1036F0003CC07301000000203B337F0100000070DC
:103700001BE77E03800000C81DEEDE04C0000088B9
:103710000FDEDC04400001240FDF3C0920000126FD
:1037200007DBF8192000027203E7F0139000025142
:1037300001FFE02290000489007F802448000904F2
:10374000801E004824000BFE400000DFF400100043
:103750004000008002001FFFFFFFFFFFFE0000008F
:103760000000000000000000000000000000000059
:103770000000000000001022103C3C0E1F00102230
:10378000100422110400102210082211040010223B
:1037900010083C1104001022101022110400102205
:1037A0001020221104001E1C1E3C3C0E04000000D0
:1037B0000000000000000000000000000000000009
:1037C00000000000000000000000000000000000F9
:1037D00000000000000000000000000000000000E9
:1037E00000000000000000000000000000000000D9
:1037F00000000000000000000000000000000000C9
:1038000000000000000000000000000000000000B8
:10381000000000004D6F76652058004D6F766520E2
:1038200059004D6F7665205A00457874727564654D
:1038300072001000C90210012C0140012201700128
:103840001801B0010E01F00104015002FA00B002AB
:10385000F0003003E600D003DC009004D2007005D5
:10386000C800A006BE000008B400B009AA00D00B32
:10387000A000600E960060118C00001582002019D7
:103880007800C01D6E00A0226400B0275A00902C62
:10389000500000314600E0343C0010383200903ACD
:1038A0002800603C1E00A03D1400803E0A00203F1E
:1038B00000001000AD0330016A0150022B017003BB
:1038C0000A019004F500B005E500D006D800F00725
:1038D000CE001009C500300ABE00500BB700700CB6
:1038E000B100900DAB00B00EA600D00FA200F010FA
:1038F0009D0010129900301395005014920070151D
:103900008E0090168B00B0178700D0188400F01935
:103910008100101B7E00301C7B00501D7900701E42
:103920007600901F7300B0207000D0216E00F0224E
:103930006B00102469003025660050266300702754
:10394000610090285E00B0295C00D02A5900F02B5D
:103950005600102D5400302E5100502F4E00703064
:103960004B0090314800B0324500D0334200F03473
:103970003E0010363B003037370050383300703986
:103980002E00903A2900B03B2300D03C1B00F03DB4
:103990001100103F0100F03F000043616E6E6F7434
:1039A00020656E746572207375626469723A2000D6
:1039B000022E2E004D61696E004D6F766520302E0F
:1039C000316D6D004D6F766520316D6D004D6F76F8
:1039D000652031306D6D004D6F76652061786973BB
:1039E000004578747275646572004D6F7665205A73
:1039F000004D6F76652059004D6F76652058007434
:103A00006F20726573756D65005761697420666F0C
:103A100072207072696E74005052494E54205041A9
:103A2000555345440045787472756465206D6F7216
:103A30006500526573756D65207072696E74005211
:103A40004553554D45204F5054494F4E533A002051
:103A5000204E6F7A7A6C653A20002000506C6561C8
:103A6000736520776169742E2E2E00486561746934
:103A70006E67206E6F7A7A6C65005052494E542002
:103A80005041555345440020204E6F7A7A6C653A78
:103A90002000200068656174206E6F7A7A6C652E54
:103AA00000507265737320627574746F6E20746F4A
:103AB000005052494E542050415553454400202057
:103AC0004E6F7A7A6C653A2000200066696C616DF1
:103AD000656E7420657874727564650057616974E9
:103AE00020666F72005052494E5420504155534544
:103AF000440020204E6F7A7A6C653A2000200066E0
:103B0000696C616D656E74206C6F616400576169EA
:103B10007420666F72005052494E542050415553E4
:103B200045440020204E6F7A7A6C653A2000746F0D
:103B300020636F6E74696E75652E2E2E00616E6443
:103B400020707265737320627574746F6E00496EB5
:103B5000736572742066696C616D656E7400505295
:103B6000494E5420504155534544000000954300B0
:103B7000008A4300007A43000048420000484200A7
:103B800000404000000000FFFFFF5A2070726F628B
:103B900065206F75742E206265640A005A20707269
:103BA0006F6265206F75742E2062656400486F6DCA
:103BB000652058592066697273740A00486F6D65F4
:103BC000205859206669727374004F6666004F6E04
:103BD0002000456E6473746F702061626F727400B0
:103BE00053746570732F6D6D004A65726B0041638D
:103BF00063656C65726174696F6E0056656C6F63A6
:103C000069747900416476616E63656420536574FC
:103C100074696E6773005654726176206D696E0028
:103C20005654726176206D696E005654726176202A
:103C30006D696E00566D696E00566D696E00566D49
:103C4000696E00566D6178204500566D617820459B
:103C500000566D6178204500566D6178205A0056F7
:103C60006D6178205A00566D6178205A00566D615A
:103C700078205900566D6178205900566D61782082
:103C80005900566D6178205800566D6178205800B3
:103C9000566D61782058004D6F74696F6E004573E2
:103CA000746570732F6D6D004573746570732F6D3F
:103CB0006D005A73746570732F6D6D005A7374655F
:103CC00070732F6D6D005973746570732F6D6D0077
:103CD0005973746570732F6D6D00587374657073CC
:103CE0002F6D6D005873746570732F6D6D004D6F7F
:103CF00074696F6E0056652D6A65726B0056652D8E
:103D00006A65726B0056652D6A65726B00567A2D76
:103D10006A65726B00567A2D6A65726B0056792D52
:103D20006A65726B0056792D6A65726B0056792D43
:103D30006A65726B0056782D6A65726B0056782D35
:103D40006A65726B0056782D6A65726B004D6F74F0
:103D5000696F6E000200002100240027002A002D58
:103D6000003000330001010000040107010A0101D5
:103D7000021020200808102040102040800201027C
:103D80000108040201010204081020408080402044
:103D9000100804020180040201804020100804027F
:103DA00001080402010102040810204080010204FD
:103DB00008102040800505050507050808080802C9
:103DC0000202020A0A0808040404040101010101B4
:103DD0000101010303030303030303040707070CA3
:103DE0000C0C0C0C0C0C0C02020202060606060659
:103DF0000606060B0B0B0B0B0B0B0B1FFFFFFFFF3E
:103E0000FFFF600000000001FF400000000000FF15
:103E10008000000000007F83CF00000C303F87FF50
:103E200080000C301F867980000C000F8C30C78317
:103E30008C30E78C30CFC7CC31F38C30DCECEC33FA
:103E4000B98C30D86C6C33198C30D06C0C33198C25
:103E500030D86C0C33198C30DC6C0E3B198C30CFA5
:103E60007C079F198C30C77C038F1940000000002D
:103E70000002600000000000061FFFFFFFFFFFF8C8
:103E80002020506C616E6E65724275666665724286
:103E9000797465733A20002046726565204D656D22
:103EA0006F72793A2000436F6D70696C65643A20D7
:103EB0004E6F7620323120323031370A00207C209C
:103EC000417574686F723A2028416C657068204FA4
:103ED000626A6563747320496E632E2C204C756C86
:103EE0007A426F7420476974205265706F736974E9
:103EF0006F7279290A004E6F7620323120323031CC
:103F00003731333A33313A343200204C6173742004
:103F1000557064617465643A2000312E312E350A83
:103F2000004D61726C696E0020536F667477617228
:103F3000652052657365740A002057617463686474
:103F40006F672052657365740A002042726F776E46
:103F5000206F75742052657365740A00204578746B
:103F600065726E616C2052657365740A00506F77DC
:103F7000657255700A0073746172740A006572721A
:103F80006F722077726974696E6720746F2066693A
:103F90006C650A004572726F723A00456E64737404
:103FA0006F7073202563202563202563202563001F
:103FB000205A3A0020593A0020583A00656E64733E
:103FC000746F7073206869743A20006563686F3A93
:103FD00000446F6E6520736176696E672066696C58
:103FE000652E0A004D3239004D36303020486F744E
:103FF000656E6420746F6F20636F6C6420746F2033
:104000006368616E67652066696C616D656E740AD0
:10401000004B64200023646566696E65202044457A
:104020004641554C545F004B692000236465666926
:104030006E65202044454641554C545F004B70202E
:104040000023646566696E65202044454641554CF1
:10405000545F00504944204175746F74756E65203B
:1040600066696E6973686564212050757420746890
:1040700065206C617374204B702C204B6920616E3D
:1040800064204B6420636F6E7374616E747320667A
:10409000726F6D2062656C6F7720696E746F20435C
:1040A0006F6E66696775726174696F6E2E680A005B
:1040B000504944204175746F74756E65206661695E
:1040C0006C6564212074696D656F75740A005049D0
:1040D00044204175746F74756E65206661696C6506
:1040E00064212054656D7065726174757265207409
:1040F0006F6F20686967680A00204B643A200020CF
:104100004B693A2000204B703A20000A20436C6132
:104110007373696320504944200A002054753A2083
:1041200000204B753A2000206D61783A2000206D08
:10413000696E3A200020643A200020626961733A77
:104140002000436172642072656D6F766564004380
:1041500061726420696E736572746564004861728F
:1041600064636F6465642044656661756C74205394
:10417000657474696E6773204C6F616465640A00CE
:1041800028230000282300006400000010270000FE
:104190000000964300009643000040400000C841E4
:1041A0000000C9420000C9420000C84400804F44DA
:1041B000202863616C63756C6174656429210A0051
:1041C00020213D2000454550524F4D204352432071
:1041D0006D69736D61746368202D202873746F722C
:1041E0006564292000290A002062797465733B20E8
:1041F00063726320002073746F726564207365744A
:1042000074696E677320726574726965766564207F
:104210002800204D61726C696E3D563430290A00C9
:1042200028454550524F4D3D00454550524F4D2079
:1042300076657273696F6E206D69736D6174636802
:1042400020004B494C4C45442E200024F4D43050DF
:10425000C38E20C2A24017828B7011127A910D81F9
:104260006CD90AA861E108C7586607615143061E68
:104270004B5D05C145A7041A411104093D9803711E
:104280003931034036DB0265339102D43054028069
:104290002E1D02632CEE01752AC501B028A0011065
:1042A0002781018F2564012B244B01E0223401ACCE
:1042B000211F018D200D01801FFC00841EED009741
:1042C0001DDF00B81CD200E61BC600201BBC00642A
:1042D0001AB200B219A8000A19A0006A189900D1F0
:1042E00017910040178B00B516840031167E00B37D
:1042F0001579003A157300C7146F0058146A00EE60
:104300001366008813630025135E00C7125B006C00
:1043100012570015125400C111510070114F0021A5
:10432000114B00D61049008D104700461044000282
:10433000104200C00F4000800F3E00420F3C0006BC
:104340000F3B00CB0E3800930E37005C0E35002774
:104350000E3400F30D3200C10D3100900D300060BD
:104360000D2E00320D2D00050D2C00D90C2B00AEAA
:104370000C2900850C29005C0C2700350C27000E49
:104380000C2600E80B2400C40B2400A00B23007DA6
:104390000B23005A0B2100390B2100180B2000F8C9
:1043A0000A1F00D90A1E00BB0A1E009D0A1D0080BC
:1043B0000A1D00630A1C00470A1B002C0A1B00117F
:1043C0000A1A00F7091A00DD091900C4091900AB1F
:1043D000091900920917007B091800630917004C9E
:1043E00009160036091600200916000A091500F5FD
:1043F000081500E0081400CC081400B8081400A444
:10440000081400900813007D0812006B0813005870
:104410000812004608120034081100230811001287
:1044200008110001081100F0071000E0071000D08B
:10443000071000C0071000B0070F00A1071000917F
:10444000070E0083070F0074070F0065070E005763
:10445000070E0049070E003B070D002E070E002037
:10446000070D0013070D0006070D00F9060C00EDFF
:10447000060D00E0060C00D4060C00C8060C00BCBB
:10448000060C00B0060C00A4060B0099060C008D6B
:10449000060B0082060B0077060B006C060B006112
:1044A000060A0057060B004C060A0042060A0038AE
:1044B000060A002E060A0024060A001A060A001040
:1044C00006090007060A00FD050900F4050900EBCE
:1044D000050900E2050900D9050900D0050900C752
:1044E000050900BE050900B5050800AD050800A5D1
:1044F0000509009C050800940508008C0508008447
:104500000508007C050800740508006C05070065B7
:104510000508005D050700560508004E0507004721
:104520000507004005080038050700310507002A87
:10453000050700230507001C050600160507000FE8
:104540000507000805060002050700FB040600F544
:10455000040700EE040600E8040600E2040700DB9E
:10456000040600D5040600CF040600C9040600C3F3
:10457000040600BD040600B7040600B1040500AC43
:10458000040600A6040600A00405009B040600958E
:10459000040500900406008A0405008504050080D7
:1045A0000406007A04050075040500700405006B1C
:1045B00004050066040500610405005C040500575D
:1045C000040500520405004D04050048040500439D
:1045D0000405003E0404003A0405003504050030DB
:1045E0000404002C04050027040400230405001E15
:1045F0000404001A04040016040500110404000D4C
:10460000040400090405000404040000040400FC80
:10461000030400F8030400F4030400F0030400ECB6
:10462000030400E8030400E4030400E0030400DCE6
:10463000030400D8030400D4030400D0030400CC16
:10464000030400C8030300C503030024F404D920B5
:104650001BC40C5C0E9804C4095F0265077101F469
:1046600005F900FB04B30048048700C10369005842
:1046700003550003034500BE023A00840231005393
:10468000022A002902250004022000E4011C00C8BF
:10469000011900AF01170098011400840113007183
:1046A0000110006101100051010E0043010D0036A0
:1046B000010B002B010B0020010B00150109000C60
:1046C00001090003010800FB000800F3000800EBEB
:1046D000000700E4000600DE000600D8000600D255
:1046E000000600CC000500C7000500C2000500BDA3
:1046F000000400B9000400B5000400B1000400ADDE
:10470000000400A9000400A5000300A20003009F0C
:104710000004009B00030098000300950002009332
:10472000000300900003008D0002008B000300884E
:104730000002008600020084000300810002007F66
:104740000002007D0002007B000200790002007779
:104750000001007600020074000200720001007186
:104760000002006F0002006D0001006C0002006A90
:104770000001006900020067000100660001006599
:10478000000100640002006200010061000100609D
:104790000001005F0002005D0001005C0001005BA1
:1047A0000001005A000100590001005800010057A3
:1047B00000010056000100550001005400010053A3
:1047C00000000053000100520001005100010050A0
:1047D0000001004F0001004E0000004E0001004D9E
:1047E0000001004C0001004B0000004B0001004A9A
:1047F0000001004900010048000000480001004796
:104800000001004600000046000100450000004590
:104810000001004400010043000000430001004289
:104820000000004200010041000000410001004082
:104830000001003F0000003F0001003E0000003E7C
:104840000001003D0000003D0001003C0000003C74
:104850000000003C0001003B0000003B0001003A6A
:104860000000003A00010039000000390001003862
:104870000000003800000038000100370000003759
:10488000000100360000003600000036000100354F
:104890000000003500000035000100340000003445
:1048A000000000340001003300000033000000333A
:1048B000000100320000003200000032000100312F
:1048C0000000003100000031000100300000003025
:1048D000000000300001002F0000002F0000002F1A
:1048E0000000002F0001002E0000002E0000002E0E
:1048F0000001002D0000002D0000002D0000002D03
:104900000001002C0000002C0000002C0000002CF6
:104910000001002B0000002B0000002B0000002BEA
:104920000001002A0000002A0000002A0000002ADE
:1049300000010029000000290000002900000029D2
:1049400000000029000100280000002800000028C5
:1049500000000028000000280001002700000027B8
:1049600000000027000000270000002700010026AB
:10497000000000260000002600000026000000269F
:104980000001002500000025000000250000002592
:104990000000002500000025000100240000002484
:1049A0000000002400000024000000240001002377
:1049B000000000230000002300000023000000236B
:1049C000000000230000002300010022000000225C
:1049D000000000220000002200000022000000224F
:1049E0000001002100000021000000210000002142
:1049F0000000002100000021000000210001002033
:104A00000000002000000020000000200000002026
:104A10000000002000000020000000200001001F16
:104A20000000001F0000001F0000001F0000001F0A
:104A30000000001F0000001F0001001E0000001EFB
:104A40000000001E0000001E0000004D38342058F9
:104A50002059205A2045004572723A204D494E5443
:104A6000454D5020424544004D494E54454D50203F
:104A7000747269676765726564004572723A204DA9
:104A8000494E54454D50204531004572723A204DF3
:104A9000494E54454D50204530004572723A204DE4
:104AA000415854454D5020424544004D41585445CD
:104AB0004D50207472696767657265640045727253
:104AC0003A204D415854454D5020453100457272B1
:104AD0003A204D415854454D50204530004B494CEB
:104AE0004C45442E20004B494C4C20636175736546
:104AF00064206279204B494C4C20627574746F6E4F
:104B00002F70696E0A004B494C4C45442E20004BD7
:104B1000494C4C2063617573656420627920746F21
:104B20006F206D75636820696E61637469766520B6
:104B300074696D65202D2063757272656E742063D3
:104B40006F6D6D616E643A200020746F6F206C6F22
:104B50006E6720657874727573696F6E2070726508
:104B600076656E7465640A0020636F6C64206578F6
:104B700074727573696F6E2070726576656E746598
:104B8000640A002042002050006F6B00526573657C
:104B90006E643A200020496E76616C696420657805
:104BA0007472756465722000290A00206279746548
:104BB000733B20637263200053657474696E67737E
:104BC0002053746F726564202800205A0020590019
:104BD000580020204D61783A2000205A00205900CA
:104BE000580020204D696E3A20004F6E20004F661D
:104BF0006600536F667420656E6473746F70733AE9
:104C0000200053657474696E672054726176656C18
:104C100020416363656C65726174696F6E3A200050
:104C200053657474696E6720526574726163742091
:104C3000416363656C65726174696F6E3A200053FD
:104C4000657474696E67205072696E742041636385
:104C5000656C65726174696F6E3A20005365747497
:104C6000696E67205072696E7420616E64205472A0
:104C70006176656C20416363656C65726174696F10
:104C80006E3A2000004D3234005072696E7420700C
:104C90006175736564004D313235004D363030201A
:104CA0004230004D3234004D32332025730061759F
:104CB000746F25692E67004578747275646572009B
:104CC0004D6F7665205A004D6F76652059004D6F07
:104CD00076652058004D6F76656D656E74004D6F7A
:104CE000766520617869730044697361626C652040
:104CF0007374657070657273004D3834004175745B
:104D00006F20686F6D6500473238004D61696E0035
:104D1000526573746F7265206661696C7361666554
:104D2000004D3530320A4D353030004C6F61642013
:104D300073657474696E67730053746F7265207362
:104D4000657474696E677300416476616E6365644F
:104D50002053657474696E6773004D61696E00500D
:104D600072696E742061626F727465640041626F73
:104D70007574204669726D77617265004E6F2053BD
:104D8000442063617264005072696E742066726FB1
:104D90006D2053440053746F70207072696E7400FC
:104DA000526573756D65207072696E74005061751F
:104DB0007365207072696E7400436F6E6669677503
:104DC000726174696F6E0054656D7065726174759F
:104DD0007265004D6F76656D656E74004368616E37
:104DE00067652066696C616D656E740054756E65EB
:104DF00000496E666F2073637265656E005761725D
:104E00006E696E673A20486F6D696E672042756DF6
:104E1000702044697669736F72203C20310A000269
:104E200002040000A0400000A04000000040466CCA
:104E30006F7700466C6F770046616E207370656512
:104E40006420310046616E20737065656420310016
:104E500042656400426564004E6F7A7A6C65004E6C
:104E60006F7A7A6C65005370656564005370656590
:104E700064004D61696E00416D6178204500416DAF
:104E80006178204500416D6178205A00416D61785C
:104E9000205A00416D6178205900416D6178205998
:104EA00000416D6178205800416D617820580041C3
:104EB0002D74726176656C00412D74726176656C3B
:104EC00000412D7265747261637400412D726574C6
:104ED0007261637400416363656C00416363656C78
:104EE000004D6F74696F6E00202F002042403A0021
:104EF00020403A004E6F204C696E65204E756D6201
:104F00006572207769746820636865636B73756D7B
:104F10002C204C617374204C696E653A2000535408
:104F20004F505045442E20005072696E74657220B7
:104F300073746F707065642064756520746F20658C
:104F400072726F72732E20466978207468652065CE
:104F500072726F7220616E6420757365204D3939ED
:104F60003920746F20726573746172742E20285416
:104F7000656D706572617475726520697320726504
:104F80007365742E2053657420697420616674659E
:104F9000722072657374617274696E67290A004EBB
:104FA0006F20436865636B73756D20776974682043
:104FB0006C696E65206E756D6265722C204C617334
:104FC00074204C696E653A2000636865636B737585
:104FD0006D206D69736D617463682C204C6173740E
:104FE000204C696E653A20004C696E65204E756DE7
:104FF000626572206973206E6F74204C6173742037
:105000004C696E65204E756D6265722B312C204C9B
:10501000617374204C696E653A20004D3131300067
:105020004D3331004D383420582059205A20450046
:1050300053442072656164206572726F720A004485
:105040006F6E65207072696E74696E672066696C38
:10505000650A00436F6F6C646F776E0046616E2067
:10506000737065656420310046616E2073706565FC
:105070006420310042656400426564004E6F7A7AB4
:105080006C65004E6F7A7A6C65004D61696E004EFA
:10509000414E494E495459494E46CDCCCC3D0AD794
:1050A000233C17B7D13877CC2B329595E6241FB126
:1050B0004F0A000020410000C84200401C4620BCAE
:1050C000BE4CCA1B0E5AAEC59D7469EEECC21124CB
:1050D0001FBECFEFD1E2DEBFCDBF00E00CBF14E0BA
:1050E000A0E0B2E0E6E8F5EF01E00BBF02C00790F8
:1050F0000D92AA30B107D9F724E1AAE0B4E001C0CB
:105100001D92A83CB207E1F710E5CCECD0E500E039
:1051100006C022970109FE010BBF0E9443FACA3C58
:10512000D10780E00807A9F70E9407A20C94B2FA01
:105130000C9400002F923F924F925F926F927F9259
:105140008F929F92AF92BF92CF92DF92EF92FF9297
:105150000F931F93CF93DF93CDB7DEB7C658D10916
:105160000FB6F894DEBF0FBECDBF0091720920E6E6
:10517000029F800111240E50184F8091920680FFEB
:105180001AC0EBECFFE384917F013FEFE31AF30ACF
:10519000811102C0780104C00E94DD77F701F3CFCE
:1051A000D7018D917D01882319F00E94DD77F8CF1A
:1051B0008AE00E94DD7710924F0610924E068FE330
:1051C000809391061092900610928F0610922404FC
:1051D000109225041092260410922704F801808171
:1051E0000F5F1F4F8032D1F38E34B1F4818190ED87
:1051F000980F9A3020F08D3211F08B3269F432968C
:10520000DF0131962C9120532A30D0F3CD01FC01DF
:10521000019620812032D9F3F0938906E093880625
:105220007F01BFEFEB1AFB0A10816AE270E0C70151
:105230000E9483FA009739F0DC0111978C9180323B
:10524000E1F311961C921D3429F0143519F017342E
:1052500009F0CDC0F7014E2F9F2F81918032D9F3F5
:1052600080538A3008F0C3C01093910620918F06B6
:1052700030919006E42FF92F6AE0AF014F5F5F4F46
:10528000629FC001639F900D1124208130E0205364
:105290003109820F931F218120532A3030F09093DF
:1052A000900680938F069A0103C09C01FA01E5CF16
:1052B000D9012F5F3F4F4C914032D1F31D3449F05B
:1052C000B090880640914E0650914F0661E070E024
:1052D00050C08E31910591F03CF48731910571F009
:1052E0008C31910569F70AC0853791054CF38737F2
:1052F000910524F0803AE3E09E0711F7B0934F0642
:10530000A0934E0674C02132F1F10FEB020F0A3167
:1053100008F05AC09F01F901A0812F5F3F4FA032D2
:10532000D1F320ED2A0F2A3008F042C09F01E02E71
:10533000F12CD701B595A795B595A795B595A795E6
:10534000AC5DBB4F07706B01002E01C0CC0C0A9402
:10535000EAF7DC90DC28DC922115310599F12B1954
:10536000D701A65FBB4F2C93208121542A3188F5A9
:10537000DF01FD0131962C912111C5CF50934F06CD
:1053800040934E0634C01D3409F0BFCF80329105E2
:1053900009F0BBCFF0934F06E0934E0663E270E056
:1053A000CF010E9483FA009711F1DC011C921FC00B
:1053B00023ED2A0F223008F4B9CFAB3211F00C9450
:1053C000473FB4CF20E0CCCF4115510569F6AD0180
:1053D000CBCF9F013196D9010C9100530A30C8F30D
:1053E000F9012F5F3F4FA081A032D1F3C1CF80914F
:1053F00091068D3409F4BFC7843511F40C94EA3E4C
:10540000873411F00C942A3F80918F06909190067A
:105410008A31910509F4E5C684F48430910544F499
:10542000823091050CF017C197FF23C00C94443FC4
:10543000049709F491C60C94443F8A35910509F408
:105440005BC76CF48B31910509F4D2C64C9711F00F
:105450000C94443F80E00E94649F0C94443F8B3541
:10546000910509F44DC78C35910509F44EC70C948C
:10547000443F80916302882311F40C94443F0E94BE
:105480009C7A89E294E00E94BD780E941D7D809103
:10549000920683FD8FC0C0903504D0903604E09012
:1054A0003704F09038042091CC073091CD0740911B
:1054B000CE075091CF07C701B6010E941FF3882382
:1054C00009F478C080912804811138C060910A02E3
:1054D00070910B02882777FD8095982F0E9425F305
:1054E0009B01AC0160914606709147068091480689
:1054F000909149060E941FF387FF20C0C092CC07FD
:10550000D092CD07E092CE07F092CF07EBECFFE30D
:1055100084918F010F5F1F4F882321F00E94DD7758
:10552000F801F6CFEDEEF1E084918F010F5F1F4F90
:10553000882321F00E94DD77F801F6CFC090350472
:10554000D0903604E0903704F09038042091CC07D6
:105550003091CD074091CE075091CF07C701B601DA
:105560000E9451F720E030E048E453E40E9478F9CB
:10557000181604F5C092CC07D092CD07E092CE0762
:10558000F092CF07EBECFFE384918F010F5F1F4F89
:10559000882321F00E94DD77F801F6CFEEECF1E0F0
:1055A00084918F010F5F1F4F882321F00E94DD77C8
:1055B000F801F6CF2091290430912A0440912B0460
:1055C00050912C046091C0077091C1078091C2076F
:1055D0009091C3070E941FF381111DC020912D04DB
:1055E00030912E0440912F04509130046091C407F3
:1055F0007091C5078091C6079091C7070E941FF35D
:10560000811109C060910C0270910D0280910E020F
:1056100090910F021AC060919C0270919D028827A0
:1056200077FD8095982F0E9425F320910C023091F0
:105630000D0240910E0250910F020E9484F32AE065
:1056400037ED43E25CE30E9484F30E9421BA0E949A
:105650001C790C94443F20916302222311F40C9492
:10566000443F11E0029709F010E00E949C7A82E525
:105670000E94867A882309F45CC10E943B786B0102
:105680007C014090C0075090C1076090C2077090A5
:10569000C3072091C4073091C5074091C6075091B8
:1056A000C70763962CAF3DAF4EAF5FAF6397809156
:1056B000290490912A04A0912B04B0912C046796A0
:1056C0008CAF9DAFAEAFBFAF679720912D043091E7
:1056D0002E0440912F04509130046F962CAF3DAFB3
:1056E0004EAF5FAF6F9720E030E0A901C701B60170
:1056F0000E941FF3882309F415C5A3019201679640
:105700006CAD7DAD8EAD9FAD67970E941FF381118B
:1057100011C063962CAD3DAD4EAD5FAD63976F96F6
:105720006CAD7DAD8EAD9FAD6F970E941FF388234A
:1057300009F4F8C420E030E0A901C701B6010E94D5
:105740001FF3881F8827881F181759F080E090E002
:10575000A0E8BFEBAB968CAF9DAFAEAFBFAFAB9742
:105760000AC020E030E040E85FE3AB962CAF3DAFED
:105770004EAF5FAFAB97A301920167966CAD7DAD65
:105780008EAD9FAD67970E9451F7A3966CAF7DAF2A
:105790008EAF9FAFA39763962CAD3DAD4EAD5FAD81
:1057A00063976F966CAD7DAD8EAD9FAD6F970E9488
:1057B00051F7A7966CAF7DAF8EAF9FAFA797A3961B
:1057C0002CAD3DAD4EAD5FADA397CA01B9010E94AE
:1057D00084F34B015C01A7962CAD3DAD4EAD5FADA2
:1057E000A797CA01B9010E9484F39B01AC01C501CE
:1057F000B4010E9452F70E94BDF96B966CAF7DAF69
:105800008EAF9FAF6B9720E030E040E05FE30E94F7
:1058100084F34B015C01A7019601C701B6010E9408
:1058200084F36B017C01A5019401C501B4010E94C0
:1058300084F39B01AC01C701B6010E9451F70E949D
:10584000BDF99B01AC01AB966CAD7DAD8EAD9FAD4E
:10585000AB970E9484F34B015C0167962CAD3DAD84
:105860004EAD5FAD6797C301B2010E9452F720E0D1
:1058700030E040E05FE30E9484F36B017C01A79677
:105880006CAD7DAD8EAD9FADA79790586B962CAD4E
:105890003DAD4EAD5FAD6B970E942EF89B01AC0104
:1058A000C501B4010E9484F39B01AC01C701B6019C
:1058B0000E9452F7A30192010E9451F76B017C01F3
:1058C0006F962CAD3DAD4EAD5FAD6F9763966CADF1
:1058D0007DAD8EAD9FAD63970E9452F720E030E022
:1058E00040E05FE30E9484F32B013C016B962CADFA
:1058F0003DAD4EAD5FAD6B97A3966CAD7DAD8EADFE
:105900009FADA3970E942EF89B01AC01C501B40185
:105910000E9484F39B01AC01C301B2010E9452F7C3
:1059200063962CAD3DAD4EAD5FAD63970E9451F7D0
:1059300014C089E40E94867A882329F00E943B786B
:105940006B017C0103C0C12CD12C76018AE40E943A
:10595000867A8823F9F00E943B786F966CAF7DAF12
:105960008EAF9FAF6F9720E030E0A901C701B6016D
:105970000E941FF381111EC020E030E0A9016F9644
:105980006CAD7DAD8EAD9FAD6F970E941FF3811101
:1059900011C0C8C320E030E0A901C701B6010E94D0
:1059A0001FF3882309F4BEC36F961CAE1DAE1EAE56
:1059B0001FAE6F97D701C601B05863968CAF9DAFED
:1059C000AEAFBFAF63976F962CAD3DAD4EAD5FAD43
:1059D0006F97505867962CAF3DAF4EAF5FAF67974C
:1059E0009C01AD01BC01CD010E9484F34B015C011F
:1059F00067962CAD3DAD4EAD5FAD6797CA01B9015D
:105A00000E9484F39B01AC01C501B4010E9452F7CE
:105A10000E94BDF9EB966CAF7DAF8EAF9FAFEB9759
:105A20008091C0079091C107A091C207B091C307B0
:105A3000A3968CAF9DAFAEAFBFAFA397A701960162
:105A4000BC01CD010E9452F7AB966CAF7DAF8EAF1B
:105A50009FAFAB972091C4073091C5074091C6070F
:105A60005091C707A7962CAF3DAF4EAF5FAFA7973A
:105A70006F962CAD3DAD4EAD5FAD6F97A7966CADFB
:105A80007DAD8EAD9FADA7970E9452F7AF966CAFDC
:105A90007DAF8EAF9FAFAF978091290490912A047C
:105AA000A0912B04B0912C04E3968CAF9DAFAEAFC8
:105AB000BFAFE397AB962CAD3DAD4EAD5FADAB97B1
:105AC000BC01CD010E9451F76B017C0120912D0496
:105AD00030912E0440912F0450913004E7962CAF62
:105AE0003DAF4EAF5FAFE797AF962CAD3DAD4EAD3E
:105AF0005FADAF97E7966CAD7DAD8EAD9FADE7978F
:105B00000E9451F74B015C018091C8079091C90731
:105B1000A091CA07B091CB07C158DF4F8883998302
:105B2000AA83BB83CF57D0409C01AD016091310463
:105B30007091320480913304909134040E9451F7A3
:105B40006B966CAF7DAF8EAF9FAF6B972091350496
:105B5000309136044091370450913804EF962CAFC1
:105B60003DAF4EAF5FAFEF978091CC079091CD07DF
:105B7000A091CE07B091CF07CD57DF4F888399838F
:105B8000AA83BB83C358D040A701960163966CAD2E
:105B90007DAD8EAD9FAD63970E9484F32B013C01D8
:105BA000A501940167966CAD7DAD8EAD9FAD6797F5
:105BB0000E9484F39B01AC01C301B2010E9452F721
:105BC0002B013C01A501940163966CAD7DAD8EADBA
:105BD0009FAD63970E9484F34B015C01A70196017E
:105BE00067966CAD7DAD8EAD9FAD67970E9484F3D7
:105BF0009B01AC01C501B4010E9451F7A3019201C0
:105C00000E94C5F76B017C0120E030E0A9010E94F1
:105C10001FF387FF0AC02BED3FE049EC50E4C701BA
:105C2000B6010E9452F76B017C01112351F02BED5C
:105C30003FE049EC50E4C701B6010E9451F76B0107
:105C40007C0120E030E0A901C701B6010E941FF3EA
:105C5000811128C0E3962CAD3DAD4EAD5FADE3970D
:105C6000A3966CAD7DAD8EAD9FADA3970E941FF343
:105C7000811118C0E7962CAD3DAD4EAD5FADE797F5
:105C8000A7966CAD7DAD8EAD9FADA7970E941FF31B
:105C9000811108C02BEDC22E2FE0D22E29ECE22E6E
:105CA00020E4F22EEB962CAD3DAD4EAD5FADEB9703
:105CB000C701B6010E9484F39B01AC010E9484F3EA
:105CC0004B015C016B962CAD3DAD4EAD5FAD6B975E
:105CD000CA01B9010E9484F39B01AC01C501B40162
:105CE0000E9452F70E94BDF94B015C012FE632E1A0
:105CF00043E85AE30E941FF387FD10C2C501B401B7
:105D00000E94C7F80E949BF8A5967FAF6EAFA5973B
:105D1000DB01AB2B31F4E1E0F0E0A596FFAFEEAF95
:105D2000A597A5962EAD3FADA597B90180E090E06F
:105D30000E9423F34B015C019B01AC01C701B6013A
:105D40000E942EF8A3966CAF7DAF8EAF9FAFA39746
:105D5000A50194016B966CAD7DAD8EAD9FAD6B973B
:105D60000E942EF8EB966CAF7DAF8EAF9FAFEB9796
:105D7000CD57DF4F288139814A815B81C358D0409C
:105D8000EF966CAD7DAD8EAD9FADEF970E9451F754
:105D9000A50194010E942EF8EF966CAF7DAF8EAFF7
:105DA0009FAFEF97A3962CAD3DAD4EAD5FADA397E2
:105DB000CA01B9010E9484F320E030E040E05FE3D3
:105DC0000E9484F39B01AC0160E070E080E89FE3F7
:105DD0000E9451F7E3966CAF7DAF8EAF9FAFE39714
:105DE000C158DF4F88819981AA81BB81CF57D040AC
:105DF00089879A87AB87BC87CD57DF4F2881398148
:105E00004A815B81C358D0402D873E874F87588B8E
:105E100060919C0270919D02882777FD8095982F54
:105E20000E9425F320910C0230910D0240910E0248
:105E300050910F020E9484F32AE037ED43E25CE3C5
:105E40000E9484F3E7966CAF7DAF8EAF9FAFE7976C
:105E50000E94897CDC01CB0188539F4FAF4FBF4F1D
:105E60006B968CAF9DAFAEAFBFAF6B9760964FACEC
:105E7000609761965FAC619762966FAC629763962C
:105E80007FAC639722242394312C99E1992EA59617
:105E9000AEADBFADA5972A163B0608F02BC10E94F8
:105EA00017730E94897C6B962CAD3DAD4EAD5FADF6
:105EB0006B97621B730B840B950B97FD11C00E94AF
:105EC000897CDC01CB0188539F4FAF4FBF4F6B964E
:105ED0008CAF9DAFAEAFBFAF6B9780E00E9436C373
:105EE0009A9409F44FC0E3962CAD3DAD4EAD5FAD35
:105EF000E39767966CAD7DAD8EAD9FAD67970E94C1
:105F000084F36B017C01A3962CAD3DAD4EAD5FAD2E
:105F1000A397B201C3010E9484F3A70196010E94D6
:105F200052F7162F072FB82EA92EE3962CAD3DADB4
:105F30004EAD5FADE397B201C3010E9484F36B01E4
:105F40007C01A3962CAD3DAD4EAD5FADA39767969A
:105F50006CAD7DAD8EAD9FAD67970E9484F39B01C4
:105F6000AC01C701B6010E9451F72B013C01812F02
:105F7000902FAB2DBA2D67968CAF9DAFAEAFBFAF54
:105F800067975BC0B10180E090E00E9423F3A39685
:105F90002CAD3DAD4EAD5FADA3970E9484F34B0198
:105FA0005C010E942BF86B017C01C501B4010E94C9
:105FB000B3F94B015C01A701960163966CAD7DAD11
:105FC0008EAD9FAD63970E9484F32B013C01A50128
:105FD00094016F966CAD7DAD8EAD9FAD6F970E94B5
:105FE00084F39B01AC01C301B2010E9452F72B0163
:105FF0003C01A501940163966CAD7DAD8EAD9FAD66
:1060000063970E9484F34B015C01A70196016F9690
:106010006CAD7DAD8EAD9FAD6F970E9484F39B01FB
:10602000AC01C501B4010E9451F767966CAF7DAF1A
:106030008EAF9FAF679709E1902E9201A301AB96B7
:106040006CAD7DAD8EAD9FADAB970E9452F769836D
:106050007A838B839C8367962CAD3DAD4EAD5FAD4F
:106060006797AF966CAD7DAD8EAD9FADAF970E943B
:1060700052F76D837E838F839887EB962CAD3DAD71
:106080004EAD5FADEB9769857A858B859C850E94C7
:1060900052F769877A878B879C87EF962CAD3DAD49
:1060A0004EAD5FADEF976D857E858F8598890E9497
:1060B00052F76D877E878F87988BCE0101960E945D
:1060C000BD78C0908706E796ECACFDAC0EAD1FAD79
:1060D000E7979E01235F3F4FAE01475F5F4FBE01D1
:1060E0006B5F7F4FCE0101960E9436C59FEF291A44
:1060F000390ACDCEC0908706E796ECACFDAC0EAD6C
:106100001FADE79725E334E041E354E06DE274E02E
:1061100089E294E00E9436C50E941C790E941D7D90
:106120000C94443FE4E9FFE384918F010F5F1F4F1C
:10613000882321F00E94DD77F801F6CFE8E0F2E055
:1061400084918F010F5F1F4F882311F40C94443FFB
:106150000E94DD77F801F4CF80E50E94867A8823DB
:1061600029F00E94FB774B015C0103C0812C912C2C
:10617000540183E50E94867A882361F00E943B786F
:1061800020E030E04AE754E40E9484F30E949BF848
:106190004B015C010E94F5AE80911002811105C097
:1061A00060E08EE192E00E94B2880E941D7DC09066
:1061B0003904D0903A04E0903B04F0903C04C80CC1
:1061C000D91CEA1CFB1C0E94897C6C197D098E0974
:1061D0009F0997FD02C00C94443F80E00E9436C3A3
:1061E000F2CF81E080936302109286060C94443FC4
:1061F0000E94B06081110C94443F80E50E94867A31
:10620000882321F00E940B78462F01C040E0609166
:10621000C8077091C9078091CA079091CB0700E029
:1062200010E020E231E409831A832B833C8300E0F1
:1062300010E025E833E40D831E832F83388700E0C8
:1062400010E020EA31E409871A872B873C8700E0B9
:1062500010E020EC3FE70D871E872F87388B4130F9
:1062600071F1423021F518A219A21AA21BA220E056
:1062700030E040EA51E40E9452F77B018C0120E0BB
:1062800030E04AE753E40E9478F9181624F4E12C30
:10629000F12C0AE713E4A701B8014BAF5CAF6DAF77
:1062A0007EAFBE01605E7F4FCE01CB9611C020E075
:1062B00030E040EA51E40E941FF387FF0BC018A2B0
:1062C00019A21AA21BA2BE01605E7F4FCE010996E1
:1062D0000E9491E218A219A21AA21BA29E01205E9E
:1062E0003F4F48EC57E0BE016B5F7F4FCE010196F8
:1062F0000E949FE10C94443F10928E060C94443F00
:1063000081E080938E060C94443F85E40E94867A57
:10631000C82E811102C00E94F5AE16E1E12E13E0F5
:10632000F12E00EC17E0B12CD12CF70181917F0107
:106330000E94867A882369F00E943B78D8016D9389
:106340007D938D939C931397B3E0DB1611F0BB24E0
:10635000B394D3940C5F1F4FE4E0DE12E6CFBB2072
:1063600019F00E94C6B603C0C1100E94C9610E9404
:1063700048550C94443F80918F0690919006873742
:10638000910511F40C94643A0CF0C9C08C34910559
:1063900009F46DC50CF06BC08831910509F49AC2FF
:1063A000B4F58231910509F484C7BCF497FF02C0AB
:1063B0000C94443F823091050CF4B1C1419711F027
:1063C0000C94443F60E08EE592E00E94B2881798FA
:1063D0001698159814980C94443F8531910509F44A
:1063E00062C23CF4449711F00C94443FE6E7F2E0BB
:1063F00019C28631910509F45AC2479711F00C94DD
:10640000443F80914E0690914F06FC015AC28E3156
:10641000910509F4D6C2C4F48A31910509F487C202
:106420000CF477C28B31910509F48FC24C9711F0AF
:106430000C94443F40E060E080914E0690914F06FE
:106440000E94486F0C94443F8032910509F4DCC3EC
:106450000CF425C48A32910509F4C2C48B34910529
:1064600011F00C94443F0E9490610C94443F893693
:10647000910509F4E2C524F58335910509F415C7A2
:106480007CF48135910509F4F3C60CF00BC78D340B
:10649000910511F00C94443F0E9447610C94443FD5
:1064A0008535910509F43AC70CF403C78C3591057D
:1064B00009F437C78836910509F4DDC40C94443FCC
:1064C0008F36910509F436C584F48B36910509F4AD
:1064D00044C60CF41FC68D36910509F4EFC58E36FF
:1064E000910509F416C50C94443F8337910509F4CE
:1064F0001BC75CF48237910511F00C94443F0E9455
:10650000F5AE0E9448550C94443F8537910509F437
:106510009CC78637910509F4A0C70C94443F8D327F
:10652000F1E09F0711F40C94293C0CF06EC0893CFB
:10653000910511F40C94903B54F58C38910509F4B5
:1065400062C574F48937910511F40C94CE3A14F4B1
:106550000C94C83A8D37910509F415C60C94443F44
:106560008B39910509F483C53CF48139910511F407
:106570000C94D33A0C94443F8E3B910509F4B6C574
:10658000883C910511F40C94483B0C94443F833DA6
:10659000910511F40C94B63BECF48C3C910511F48C
:1065A0000C94B03B4CF48B3C910511F00C94443F9F
:1065B0000E94537A0C94443F8D3C910511F40C9445
:1065C000B33B8E3C910511F00C94443F0E94CFB632
:1065D0000C94443F8D3D910511F40C94B93B4CF45F
:1065E0008C3D910511F00C94443F0E94927A0C94DA
:1065F000443F823E910511F40C94BC3B8C32914097
:1066000011F40C94003C0C94443F843F41E0940707
:1066100011F40C94103D0CF047C08E35A1E09A07A0
:1066200011F40C94393E94F48F32E1E09E0711F49A
:106630000C942F3C14F40C942C3C8033914011F0BA
:106640000C94443F0E94845A0C94443F833631E0BA
:10665000930711F40C94BF3E3CF48F35914011F434
:106660000C946D3E0C94443F8039A1E09A0711F4DC
:106670000C94323C8C3A914011F00C94443F94EBD2
:10668000892E97E0992E20ECA22E27E0B22E3BE730
:10669000232E36E0332E00E010E0822D80956096A8
:1066A0008FAF60970C94353C8835E2E09E0711F47B
:1066B0000C941C3DC4F4863F21E0920711F40C9425
:1066C000163D14F40C94133D873F41E0940711F4F8
:1066D0000C94193D8C31924011F00C94443F0E946F
:1066E0004B7A0C94443F8C38A3E09A0711F40C9435
:1066F0001F3E4CF48B38934011F00C94443F0E94A1
:106700001C550C94443F803AF3E09F0709F4BAC249
:10671000873E934011F40C94D83E0C94443F009172
:106720004E0610914F0680E50E94867A882369F014
:106730000E94FB776B017C01BB24B394611571054A
:106740008105910531F4B12C04C0B12CC12CD12CA0
:10675000760183E50E94867A8823F9F00E943B78CF
:1067600020E030E04AE754E40E9484F30E949BF862
:106770006B017C01B11013C0611571058105910594
:1067800071F40115110559F0D8018C91882339F065
:1067900061E0C8010E94A28807C0BB2091F360E0BD
:1067A0008BE492E00E94B28881E08093CB090E9442
:1067B000F5AE0E941D7DC114D104E104F104D1F0B5
:1067C0008090390490903A04A0903B04B0903C042F
:1067D0008C0C9D1CAE1CBF1C0E94897C6819790919
:1067E0008A099B0997FF1AC08091CB0981110C94EB
:1067F000513F14C08091CB09882321F080E00E9492
:1068000036C3F8CF8091111260E0882319F08CE331
:1068100092E002C087E292E00E94B2881092CB0917
:106820000C94443F84918F010F5F1F4F882321F008
:106830000E94DD77F801F6CF1092BD1440E050E0E1
:10684000BA0189E692E10E945F5E8BE1E9E6F2E13E
:10685000DE01159601900D928A95E1F780916712FD
:10686000909168129C838B838EE093E09A83898356
:1068700040E050E0BE016F5F7F4F82E094E00E94F5
:106880003B84CE0101960E948750E7E6F2E08491B6
:106890008F010F5F1F4F882311F40C94443F0E9417
:1068A000DD77F801F4CF0E943A4F0C94443F1092E8
:1068B0001112109212120C94443F203209F41082EB
:1068C000319620812111F9CF40E061E00E94486FAC
:1068D0000C94443F19821A821B821C8218A219A2AE
:1068E0001AA21BA280918506882341F040E0BE01D8
:1068F0006F5F7F4FCE0180960E9460AC8091121234
:10690000882319F081E0809311120E9490610C9409
:10691000443F109211120E94076287E892E0909320
:10692000500A80934F0A0E94ADDC0C94443F809142
:106930001212882311F40C94443F83E50E94867A56
:1069400081110C94563F0C94443F8091121288237D
:1069500051F1ECE8F2E084918F010F5F1F4F882323
:1069600021F00E94DD77F801F6CF6091B4147091A8
:10697000B5148091B6149091B7144AE00E94B366A2
:106980008FE20E94DD776091B0147091B114809114
:10699000B2149091B3144AE00E94B3668AE00E9458
:1069A000DD770C94443FEEE9F2E084918F010F5FB4
:1069B0001F4F882311F40C94443F0E94DD77F801A7
:1069C000F4CF80911212882311F40C94443F83E099
:1069D00094E10E94254B83E094E10E94284F10929D
:1069E000101210920F12E0904E06F0904F06809118
:1069F0001212882311F40C94443F0E94304F1D82E0
:106A000018861C821B828EE093E09A83898385E638
:106A100092E19093851280938412F70180818F32E6
:106A200009F06BC06FE270E0C7010E9483FA8C012D
:106A30000F5F1F4F9E012F5F3F4F59010115110539
:106A400009F461C06FE270E0C8010E9483FA6C0132
:106A5000009709F459C00817190708F055C04C01F0
:106A6000801A910AA401B801CE0180960E94A3FA6F
:106A7000E0E2F0E0EC0FFD1FE80DF91D10828E0141
:106A8000005E1F4FD8018D918D01882319F00E945F
:106A9000DD77F8CF8AE00E94DD77609184127091F3
:106AA00085126115710519F06C5F7F4F02C060E0BF
:106AB00070E021E0AE01405E5F4FCE0105960E947E
:106AC0004183811112C0BE01605E7F4F85ED92E06F
:106AD0000E9493648EE20E94DD778AE00E94DD7757
:106AE000C5010E9487500C94443FB0928512A09239
:106AF000841286010F5F1F4FA1CF86E892E1909329
:106B0000851280938412870160918412709185129E
:106B10006115710519F06C5F7F4F02C060E070E095
:106B200018A21BA222E0A801CE0180960E944183F8
:106B3000F82E882311F1CE0180960E94634BF82E27
:106B40008823D9F06CA57DA58EA59FA541E00E9464
:106B50002F5CF82E882389F0E8A9B0E2EB9FF001C2
:106B60001124E35CFB4F309739F085EE80831BA244
:106B70000E94F15BF82E01C0F12CCE0180960E949C
:106B80008250FF2011F1BFEAEB2EB2E0FB2EF7019D
:106B90008491882331F0FFEFEF1AFF0A0E94DD771E
:106BA000F6CFD8018D918D01882319F00E94DD77F1
:106BB000F8CF8AE00E94DD771092B4141092B514D9
:106BC0001092B6141092B71419C0ADEBEA2EA2E0E1
:106BD000FA2EF7018491882331F0FFEFEF1AFF0AB4
:106BE0000E94DD77F6CFD8018D918D01882319F0B1
:106BF0000E94DD77F8CF8EE20E94DD77CE0101960C
:106C00000E9487500C94443F8091111281110E9480
:106C1000F5AE00914E0610914F0680E50E94C179B5
:106C2000882321F00E942C78F82E01C0F12C80914D
:106C30001212882311F40C94443F4F2D61E0C801D7
:106C40000E94486F83E50E94867A882381F00E9423
:106C50000B78AB01BC014093B4145093B51460930E
:106C6000B6147093B71483E094E10E945F5E809144
:106C70001212882319F081E080931112F1100C9404
:106C8000443F43CE80914E0690914F0621E02093E1
:106C9000101240E060E00E94486F0C94443F0E9454
:106CA0005C61FCE3CF2ED12CE12CF12CA7019601E5
:106CB0000E94F4F6162F072FCA01B901A701960109
:106CC0000E94F4F6D62EC72ECA01B90128E130E0A1
:106CD00040E050E00E94F4F6FB01C9016DE671E06E
:106CE0000E9416FA9B014D2D5C2DDE0111967D014F
:106CF0002115310599F00F931F93CF92DF92FF93E7
:106D0000EF939F938F933F932F9381E193E09F9312
:106D10008F93FF92AF930E94B9F212C00097B1F027
:106D20000F931F93CF92DF92FF93EF939F938F93D5
:106D300081E093E09F938F93FF92AF930E94B9F20B
:106D40000FB6F894DEBF0FBECDBF30C0309779F0DC
:106D50000F931F93CF92DF92FF93EF9385EF92E013
:106D60009F938F93FF92AF930E94B9F2E9CF452B87
:106D700069F00F931F93CF92DF928DEE92E09F9375
:106D80008F93FF92AF930E94B9F2DACF0F931F93C4
:106D900089EE92E09F938F93FF92AF930E94B9F296
:106DA0000F900F900F900F900F900F9060E0C70121
:106DB0000E94A288EBECFFE384918F010F5F1F4FCD
:106DC000882321F00E94DD77F801F6CFB70185E234
:106DD00093E00E9493648AE00E94DD770C94443F24
:106DE00083E50E94867A882311F40C94443F0E9424
:106DF0001B78E82E80E50E94867A882311F40C9493
:106E0000443F80E50E94867A882341F00E940B78F7
:106E100077FF02C00C94443F8B0102C00DE010E0EC
:106E2000802FE2E3F3E09491891739F0319693E0F3
:106E3000EA35F907C1F70C94673FE4E9FFE3849171
:106E40008F010F5F1F4F882321F00E94DD77F8012B
:106E5000F6CFEAE5F3E084918F010F5F1F4F88239F
:106E600011F40C94443F0E94DD77F801F4CF0E94A6
:106E700007620C94443F88E690E00E9403D8811199
:106E80000C94443F8091920683FF01C0FDC783E5C7
:106E90000E94867A882309F4F7C70E943B780E94F3
:106EA00096F87093850F6093840F80E00E94648B46
:106EB0000E943B7820E030E040E752E40E941FF35C
:106EC00018163CF00E94476160E085E793E00E945D
:106ED000B2880E943B782091460630914706409147
:106EE0004806509149060E9478F918160CF0CCC754
:106EF00084ED92E09F938F9389E693E09F938F9325
:106F00001F920E9495600F900F900F900F900F901E
:106F1000BBC78EE40E94867A882309F4B5C70E9415
:106F20000B7860933D0670933E0680933F069093E6
:106F30004006AAC783E50E94867A882321F00E9432
:106F40001B78C82E01C0C12CC0929206EBECFFE367
:106F500084918F010F5F1F4F882321F00E94DD77FE
:106F6000F801F6CFE8E9F3E084918F010F5F1F4F3E
:106F7000882321F00E94DD77F801F6CFCC2099F12B
:106F8000EAE8EE2EE3E0FE2E00E010E020E0D12C57
:106F9000C601002E02C0959587950A94E2F780FFFE
:106FA00017C099249394920E222319F08CE20E9428
:106FB000DD77F70125913491F90184915901FFEFB3
:106FC000AF1ABF0A882329F00E94DD779501F4CF1C
:106FD000922E0F5F1F4F22E0E20EF11C05301105CB
:106FE00071F0292DD5CFE4E9F3E084918F010F5F93
:106FF0001F4F882321F00E94DD77F801F6CF8AE049
:107000000E94DD7741C78091920683FD3DC783E5ED
:107010000E94867A882309F437C70E943B780E9431
:1070200096F86739710514F066E970E07093810F86
:107030006093800F0E94198B27C789E690E00E9419
:1070400003D881110C94CD42EFE9F3E084918F01D4
:107050000F5F1F4F882321F00E94DD77F801F6CFE4
:107060000E9499EC8AE00E94DD770C94CD4283E582
:107070000E94867A882309F407C70E941B788093B0
:1070800045068D3318F08CE3809345060E94897C79
:107090006B017C012091450630E0A8EEB3E00E9430
:1070A00042F7C60ED71EE81EF91EC0924106D092C6
:1070B0004206E0924306F0924406E6C68DE690E072
:1070C0000E9403D88111E0C68091920683FDDCC640
:1070D00083E50E94867A60968FAF6097811113C70F
:1070E00082E50E94867A81110EC7CEC680919206F3
:1070F00083FDCAC683E50E94867A6C968FAF6C9733
:1071000081110C94254182E50E94867A81110C94AC
:107110002541BAC683E50E94867A882339F00E9409
:107120000B788B016F3F710519F010F00FEF10E035
:1071300080E50E94867A882331F00E941B78823095
:1071400008F0A2C601C080E0E82FF0E0EE0FFF1FBC
:10715000E352FF4E1183008397C680E50E94867A32
:10716000882339F00E940B786230710508F08CC6D4
:1071700002C060E070E0FB01EE0FFF1FE352FF4E24
:107180001182108281C68CE40E94C179882319F093
:107190000E943B7804C060E070E080E090EC2796AD
:1071A0006CAF7DAF8EAF9FAF27978AE50E94867A3E
:1071B000882319F00E943B7803C060E070E0CB01A7
:1071C00020E030E040E251E40E9452F723966CAF99
:1071D0007DAF8EAF9FAF239788E50E94867A882384
:1071E00019F00E943B7803C060E070E0CB0120E022
:1071F00030E040E251E40E9452F76BAF7CAF8DAFBC
:107200009EAF89E50E94867A882319F00E943B7818
:1072100003C060E070E0CB0120E030E04AE853E4D6
:107220000E9452F720E030E040E251E40E9451F722
:1072300068A379A38AA39BA319821A821B821C824A
:1072400080918506811120C6C12CE12C8E010F5F33
:107250001F4F9E01205E3F4FAE01455C5F4FBE0158
:10726000615C7F4FCE018D5B9F4F0E948AAD0CC643
:107270000E944D520E94F5AE0E946E781092DE1070
:107280001092DD101092E0101092DF1068EE73E0A3
:1072900080E090E00E94927560E08BE094E00E94B4
:1072A000B288F2C510928D06EFC581E080938D06FD
:1072B000EBC583E50E94867A882399F00E943B788B
:1072C00020E030E04AE754E40E9484F30E949BF8F7
:1072D0006093530270935402809355029093560228
:1072E000D3C588E50E94C17981110C94AA4289E531
:1072F0000E94C17981110C94AA428AE50E94C17949
:1073000081110C94AA4285E40E94C17981110C94E8
:10731000AA420E94F5AE0E946E78B6C50E94707AAD
:10732000B3C50E942DB6B0C5E9EFF4E084918F019A
:107330000F5F1F4F882321F00E94DD77F801F6CF01
:10734000EBEEF4E084918F010F5F1F4F882321F053
:107350000E94DD77F801F6CFE4EDF4E084918F012F
:107360000F5F1F4F882321F00E94DD77F801F6CFD1
:10737000E4ECF4E084918F010F5F1F4F882321F02C
:107380000E94DD77F801F6CFE3EBF4E084918F0102
:107390000F5F1F4F882321F00E94DD77F801F6CFA1
:1073A000E2EAF4E084918F010F5F1F4F882321F000
:1073B0000E94DD77F801F6CFE3E9F4E084918F01D4
:1073C0000F5F1F4F882321F00E94DD77F801F6CF71
:1073D000EEE7F4E084918F010F5F1F4F882321F0C7
:1073E0000E94DD77F801F6CFE8E6F4E084918F01A2
:1073F0000F5F1F4F882321F00E94DD77F801F6CF41
:10740000E3E5F4E084918F010F5F1F4F882321F0A3
:107410000E94DD77F801F6CFE6E3F4E084918F0176
:107420000F5F1F4F882321F00E94DD77F801F6CF10
:10743000EEE1F4E084918F010F5F1F4F882309F480
:1074400023C50E94DD77F801F5CF60E080914E06FC
:1074500090914F060E94A28817C585E40E94C179C9
:10746000882381F00E942C78882361F0EBECFFE305
:1074700084918F010F5F1F4F882321F00E94DD77D9
:10748000F801F6CF81E40E94C179882381F00E943F
:107490002C78882361F0E1EFF5E084918F010F5F94
:1074A0001F4F882321F00E94DD77F801F6CF00916D
:1074B0004E0610914F06D8018D918D01882309F455
:1074C0009ECD0E94DD77F7CFEDE0F6E084918F014D
:1074D0000F5F1F4F882321F00E94DD77F801F6CF60
:1074E000E5E0F6E084918F010F5F1F4F882321F0C4
:1074F0000E94DD77F801F6CF1E9903C00FEE12E06F
:1075000002C00AEE12E0F80181918F01882319F080
:107510000E94DD77F8CF8AE00E94DD77EDEFF5E09D
:1075200084918F010F5F1F4F882321F00E94DD7728
:10753000F801F6CF1D9903C00FEE12E002C00AEE6B
:1075400012E0D8018D918D01882319F00E94DD771A
:10755000F8CF8AE00E94DD77E5EFF5E084918F01B6
:107560000F5F1F4F882321F00E94DD77F801F6CFCF
:107570001C9903C00FEE12E002C00AEE12E0F801FF
:1075800081918F01882309F43ACD0E94DD77F7CFEE
:1075900081E08093B0078093500676C41092B007C4
:1075A0001092500671C483E50E94867A882319F0F0
:1075B0000E940B7802C060E070E08B01112702305E
:1075C0001105C8F0E4E9FFE384918F010F5F1F4FBD
:1075D000882321F00E94DD77F801F6CFE7E2F6E09C
:1075E00084918F010F5F1F4F882309F44DC40E94BF
:1075F000DD77F801F5CF88E40E94867A8823A9F028
:107600000E940B78683771053CF06332F1E07F0728
:107610002CF062E271E002C068E770E0F801EE0F62
:10762000FF1FE75AF94F7183608386E40E94867AD0
:10763000882399F00E940B786F3F710519F014F0C0
:107640006FEF70E0F801EE0FFF1FEB5AF94F77FF75
:1076500002C060E070E07183608382E40E94867AF9
:10766000882309F411C40E940B786530710534F049
:10767000683871052CF067E870E002C065E070E0E2
:10768000F801EE0FFF1FEF5AF94F71836083FCC3BF
:1076900088EC90E00E9403D88111F6C384E40E9434
:1076A000C1798823D1F10E943B7811E020E030E0DD
:1076B000A9010E941FF3811101C010E0109362061E
:1076C000112359F10091610610E00E943B78F80106
:1076D000EE0FFF1FEE0FFF1FE35AF94F6083718318
:1076E0008283938320E030E0A90160915D06709170
:1076F0005E0680915F06909160060E941FF38111E3
:107700000CC080E090E0A0E4B0E480935D0690932C
:107710005E06A0935F06B09360060E947878B4C3BB
:1077200006E113E056EEE52E50E1F52ED8018D91DD
:107730008D010E94C179882349F00E943B780E9404
:107740009BF8F7016083718382839383F4E0EF0EEB
:10775000F11C23E00A31120749F70E94677794C3AE
:107760000E9482D291C30E94EF798EC30E94E7D219
:107770008BC30E9443D888C380E50E94C1798823C7
:1077800009F482C30E940B78F62E062F172F83E58B
:107790000E94867A882321F00E940B786B0103C037
:1077A000CC24CA94DC2C96012F5F3F4F2330310547
:1077B00008F06AC317FD68C30E94F5AE3FEFC31619
:1077C000D30631F0CA94CD2871F000E010E00DC06E
:1077D0008F2D0E94287C31E020E0892B09F030E0D9
:1077E000032F122F02C001E010E08F2D0E94287C91
:1077F0008017910709F448C380E00E9436C3F5CF93
:1078000083E50E94867A882319F00E940B7802C0D3
:1078100064E071E079A368A380E50E94867A8823FA
:1078200039F00E940B78693853E1750730F402C0D3
:1078300068EE73E07A83698304C088E893E19A83F1
:107840008983BE01605E7F4FCE0101960E94A674BF
:107850001BC30E94E75918C30E94046815C30E9405
:10786000ABA712C30E94F5AE0FC3D1018D911D01CC
:10787000882309F4A3C0F5014080518062807380A1
:10788000F801E95AFD4F2081318142815381F8018D
:10789000E159F94F60817181828193810E9452F791
:1078A00020E030E040E05FE30E9484F39B01AC0104
:1078B000C301B2010E9478F9181644F4F801E75B9D
:1078C000F94FC590D590E590F49003C0C12CD12C10
:1078D0007601F801ED59F94F2081318142815381C0
:1078E000C301B2010E9451F79B01AC01C701B6016F
:1078F0000E9451F76B017C0120E030E040EA51EC3E
:107900000E9478F987FD2BC020E030E040EA51E486
:10791000C701B6010E941FF318160CF1D4012D9176
:107920003D914D915C91C701B6010E9451F79B01B9
:10793000AC01C301B2010E9452F7F501608371836B
:1079400082839383D401CD92DD92ED92FC921397C2
:1079500060968FAD6097820D0E9426792FC0E4E972
:10796000FFE384918F010F5F1F4F882321F00E9456
:10797000DD77F801F6CFE3E7F6E084918F010F5F42
:107980001F4F882321F00E94DD77F801F6CF61E0D8
:1079900085E696E00E94B2880E942B8A88E290E0F9
:1079A0009A83898388EC90E099A388A3BE016F5FD6
:1079B0007F4FCE0180960E94A67466C2B4E08B0E03
:1079C000911C0C5F1F4FE4E0AE0EB11C0C30110592
:1079D00009F04BCF0E94C6B60E94485560E085E58D
:1079E00096E00E94B28883E992E099A388A304E616
:1079F00010E01A830983BE01605E7F4FCE010196BD
:107A00000E94A6748AEB92E099A388A31A83098343
:107A1000BE01605E7F4FCE0101960E94A67434C203
:107A20000E9494D331C20E9446B12EC20E940EB071
:107A30002BC20E94DB5928C20E94B060882319F033
:107A400081E00E94649F85E40E94C179882319F037
:107A50000E943B7804C060E070E080E090EC2F96DC
:107A60006CAF7DAF8EAF9FAF2F978AE50E94867A6D
:107A7000882319F00E943B7804C060E070E080E247
:107A800091E42B966CAF7DAF8EAF9FAF2B9788E5BF
:107A90000E94867A882319F00E943B7804C060E037
:107AA00070E080E291E427966CAF7DAF8EAF9FAF20
:107AB000279789E50E94867A882319F00E943B78EF
:107AC00004C060E070E085E893E423966CAF7DAF7E
:107AD0008EAF9FAF239785E50E94C179882319F067
:107AE0000E943B7804C060E070E088EC92EC6BAFE1
:107AF0007CAF8DAF9EAF8CE40E94C179882319F0D2
:107B00000E943B7803C060E070E0CB0168A379A3DA
:107B10008AA39BA382E40E94867A882321F00E9494
:107B20000B78F62E02C085E0F82ED09002128091DC
:107B3000850681117EC0CC24C394EF2C8E01055C98
:107B40001F4F9E01215C3F4FAE014D5B5F4FBE0159
:107B5000695B7F4FCE01855B9F4F0E948AAD882372
:107B600009F467C081E08093CB0911E08091CB09D3
:107B7000882309F44AC060E08F2D0E941C75809113
:107B800084068823F1F110937F0640E050E0BA01AB
:107B900080E694E90E94D3898091CB09882321F063
:107BA00081E00E9436C3F8CF1092800610928106C1
:107BB0001092820610928306109284060E94648BB3
:107BC0000E9476D110937F0640E050E0BA0186EB28
:107BD00092E90E94D3890E94897C685370458F4F37
:107BE0009F4F6093800670938106809382069093E6
:107BF0008306109284061093CB0961E08F2D0E94BA
:107C00001C7581E00E9436C3B1CF00E010E028E48B
:107C100032E409831A832B833C8380918506882371
:107C200041F04F2DBE016F5F7F4FCE0180960E94C5
:107C300060ACF1E0DF1228C10E94906125C183E5AC
:107C40000E94867A882321F00E940B788B0102C063
:107C500000E010E080E50E94867A882321F00E94EF
:107C60000B78CB0102C080E090E0B8010E94ED5497
:107C70000BC183E50E94C179811104C006E113E0C4
:107C8000F12C0FC010E00E941B78682F812F0E94FA
:107C900045901F5F1530B9F7F1CFF394B4E0FB16B0
:107CA00071F0D8018D918D010E94C1798823A9F3CB
:107CB0000E941B78682F8F2D0E944590EECF82E4A2
:107CC0000E94C179882331F00E941B78682F84E0DC
:107CD0000E9445900E943F67D7C083E50E94867A44
:107CE000882309F449C00E941B78813039F0823022
:107CF00009F042C006E113E0F12C23C006E113E0D5
:107D0000F12CF80181918F010E94867A882339F045
:107D10000E941B784FEF682F8F2D0E949B8FF3944A
:107D2000F4E0FF12EECF82E40E94867A882321F1EC
:107D30000E941B784FEF682F1CC0F394B4E0FB1631
:107D400079F0D8018D918D010E94867A8823A9F35C
:107D50000E941B78482F6FEF8F2D0E949B8FEDCFD5
:107D600082E40E94867A882339F00E941B78482F8B
:107D70006FEF84E00E949B8F0E943F6785C0E4E91B
:107D8000FFE384918F010F5F1F4F882321F00E9432
:107D9000DD77F801F6CFE1E9F6E084918F010F5F1E
:107DA0001F4F882309F470C00E94DD77F801F5CFDA
:107DB00081E0809363021092860683E50E94C17978
:107DC000811103C00E94C8D85FC00E942C78811125
:107DD0005BC0F8CFF0908F06FF2021F1EBECFFE3C2
:107DE00084918F010F5F1F4F882321F00E94DD7760
:107DF000F801F6CF84E50E94DD776F2D70E080E01A
:107E000090E04AE00E94B36680E20E94DD7709EFCD
:107E100012E0F80181918F01882309F4F0C80E94D3
:107E2000DD77F7CF10928706EBECFFE384918F01AB
:107E30000F5F1F4F882321F00E94DD77F801F6CFF6
:107E400060E070E080EA96E00E94EB678AE00E94C2
:107E5000DD771AC0EBECFFE384918F010F5F1F4FBA
:107E6000882321F00E94DD77F801F6CF6091880623
:107E70007091890682EB96E00E94936482E20E94F0
:107E8000DD778AE00E94DD770E945ED886C34115C7
:107E9000510519F4AF014150510920E030E00C9434
:107EA000972980E00E9436C30C94EC330E940B7833
:107EB000AB01BC014093B4145093B5146093B61455
:107EC0007093B71483E094E10E945F5EDDCF802F52
:107ED0000E9465686E2D802F0E94507CF12CB701A6
:107EE000802F0E9484680630110529F4F092E0107A
:107EF000E092DF10C9CF0830110531F6F092DE10A4
:107F0000E092DD10C1CF0E943B780E9496F87093FA
:107F1000850F6093840F80E00E94648B0E943B7801
:107F200020E030E040E752E40E941FF3181644F0CE
:107F30000E94476160E08EEC93E00E94B28802C02C
:107F40000E9490616091840F7091850F882777FD62
:107F50008095982F0E9425F3209146063091470680
:107F600040914806509149060E9478F918160CF085
:107F700064C184ED92E09F938F9382EC93E09F9392
:107F80008F931F920E9495600F900F900F900F900B
:107F90000F9081E08093830267961CAE1DAE1EAEEB
:107FA0001FAE67976B961CAE1DAE1EAE1FAE6B97D5
:107FB00010E0A0961FAEA0973CE3A4963FAFA49715
:107FC0004CE1A8964FAFA89756E4AC965FAFAC973C
:107FD000C12CD12C60E8E62E7FEBF72E812C912C62
:107FE00054016091840F7091850F882777FD8095EB
:107FF000982F0E9425F3062F772E682E592E262FB4
:10800000372F482F592FB601C7010E941FF388232D
:10801000D9F020914606309147064091480650918C
:108020004906602F772D862D952D0E941FF3182F5E
:10803000111F1127111F60968FAD6097882341F0A3
:10804000112331F011E0E7C00C2D7D2C6E2C5F2C3C
:108050000E94897C6B017C01DC01CB016B962CAD0D
:108060003DAD4EAD5FAD6B97821B930BA40BB50B73
:10807000B7FD3BC0D701C60188519C4FAF4FBF4FE2
:108080006B968CAF9DAFAEAFBFAF6B970E9499EC74
:10809000EEEBF3E084911F019FEF291A390A882340
:1080A00021F00E94DD77F101F5CF81149104A10444
:1080B000B104A9F0C501B40168517C4F8F4F9F4FA7
:1080C0006C197D098E099F0928EE33E040E050E0ED
:1080D0000E94F4F6CA01B9010E94246703C08FE32D
:1080E0000E94DD778AE00E94DD7780E00E9436C33F
:1080F0000E941D7DA09146066C96AFAF6C972090B4
:10810000470630904806409049062A2F322D432DCD
:10811000542D602F772D862D952D0E9451F79F7736
:1081200020E030E040E251E481149104A104B10464
:1081300029F40E941FF387FD05C006C00E9478F94C
:10814000181614F446015701112309F44AC0679622
:108150002CAD3DAD4EAD5FAD6797211531054105A5
:10816000510541F0D701C601821B930BA40BB50B3F
:10817000B7FD37C06C962FAD6C97322D432D542D23
:10818000A0966FADA097A4967FADA497A8968FAD4B
:10819000A897AC969FADAC970E9451F720E030E0D5
:1081A00040EC5FE30E941FF387FD4CCFD701C6016F
:1081B000805A9541AF4FBF4F67968CAF9DAFAEAF22
:1081C000BFAF67976C969FAD6C97A0969FAFA09737
:1081D000A4962FAEA497A8963FAEA897AC964FAEA4
:1081E000AC97809183028823B1F081149104A1049B
:1081F000B10429F4C02ED72CE62CF52CF2CEA8EE33
:10820000CA1AA3E0DA0AE108F108C818D908EA088E
:10821000FB08F7FCEFCF80918302882309F434CE6A
:1082200060E0112329F082EA93E00E94B2882CCE0C
:1082300080EB93E00E94B28827CE6096FFAD6097F6
:10824000F111A7CE8FED92E096CE0E943B780E946E
:1082500096F86739710514F066E970E07093810F44
:108260006093800F0E94198B0E943B7820E030E0E1
:1082700040EA50E40E9478F9181614F40E949061C4
:108280006091800F7091810F882777FD8095982FDE
:108290000E9425F320914A0630914B0640914C06EE
:1082A00050914D060E941FF360E087FF03C08EEFE0
:1082B00093E002C081EF93E00E94B28881E0809356
:1082C0008302809187068093610667961CAE1DAE7F
:1082D0001EAE1FAE67976B961CAE1DAE1EAE1FAED8
:1082E0006B9760961FAE6097A0961FAEA097BCE3F9
:1082F000A496BFAFA497ECE1A896EFAFA897F6E4D9
:10830000AC96FFAFAC97C12CD12C40E8E42E5FEBCC
:10831000F52E812C912C54016091800F7091810F6A
:10832000882777FD8095982F0E9425F3162F072F19
:10833000782E692E262F372F482F592FB601C701C7
:108340000E941FF3882331F120914A0630914B0699
:1083500040914C0650914D06612F702F872D962D20
:108360000E941FF3881F8827881F60968FAF609731
:108370006C962FAD6C97222389F0882379F0809139
:108380008302882309F480CD60E083EE93E00E94AD
:10839000B2887ACD1C2D0D2D7E2C6F2C0E94897CED
:1083A0006B017C01DC01CB016B962CAD3DAD4EAD7C
:1083B0005FAD6B97821B930BA40BB50BB7FD3BC056
:1083C000D701C60188519C4FAF4FBF4F6B968CAF02
:1083D0009DAFAEAFBFAF6B970E9499ECEDEEF3E0AF
:1083E00084912F019FEF491A590A882321F00E9496
:1083F000DD77F201F5CF81149104A104B104A9F055
:10840000C501B40168517C4F8F4F9F4F6C197D0996
:108410008E099F0928EE33E040E050E00E94F4F618
:10842000CA01B9010E94246703C08FE30E94DD776F
:108430008AE00E94DD7780E00E9436C30E941D7DA5
:1084400020904A0630904B0640904C0650904D06C6
:108450009101A201612F702F872D962D0E9451F757
:108460009F7720E030E040EA50E481149104A104B9
:10847000B10429F40E941FF387FD05C006C00E94C5
:1084800078F9181614F4460157016096AFAD60975D
:10849000AA2309F443C067962CAD3DAD4EAD5FAD48
:1084A0006797211531054105510541F0D701C601F6
:1084B000821B930BA40BB50BB7FD30C09101A20139
:1084C000A0966FADA097A4967FADA497A8968FAD08
:1084D000A897AC969FADAC970E9451F720E030E092
:1084E00040EC5FE30E941FF387FD49CFD701C6012F
:1084F000805A9541AF4FBF4F67968CAF9DAFAEAFDF
:10850000BFAF6797A0962FAEA097A4963FAEA49753
:10851000A8964FAEA897AC965FAEAC9780918302B9
:10852000882309F42CCF81149104A104B10429F407
:10853000C12ED02EE72CF62CEFCE98EEC91A93E080
:10854000D90AE108F108C818D908EA08FB08F7FEBB
:1085500016CFEECF0E94F5AE88E50E94C179882340
:1085600019F0179A1092B10789E50E94C179882302
:1085700019F0169A1092B2078AE50E94C1798823F1
:1085800019F0159A1092B30785E40E94C1798823E7
:1085900009F47ACC0E946C7877CCCA57DF4F0FB6BB
:1085A000F894DEBF0FBECDBFDF91CF911F910F9129
:1085B000FF90EF90DF90CF90BF90AF909F908F9003
:1085C0007F906F905F904F903F902F9008950F9302
:1085D000CF93DF93C82FD62F04E0262F41E3682FD7
:1085E00084E891E10E94677B8823C9F02D2F41E345
:1085F0006C2F84E891E10E942ADA8C2F0E943B5173
:108600008FEF8D0F8C0F0E943B512D2F44E36C2F69
:1086100084E891E1DF91CF910F910C942ADADF91F8
:10862000CF910F9108957F928F929F92AF92BF92B8
:10863000CF92DF92EF92FF920F931F93CF93DF932E
:10864000CDB7DEB72A970FB6F894DEBF0FBECDBF09
:1086500010920A1180910211882351F00E94FB822E
:1086600040E050E0BA018CE093EE0E94D389C9C487
:1086700040919C0250919D028091061190910711AA
:10868000A0910811B09109119A01280F391F4436A1
:10869000510524F4253631053CF41CC044365105FF
:1086A00051F024363105B4F484E690E090939D02B5
:1086B00080939C0213C08B309105A105B1051CF07D
:1086C0002A50310907C0863F9F4FAF4FBF4F74F408
:1086D000265F3F4F30939D0220939C02109206111B
:1086E00010920711109208111092091180919C02AA
:1086F00090919D028A3091053CF0883E23E09207DC
:108700002CF087EE93E002C08AE090E090939D0207
:1087100080939C020E94CF88782E0E94CF6980911E
:10872000B811853198F4772049F08091DD1090914F
:10873000DE10892B19F00EE513E102C001E412E10D
:1087400023E14FE061E089E00E94E6508091B8119A
:108750008D3108F084C1883008F03FC080918406D4
:10876000711002C0811139C06091840F7091850F22
:10877000882777FD8095982F0E9425F320E030E030
:1087800040E05FE30E9452F70E9496F8643671055C
:108790002CF46A30710524F04CE003C042E101C0C2
:1087A00046E022E130E0241B310937FF02C02F5F91
:1087B0003F4F359527953195219531092B5F2093B2
:1087C000BB1127E02093BC11CB010E9457870E9468
:1087D0002C6A8EE392E10E941F6A8091B8118D315C
:1087E000D0F58091BA118531B0F120E030E040E061
:1087F0005FE360914606709147068091480690912C
:1088000049060E9452F70E9496F89B016436710552
:108810000CF0F4C22A3031050CF4EEC24CE022E137
:1088200030E0241B310937FF02C02F5F3F4F3595E1
:1088300027953195219531092B5F2093BB112CE1B0
:108840002093BC11CB010E9457870E942C6A8EE3B3
:1088500092E10E941F6A8091B811853140F58091A4
:10886000BA11813120F16091840F7091850F8827B2
:1088700077FD8095982F0E9425F320914606309130
:10888000470640914806509149060E9478F918160B
:108890000CF0B6C21092A41102E022E041E16DE0BA
:1088A00084E891E10E94AADA81E08093A41180918A
:1088B000B811883008F03FC080919606711002C050
:1088C000811139C06091800F7091810F882777FDE9
:1088D0008095982F0E9425F320E030E040E05FE390
:1088E0000E9452F70E9496F8643671052CF46A30A3
:1088F000710524F04CE003C042E101C046E022E1F2
:1089000030E0241B310937FF02C02F5F3F4F359500
:1089100027953195219531092F5A2093BB1127E0D6
:108920002093BC11CB010E9457870E942C6A8EE3D2
:1089300092E10E941F6A8091B8118D31D0F580912B
:10894000BA118531B0F120E030E040E05FE36091A2
:108950004A0670914B0680914C0690914D060E94FC
:1089600052F70E9496F89B01643671050CF053C2D1
:108970002A3031050CF44DC24CE022E130E0241BDA
:10898000310937FF02C02F5F3F4F3595279531954D
:10899000219531092F5A2093BB112CE12093BC1152
:1089A000CB010E9457870E942C6A8EE392E10E94BD
:1089B0001F6A8091B811853140F58091BA118131DB
:1089C00020F16091800F7091810F882777FD80954D
:1089D000982F0E9425F320914A0630914B06409132
:1089E0004C0650914D060E9478F918160CF015C2ED
:1089F0001092A41102E022E042E168E584E891E1EE
:108A00000E94AADA81E08093A4118091B8118C3180
:108A100030F58091BA11843110F18091DD10909180
:108A2000DE10019644E6489F9001499F300D1124C5
:108A300037FF02C021503F4F832F932F990F990B7F
:108A4000009769F028E62093BB112BE12093BC111D
:108A50000E9457870E942C6A85E20E94EE698091ED
:108A6000B811843328F48091BA118A3208F0DEC13B
:108A70008091B811853328F48091BA11813308F0C0
:108A8000FAC180911112882309F44DC08091B81168
:108A9000843308F048C08091BA11823308F443C08F
:108AA00080910614882309F4EAC18091B014909152
:108AB000B114A091B214B091B3140097A105B105FF
:108AC00009F4DDC1BC01CD016D597F4F8F4F9F4F20
:108AD00024E630E040E050E00E94F4F66091B414E7
:108AE0007091B5148091B6149091B7140E94F4F669
:108AF000622F48E4649FB0011124882777FD809598
:108B0000982F0E9425F32AE037ED43E25CE30E94B0
:108B100084F30E949BF8262F02E042E367E384E897
:108B200091E10E94AADA8091B811813308F05DC00A
:108B30008091BA11893208F458C00E945C616B01BF
:108B40007C018CE3882E912CA12CB12CC701B6019D
:108B5000A50194010E94F4F6CA01B901A50194018E
:108B60000E94F4F6CA01962E872E59018E010F5FDE
:108B70001F4F41E8C41641E5D40641E0E406F10484
:108B800008F47FC1B90128E130E040E050E00E94E4
:108B9000F4F679018F929F92C50168E170E00E941E
:108BA00016FA9F938F933F932F932EE737E03F93CF
:108BB0002F931F930F930E94B9F20FB6F894DEBF64
:108BC0000FBECDBF9AE0E916F10408F489C198E020
:108BD000892F880F890F8195855A8093BB1180E377
:108BE0008093BC11C8010E942C6AE0917E11F09123
:108BF0007F1184818111CCC06091C0077091C10741
:108C00008091C2079091C3070E9496F8CB010E9401
:108C1000EE86BC018CEA96E00E948EFA6091C40751
:108C20007091C5078091C6079091C7070E9496F87A
:108C3000CB010E94EE86BC0187EA96E00E948EFA84
:108C40002CEA35EC47E257E36091C8077091C907F9
:108C50008091CA079091CB070E9452F720E030E044
:108C600048EC52E40E9484F30E9496F86B017C0168
:108C700097FD19C090E1C91697E2D906E104F10405
:108C8000E4F0C701B60120E137E240E050E00E9485
:108C900016F7CA01B9012AE030E040E050E00E9436
:108CA00016F7605D0BC0F094E094D094C094C11CA2
:108CB000D11CE11CF11C6DE201C060E260939806DA
:108CC00028EEC21623E0D206E104F10494F0C701B5
:108CD000B60128EE33E040E050E00E9416F7CA01EA
:108CE000B9012AE030E040E050E00E9416F7605DF4
:108CF00001C060E260939906C701B60124E630E046
:108D000040E050E00E9416F79AE0892E912CA12CA9
:108D1000B12CCA01B901A50194010E9416F7605D4A
:108D200060939A06C701B601A50194010E9416F747
:108D3000162F662381F08EE280939B06CA01B9014B
:108D4000A50194010E9416F7605D60939C06105D7A
:108D500010939D0617C0CA01B901A50194010E9494
:108D600016F7662339F08EE280939B06605D609370
:108D70009C0605C080E280939C0680939B0680E25F
:108D800080939D0668E976E080EA96E00E948EFA7C
:108D90008091B8118632A8F48091BA118E3188F092
:108DA00008E020E84EE160E084E891E10E94AADA60
:108DB0008091B811863228F48091BA118F3108F071
:108DC00091C08091B811823328F48091BA118C320D
:108DD00008F0F8C08091B8118F3308F012C180916B
:108DE000BA11883308F40DC11092BB118EE3809341
:108DF000BC110E94806A05C146E011CD42E10FCD51
:108E000002E022E041E16DE084E891E10E94AADA0B
:108E10004ECD46E0B2CD42E1B0CD02E022E042E1EB
:108E200068E584E891E10E94AADAEFCD07E028E046
:108E30004AE26AE284E891E10E94AADA05E022E0CF
:108E40004CE262E384E891E10E94AADA6AE08AE2F5
:108E5000BEDB609186117091871182E38093A0112F
:108E60008BE28093A11120EA31E142E384E891E1B1
:108E70000E94897BFDCD6AE486E3A9DB02CE60E037
:108E800038CE44E6A416B104C0F48F929F92C50177
:108E900068E170E00E9416FA9F938F9384E797E051
:108EA0009F938F931F930F930E94B9F20FB6F8947C
:108EB000DEBF0FBECDBF95E08BCE8F929F923F93CA
:108EC0002F938CE697E09F938F931F930F930E94AD
:108ED000B9F20FB6F894DEBF0FBECDBF96E078CEE4
:108EE00097E076CE1092A41183E08093BB1185E2C7
:108EF0008093BC11772029F08CE392E10E941F6AD5
:108F00000DC080917B06811102C08FE305C0809166
:108F1000B1078111F1CF80E20E94EE698BE080936E
:108F2000BB1115E21093BC118CEA96E00E942C6AEA
:108F30008BE28093BB111093BC11772029F08AE358
:108F400092E10E941F6A0DC080917C06811102C0CF
:108F50008FE305C08091B2078111F1CF80E20E94BA
:108F6000EE6983E38093BB1115E21093BC1187EA8D
:108F700096E00E942C6A83E58093BB111093BC118C
:108F8000772029F088E392E10E941F6A0DC080914A
:108F90007D06811102C08FE305C08091B307811166
:108FA000F1CF80E20E94EE698BE58093BB1185E2F0
:108FB0008093BC1180EA96E00E942C6A81E0809345
:108FC000A411FFCE84E00E94D66983E08093BB1198
:108FD00012E31093BC1186E00E940D6A0E94CF69D3
:108FE0008CE08093BB111093BC1180919C029091F6
:108FF0009D020E9457870E942C6A85E20E94EE69BA
:10900000E9CE2A960FB6F894DEBF0FBECDBFDF9132
:10901000CF911F910F91FF90EF90DF90CF90BF9075
:10902000AF909F908F907F9008951F93CF93DF9381
:1090300010920A118091061190910711A0910811C8
:10904000B091091181309048A105B10540F010920E
:109050000611109207111092081110920911C09177
:10906000061140919406141604F5842F992787FD64
:10907000909505972C2F332727FD30952817390712
:10908000A4F045301CF0CBEFC40F01C0C0E08C2F22
:10909000992787FD9095A92FB92F8093061190935A
:1090A0000711A0930811B0930911C0930311D0E0E8
:1090B00012E0C11109C080919E028823D9F121E0FC
:1090C00041E069E277E020C0C13049F480919E021E
:1090D000882381F120E041E06AE177E015C0C230E9
:1090E00049F480919E02882329F120E041E06AE062
:1090F00077E00AC0C33061F480919E028823D1F0EA
:1091000020E041E063E077E08D2F0E944F9212C093
:10911000C43081F480919E02882351F021E040E028
:1091200068EF76E08D2F0E944F928D2F0E94376A54
:1091300010939E02DF5FCF5FD53009F0BACFD09396
:109140009406DF91CF911F9108951F93CF93DF93E2
:1091500010920A118091061190910711A0910811A7
:10916000B091091181309048A105B10540F01092ED
:109170000611109207111092081110920911C09156
:10918000061140919306141604F5842F992787FD44
:10919000909505972C2F332727FD309528173907F1
:1091A000A4F045301CF0CBEFC40F01C0C0E08C2F01
:1091B000992787FD9095A92FB92F80930611909339
:1091C0000711A0930811B0930911C0930311D0E0C7
:1091D00012E0C11109C080919E028823D9F121E0DB
:1091E00041E06BEE76E020C0C13049F480919E02F0
:1091F000882381F120E041E062EE76E015C0C230C4
:1092000049F480919E02882329F120E041E062ED3B
:1092100076E00AC0C33061F480919E028823D1F0C9
:1092200020E041E060ED76E08D2F0E944F9212C069
:10923000C43081F480919E02882351F021E040E007
:1092400065EC76E08D2F0E944F928D2F0E94376A39
:1092500010939E02DF5FCF5FD53009F0BACFD09375
:109260009306DF91CF911F9108950F931F93CF9392
:10927000DF9310920A118091061190910711A0912D
:109280000811B091091181309048A105B10540F055
:1092900010920611109207111092081110920911E4
:1092A000C0910611409195061416D4F4842F992785
:1092B00087FD909501972C2F332727FD3095281790
:1092C000390774F0CFEFC40F8C2F90E0A0E0B0E02E
:1092D0008093061190930711A0930811B093091180
:1092E0001092041180910311C81714F4C093031154
:1092F00080910311992787FD909504962C2F332791
:1093000027FD30958217930724F48CEF8C0F809300
:10931000031110910311D0E081E002E0111123C08C
:109320008823B9F01C16ACF040910611509107113A
:1093300060910811709109114F5F5F4F6F4F7F4F20
:10934000409306115093071160930811709309110F
:10935000CF5F80919E02882309F469C021E041E03B
:109360006DE577E04EC0113019F58823B9F0C230B1
:10937000ACF4409106115091071160910811709161
:1093800009114F5F5F4F6F4F7F4F4093061150930E
:1093900007116093081170930911CF5F80919E02AD
:1093A000882309F444C020E040E068E477E029C065
:1093B0001230E9F480910211811105C080919E0262
:1093C0008823A9F109C0C230C9F70E94318A80916F
:1093D0000411882399F333C081E0C23009F080E0A2
:1093E00024E043E457E06D2F0E9476DB20C0133069
:1093F00061F480919E028823D1F020E041E061E495
:1094000077E08D2F0E944F9212C0143081F480912A
:109410009E02882351F021E040E066E377E08D2F43
:109420000E944F928D2F0E94376A00939E02DF5F49
:109430001F5FD53011F080E071CFD0939506DF919A
:10944000CF911F910F9108952F923F924F925F926B
:109450006F927F928F929F92AF92BF92CF92DF9244
:10946000EF92FF920F931F93CF93DF93CDB7DEB7A9
:109470002B970FB6F894DEBF0FBECDBF9E838D83B2
:10948000DC0159962D903C905A97F1014184528409
:1094900063847484FFEF4F1A5F0A6F0A7F0A149681
:1094A000CD90DD90ED90FC901797C114D104E104AC
:1094B000F10439F02FEFC21AD20AE20AF20A1B862F
:1094C00007C0D101CD90DD90ED90FC90B1E0BB875D
:1094D000460157011F82188619861A86F101818577
:1094E0009285A385B4852F81388549855A852817AB
:1094F00039074A075B0708F08DC04C145D046E0401
:109500007F0450F482E0C82ED12CE12CF12C92E0A3
:10951000892E912CA12CB12C9E012F5F3F4FB701BA
:10952000A601C1010E94665C882309F473C0898189
:109530009A81AB81BC81892B8A2B8B2B41F0460110
:1095400057013FEF831A930AA30AB30A05C0C81450
:10955000D904EA04FB0489F08F819885A985BA852E
:109560000196A11DB11D8F839887A987BA879FEFA8
:10957000C91AD90AE90AF90AB1CF0FEF1FEF2FEF85
:109580003FE0B501A401C1010E94AF5FF82E88231E
:1095900009F440C0ED81FE81448155816681778167
:1095A000411551056105710539F095018401C1012D
:1095B0000E94AF5F882371F1AD81BE8114968D92B8
:1095C0009D92AD92BC921797BB85BB2351F0D501FC
:1095D000C4010196A11DB11DF10180839183A28375
:1095E000B383ED81FE8185899689A789B08D892B0A
:1095F0008A2B8B2B81F4AD81BE8155968D929D92E5
:10960000AD92BC92589711968C91119780681196E3
:109610008C9301C0F12C8F2D2B960FB6F894DEBFE2
:109620000FBECDBFDF91CF911F910F91FF90EF90B3
:10963000DF90CF90BF90AF909F908F907F906F9072
:109640005F904F903F902F900895CF93DF93EC0160
:109650008B81882391F1898187FF2BC06C857D8563
:109660008E859F8541E00E942F5C882331F1E88937
:1096700080E2E89FF0011124E35CFB4F3097E9F0B2
:109680008081853ED1F08B81823040F449895A89AE
:109690006B897C89448F558F668F778F4D895E8962
:1096A0006F89788D538F428F758B648B89818F770B
:1096B0008983DF91CF910C94F15B81E0888380E016
:1096C000DF91CF910895CF93DF93EC018B818130AF
:1096D00099F4898181FF10C049895A896B897C89F5
:1096E000452B462B472B59F140E050E0BA01CE0103
:1096F0000E945F5E811102C080E022C04D895E89B8
:109700006F89788D898D9A8D0E943E608823A1F3A0
:109710001D8A1E8A1F8A188E198A1A8A1B8A1C8A19
:10972000898180688983CE0190DF882329F340E016
:1097300050E0BA01CE01DF91CF910C945F5E81E0E1
:10974000DF91CF9108956F927F928F929F92AF9207
:10975000BF92CF92DF92EF92FF920F931F93CF931E
:10976000DF931F92CDB7DEB78C015B014A01722EE9
:10977000DB0159968D919C915A97F801928F818FB8
:1097800040E050E0BA01C5010E945F5EE12CF501A6
:1097900080859185A285B3854189528963897489C1
:1097A00084179507A607B70708F0CEC035E0B69531
:1097B000A795979587953A95D1F7F82FFF70FF2ECB
:1097C000D50113968C91823008F49BC141E050E0A2
:1097D000BE016F5F7F4FC5010E94E55C019719F4E0
:1097E000898190E002C08FEF9FEF019609F489C153
:1097F000F50180859185A285B3854F96A11DB11D88
:1098000080879187A287B387F0E2FF9EB001112481
:10981000635C7B4F6115710509F473C1DB018C91A9
:10982000882311F0853EB9F4E1100EC08091B40692
:109830009091B506A091B606B091B706F80184875D
:109840009587A687B787F08ADB018C91EE24E39495
:1098500081119DCF79C04BE050E0C4010E944FFAC6
:10986000892B09F094CF77FC4CC120E2F29EF001E5
:109870001124E35CFB4F8385817121F0872D827178
:1098800009F05EC04091B4065091B5066091B606ED
:109890007091B706D8011C964D935D936D937C93A0
:1098A0001F975096FC924489558960E070E0BA0198
:1098B00055274427828D938DA0E0B0E0482B592B8B
:1098C0006A2B7B2BD80155964D935D936D937C93BA
:1098D00058978385887159F4848D958DA68DB78DA1
:1098E000F801818B928BA38BB48B81E010C0803107
:1098F00039F598012F5E3F4FD80159968D919C9173
:109900005A970E94F85E8823D9F084E0F801838397
:10991000872D8F70D80111968C931197F8011482BE
:1099200015821682178218961D921D921D921C9206
:109930001B9774FED9C0C801C6DE8111D5C0E2C034
:10994000D80113961C92DDC0872D8274823409F0F1
:10995000D8C0EE20E1F0D8015096FC9050971C96AC
:109960006D917D918D919C911F9741E00E942F5C9C
:10997000882309F4C6C0F8018089F0E28F9FC001F6
:109980001124835C9B4F009709F08EC0BAC0D501AB
:1099900013968C911397823009F4B3C051968D9130
:1099A0009D910D90BC91A02D803E9F4FAF41B10580
:1099B00008F0A7C0C50148DD882309F4A2C00E94B1
:1099C000F15B882309F49DC0D5015996ED91FC9176
:1099D0005A971496CD90DD90ED90FC901797B2E0D9
:1099E000CB1AD108E108F108058404C0CC0CDD1CB9
:1099F000EE1CFF1C0A94D2F786859785A089B18951
:109A0000C80ED91EEA1EFB1E81E08093B306C092E9
:109A1000B406D092B506E092B606F092B70680E0A2
:109A200092E0EDE3F4E0DF019C011D922150304013
:109A3000E1F766246394D5015996ED91FC915A970C
:109A40008481681698F42DE334E0B701A601460D31
:109A5000511D611D711D8091B1069091B2060E9449
:109A6000855B882309F44DC06394E5CF40E052E064
:109A700060E070E0058404C0440F551F661F771F27
:109A80000A94D2F751968D919D910D90BC91A02D85
:109A9000840F951FA61FB71FF501818B928BA38B97
:109AA000B48B8DE394E0F12C20E2DC011D922A9529
:109AB000E9F72BE0F401DC0101900D922A95E1F722
:109AC00021E238E2FC01318B208B40E058E05787DF
:109AD0004687338B228B318F208F578B468B0E948A
:109AE000F15B8111C2CE0DC075FE09C0F80141893C
:109AF000528963897489C8010E945F5E03C081E056
:109B000001C080E00F90DF91CF911F910F91FF90E6
:109B1000EF90DF90CF90BF90AF909F908F907F900D
:109B20006F9008952F923F924F925F926F927F9223
:109B30008F929F92AF92BF92CF92DF92EF92FF925D
:109B40000F931F93CF93DF9300D01F921F92CDB737
:109B5000DEB78C015B014D83252EDC0113968C91C1
:109B600013978130C9F411968C9181FF15C082FF43
:109B700019C0F8014189528963897489808591856A
:109B8000A285B38584179507A607B70759F0C801C2
:109B90000E945F5E811106C081E0F80180838FEF33
:109BA0009FEF2DC1ED80F22C80C0D8015996ED9128
:109BB000FC915A9734803A94DB01CA0169E0B6956A
:109BC000A795979587956A95D1F738224A01B1E014
:109BD0009B22332009F475C080E092E0881999092E
:109BE00067018E159F0508F46C01D8015996ED9117
:109BF000FC915A9714964D905D906D907C901797BC
:109C0000B2E04B1A510861087108058404C0440C85
:109C1000551C661C771C0A94D2F786859785A08907
:109C2000B189480E591E6A1E7B1E430C511C611CD3
:109C3000711CC114E2E0DE0609F08BC08091B4060D
:109C40009091B506A091B606B091B706841595051A
:109C5000A605B70569F41092B3068FEF9FEFDC01FC
:109C60008093B4069093B506A093B606B093B7065A
:109C70009501B301A2018091B1069091B2060E94B4
:109C8000855B882309F488CFF80180859185A285BA
:109C9000B3858C0D9D1DA11DB11D80879187A28765
:109CA000B387AC0CBD1CEC18FD08D80118964D917B
:109CB0005D916D917C911B97E114F10409F075CFD2
:109CC0007EC08114910409F087CFD80114964D917C
:109CD0005D916D917C911797411551056105710555
:109CE00059F455968D919D910D90BC91A02D0097A2
:109CF000A105B10541F522C09E012F5F3F4FCF0165
:109D00000E94665C882309F447CF89819A81AB81E0
:109D1000BC81F801218D328DF9012789203139F478
:109D2000883FFFEF9F07A105B10540F40CC0883FB5
:109D30002FEF9207A2072FE0B20728F0C80184DBBB
:109D400081114ACF29CFF80184839583A683B783F5
:109D500043CF8114910419F5D80118964D915D9166
:109D60006D917C911B9751968D919D910D90BC9119
:109D7000A02D481759076A077B0788F00E94F15BFE
:109D8000882309F409CF81E08093B3064092B4069A
:109D90005092B5066092B6067092B70608C041E0D0
:109DA000C301B2010E942F5C882309F4F5CEA601FD
:109DB000B501C401835C9B4F0E945CFA65CF51964C
:109DC0008D919D910D90BC91A02D84179507A607AC
:109DD000B70740F4F801418B528B638B748B818100
:109DE00080688183D80111968C9183FD03C08D8199
:109DF000922D05C0C80129DC8111F9CFCDCE0F907D
:109E00000F900F900F900F90DF91CF911F910F91B6
:109E1000FF90EF90DF90CF90BF90AF909F908F908A
:109E20007F906F905F904F903F902F900895CF93C9
:109E3000DF931F92CDB7DEB7698341E050E0BE01EA
:109E40006F5F7F4F04966EDE0F90DF91CF91089584
:109E5000CF93DF93EC01F9DB1B82DF91CF91089563
:109E60001092111280910614882319F083E094E176
:109E7000EFCF0895CF92DF92EF92FF921F93CF938F
:109E8000DF931092121280916C12882319F089E6E8
:109E900092E1DEDF1092E0131092DD1385E38093F0
:109EA000DC130E94897CEB01A8958091DC130E9451
:109EB00065688CED93E10E94857C2398229A219A13
:109EC000209A289A85E08093DE1382E58CBD1DBC24
:109ED0001AE08FEF0E94D1771150D9F720E030E0DF
:109EE000A90160E08CED93E10E94AD7C182F809376
:109EF000DF13813049F00E94897C6C1B7D0B613D32
:109F0000774060F381E054C02AEA31E040E050E05D
:109F100068E08CED93E10E94AD7C82FF03C010935A
:109F2000E0130EC014E00E94D6778093DF13115027
:109F3000D1F78A3A11F082E03BC082E08093E013CF
:109F40008091E013823031F4C12CD12CE12C70E4EB
:109F5000F72E03C0C12CD12C760120E030E0A901FE
:109F600067E38CED93E10E94AD7CA701960169E265
:109F70008CED93E10E94AD7C8093DF13882349F040
:109F80000E94897C6C1B7D0B613D774030F38AE039
:109F90000FC08091E013823011F520E030E0A9017C
:109FA0006AE38CED93E10E94AD7C882351F088E058
:109FB0008093DD138CED93E10E94857CEBECFFE355
:109FC0001AC00E94D677807C803C19F483E080938D
:109FD000E0130E94D6770E94D6770E94D6778CED48
:109FE00093E10E94857C1092DE1381E00E948F6ACB
:109FF000811132C015C08491EF012196882321F090
:10A000000E94DD77FE01F7CFECEAF4E18491EF01E5
:10A010002196882309F457C00E94DD77FE01F6CF10
:10A0200080E00E948F6A811117C0E4E9FFE3849108
:10A03000EF012196882321F00E94DD77FE01F7CF02
:10A04000E8E9F4E18491EF012196882309F43BC00B
:10A050000E94DD77FE01F6CF61EE73E189E692E1C1
:10A060000E945E5F811116C0E4E9FFE38491EF0175
:10A070002196882321F00E94DD77FE01F7CFE7E8E3
:10A08000F4E18491EF0121968823E9F00E94DD77C5
:10A09000FE01F7CF81E080931212EBECFFE3849195
:10A0A000EF012196882321F00E94DD77FE01F7CF92
:10A0B000EBE7F4E18491EF012196882321F00E94DF
:10A0C000DD77FE01F7CF8BE1E9E6F2E1AAE8B2E144
:10A0D00001900D928A95E1F7809167129091681234
:10A0E000909389128093881285E692E1909385126D
:10A0F00080938412DF91CF911F91FF90EF90DF90BA
:10A10000CF900895FC0123812111A2CE08952EE065
:10A1100033E0FC01318320830496F4CFCF92DF92A9
:10A12000EF92FF920F931F93CF93DF938C01EB017C
:10A130006A0179010E943D8923E020939E021093D9
:10A14000900700938F07D0938E07C0938D07A601C9
:10A15000662757FD6095762F4093890750938A07AD
:10A1600060938B0770938C07C701AA2797FDA09572
:10A17000BA2F841B950BA60BB70B80938507909382
:10A180008607A0938707B093880788819981AA27BB
:10A1900097FDA095BA2F841B950BA60BB70B809348
:10A1A000061190930711A0930811B09309118DE93E
:10A1B00090E89093680280936702DF91CF911F919E
:10A1C0000F91FF90EF90DF90CF9008958F929F9224
:10A1D000AF92BF92CF92DF92EF92FF920F931F93B5
:10A1E000CF93DF93882EB62EA42EF22EE801242FD3
:10A1F000220F220F220F0F2D462F682F84E891E1A6
:10A200000E94677B882351F10B2D0F0DCA2CD12C96
:10A21000B01621F17E019A2C182D9920D9F0F70162
:10A22000849160918611709187111093A011B09262
:10A23000A1111092A3118093A21120EA31E14BE306
:10A2400084E891E10E94897BFFEFEF1AFF0A9A945C
:10A25000185FE3CFCC0DDD1DB394DACFDF91CF9142
:10A260001F910F91FF90EF90DF90CF90BF90AF9034
:10A270009F908F90089560918611709187118093BF
:10A28000A01181E38093A11181E08093A31180EF5D
:10A290008093A21120EA31E14BE384E891E10C9430
:10A2A000897B0F931F93CF93DF938C01EB01DC012C
:10A2B00013968C918823C1F18250823028F48FE26A
:10A2C0008883198281E031C0F801648575858685AF
:10A2D000978540E00E942F5C882339F1D801509681
:10A2E000EC91B0E2EB9FF0011124E35CFB4F30975F
:10A2F000D9F090E020E03EE24081403269F0283021
:10A3000029F4DE01A90FB11D3C939F5F4081DE015E
:10A31000A90FB11D4C939F5F2F5F31962B3061F7D2
:10A32000C90FD11D188201C080E0DF91CF911F912C
:10A330000F910895CF93DF938091BD11811107C0D4
:10A3400081E08093BD1184E891E10E948D7BC091F2
:10A350008611D0918711E091B511F091B61182E08C
:10A360001995E091B511F091B61181E0199520E0B1
:10A3700030E044E1BE0184E891E10E94897B27EB53
:10A3800031E147E1BE0184E891E10E94897BE091DF
:10A39000B511F091B61180E0DF91CF911994CF9370
:10A3A000DF93C091DB13CC23C1F0C150C093DB130A
:10A3B0008FE1C89FE0011124CB55DD4E8BE1FE01FA
:10A3C0003496AAE8B2E101900D928A95E1F78A816C
:10A3D0009B8190938912809388121092031181E0DF
:10A3E0008093041183E080939E02DF91CF910895C2
:10A3F000CF92DF92EF92FF920F931F93CF93DF9351
:10A40000EC010E94897C0E811F8128853985011508
:10A4100011052105310559F53C853323A9F12A851C
:10A4200031503C8731E0320F3A874D85341301C0FB
:10A430001A86FE0134E0239FE00DF11D11240685EC
:10A440001785208931890A831B832C833D836B0107
:10A450007C01C00ED11EE11CF11CCE82DF82E88699
:10A46000F9868C819D81892B79F0769A0DC06B01DC
:10A470007C01C01AD10AE20AF30AF7FC05C07698FB
:10A480001E821F8218861986DF91CF911F910F912E
:10A49000FF90EF90DF90CF9008951092850F10926B
:10A4A000840F80E00E94648B1092810F1092800FC5
:10A4B0000E94198B0E9447611092850F1092840FA1
:10A4C00080E00E94648B10929A0F9FB7F894E2E0AC
:10A4D000F1E080818F7B80839FBF1092810F10926B
:10A4E000800F1092980F759808951092DE101092B8
:10A4F000DD101092E0101092DF10CFDF0C942B8A49
:10A500009091E2118091E311981731F08091E3115D
:10A510008F5F8F708093E31108950F931F93CF93F4
:10A52000DF93EC01FC01E65AFF4F1082138234974F
:10A53000138212828EE093E091838083B59610821D
:10A540001382349713821282918380838E010A567C
:10A550001F4F9E0124533E4FF801B8016C5F7F4F9F
:10A56000AC01CF01801B910B860F971FDC011C9261
:10A5700013961C9213821282518340837F96E217B6
:10A58000F30779F7CE0183539E4F29E1DC01119641
:10A590002C93119714961C920596DC0157961C92E9
:10A5A0008296DC011C9213961C920497DC01139690
:10A5B0001C921E9212972EE033E02D933C93198249
:10A5C00018821B821A828F549F4FDC011D921D92AC
:10A5D0001D921C9213970496DC011D921D921D92F0
:10A5E0001C9213971082FE01E15FFD4F108286E3FB
:10A5F00091E0F8019C01119221503040E1F7FE01F9
:10A60000E355FD4F81E08083E955F24011821082CD
:10A610000E94897CC755DD4F68577C4E8F4F9F4FF6
:10A62000688379838A839B83DF91CF911F910F91F8
:10A6300008952F923F924F925F926F927F928F92E6
:10A640009F92AF92BF92CF92DF92EF92FF920F93C1
:10A650001F93CF93DF93CDB7DEB768970FB6F8940B
:10A66000DEBF0FBECDBF1C015B018A01DC01D796A6
:10A670006D917D918D919C91DA970E9423F36B01EE
:10A680007C01F50120813181428153810E9484F354
:10A690000E9418F80E949BF869877A878B879C87AD
:10A6A000D8012D913D914D915C91C701B6010E9459
:10A6B00084F30E9418F80E949BF86D877E878F872D
:10A6C000988B29853A854B855C852837310541056E
:10A6D000510540F488E790E0A0E0B0E089879A87D0
:10A6E000AB87BC872D853E854F8558892837310536
:10A6F0004105510540F488E790E0A0E0B0E08D8787
:10A700009E87AF87B88B91012D5B3F4FD9018D910B
:10A710009D910D90BC91A02D8D839E83AF83B887B2
:10A72000BC01CD010E9425F369837A838B839C83CE
:10A7300069857A858B859C850E9423F3698B7A8B4A
:10A740008B8B9C8B20E030E0A90169817A818B8121
:10A750009C810E941FF3882339F1A7019601C7014C
:10A76000B6010E9484F34B015C0129893A894B8927
:10A770005C89CA01B9010E9484F39B01AC01C50147
:10A78000B4010E9451F74B015C0129813A814B8150
:10A790005C81CA01B9010E9452F79B01AC01C5015D
:10A7A000B4010E942EF803C060E070E0CB010E946B
:10A7B00018F80E9496F82B013C016D817E818F81F3
:10A7C000988590958095709561957F4F8F4F9F4F9D
:10A7D0000E9425F34B015C016D857E858F859889EC
:10A7E0000E9423F36D837E838F83988720E030E07F
:10A7F000A901C501B4010E941FF3882349F12D81ED
:10A800003E814F815885CA01B9010E9484F36D8B46
:10A810007E8B8F8B988FA7019601C701B6010E948E
:10A8200084F39B01AC016D897E898F89988D0E948C
:10A8300051F76B017C01A5019401C501B4010E948F
:10A8400052F79B01AC01C701B6010E942EF803C06C
:10A8500060E070E0CB010E94C7F8F1018288938824
:10A86000A488B58875016401C418D508E608F708FE
:10A870000E9496F8C61AD70AE80AF90AF7FE6BC0D2
:10A8800020E030E0A90169817A818B819C810E945E
:10A890001FF3882309F447C029813A814B815C81E9
:10A8A000CA01B9010E9452F76B017C01C501B401D4
:10A8B0000E9423F39B01AC01C701B6010E9484F3FF
:10A8C0006B017C0129893A894B895C89CA01B901EC
:10A8D0000E9484F39B01AC01C701B6010E9451F7AD
:10A8E0006B017C012D813E814F815885CA01B901E0
:10A8F0000E9484F39B01AC01C701B6010E9452F78C
:10A900006B017C0120E030E040E850E469817A810D
:10A910008B819C810E9484F39B01AC01C701B6012D
:10A920000E942EF803C060E070E0CB010E9418F88E
:10A930000E9496F82B013C0197FF03C0412C512C3B
:10A940003201481459046A047B0410F024013501D3
:10A95000C12CD12C76018FB7F894D1019C9193FD35
:10A9600022C0F101468A578A608E718EC40CD51CB4
:10A97000E61CF71C5A96CD92DD92ED92FC925D9703
:10A9800029853A854B855C85DB962D933D934D93C8
:10A990005C93DE97FF962D853E854F8558892083F1
:10A9A0003183428353838FBF68960FB6F894DEBF1E
:10A9B0000FBECDBFDF91CF911F910F91FF90EF9010
:10A9C000DF90CF90BF90AF909F908F907F906F90CF
:10A9D0005F904F903F902F9008955F988EBD00003C
:10A9E0000DB407FEFDCF8EB56EBD00000DB407FEA1
:10A9F000FDCF8EB55F9A0895CF93DF9300D01F925D
:10AA00001F92CDB7DEB795E0EFE9F2E0DE011196D7
:10AA100001900D929A95E1F7E1E0F0E0EC0FFD1F57
:10AA2000E80FF11D808190E00F900F900F900F9034
:10AA30000F90DF91CF91D1CF1F93CF93DF93C6E1DA
:10AA4000D3E010E089910E94C179882321F00E940F
:10AA50000B78812FD1DF1F5F1430A1F782E40E94B1
:10AA6000C179882321F00E940B7884E0C5DF83E55B
:10AA70000E94C179882341F0C0E00E940B788C2F9E
:10AA8000BBDFCF5FC530C9F7DF91CF911F9108952C
:10AA90004F925F926F927F928F929F92AF92BF92EE
:10AAA000CF92DF92EF92FF92CF93DF93EEE3F7E145
:10AAB0008491EF012196882321F00E94DD77FE0129
:10AAC000F7CF6091C0077091C1078091C207909144
:10AAD000C30742E00E94D4D1EAE3F7E18491EF0199
:10AAE0002196882321F00E94DD77FE01F7CF609147
:10AAF000C4077091C5078091C6079091C70742E0CF
:10AB00000E94D4D1E6E3F7E18491EF0121968823F6
:10AB100021F00E94DD77FE01F7CF6091C8077091A8
:10AB2000C9078091CA079091CB0742E00E94D4D117
:10AB3000E2E3F7E18491EF012196882321F00E945E
:10AB4000DD77FE01F7CF6091CC077091CD07809142
:10AB5000CE079091CF0742E00E94D4D18FB7F894EE
:10AB60004090450F5090460F6090470F7090480FEF
:10AB70008090490F90904A0FA0904B0FB0904C0FCF
:10AB8000C0904D0FD0904E0FE0904F0FF090500FAF
:10AB90008FBFE8E2F7E18491EF012196882321F04D
:10ABA0000E94DD77FE01F7CFC301B2010E94246746
:10ABB000E4E2F7E18491EF012196882321F00E94DD
:10ABC000DD77FE01F7CFC501B4010E942467E0E202
:10ABD000F7E18491EF012196882321F00E94DD772F
:10ABE000FE01F7CFC701B6010E9424678AE0DF911A
:10ABF000CF91FF90EF90DF90CF90BF90AF909F905C
:10AC00008F907F906F905F904F900C94DD77AF9214
:10AC1000BF92CF92DF92EF92FF920F931F93CF9349
:10AC2000C82F882319F0E8E0F7E10CC0EBECFFE354
:10AC300084918F010F5F1F4F8823A9F30E94DD7756
:10AC4000F801F6CF84918F010F5F1F4F882321F009
:10AC50000E94DD77F801F6CFCC2319F0EBEEF6E198
:10AC60000CC0EBECFFE384918F010F5F1F4F882333
:10AC7000A9F30E94DD77F801F6CF84918F010F5F71
:10AC80001F4F882321F00E94DD77F801F6CF8AE07C
:10AC90000E94DD77C1112DC0EBECFFE384918F01A1
:10ACA0000F5F1F4F882321F00E94DD77F801F6CF58
:10ACB000E8EDF6E184918F010F5F1F4F882321F0AB
:10ACC0000E94DD77F801F6CF80916206882321F09B
:10ACD0008AE00E94DD7762C3EDECF6E184918F019A
:10ACE0000F5F1F4F882309F459C30E94DD77F801D5
:10ACF000F5CF40915D0650915E0660915F067091C0
:10AD0000600684EC96E10E9466D28AE00E94DD77BC
:10AD10008091620681111BC0CC2319F0E9EBF6E1AA
:10AD20000CC0EBECFFE384918F010F5F1F4F882372
:10AD3000A9F30E94DD77F801F6CF84918F010F5FB0
:10AD40001F4F882321F00E94DD77F801F6CFC11153
:10AD500024C0EBECFFE384918F010F5F1F4F88232A
:10AD600021F00E94DD77F801F6CFE8EAF6E1849160
:10AD70008F010F5F1F4F882321F00E94DD77F801BC
:10AD8000F6CFEBECFFE384918F010F5F1F4F882319
:10AD900021F00E94DD77F801F6CF409174075091C1
:10ADA0007507609176077091770780EA96E10E94B7
:10ADB00066D2409178075091790760917A07709137
:10ADC0007B078DE996E10E9466D240917C07509105
:10ADD0007D0760917E0770917F078AE996E10E9466
:10ADE00066D24091800750918107609182077091EF
:10ADF000830787E996E10E9466D28AE00E94DD77A8
:10AE0000C11124C0EBECFFE384918F010F5F1F4F52
:10AE1000882321F00E94DD77F801F6CFE9E7F6E11B
:10AE200084918F010F5F1F4F882321F00E94DD77EF
:10AE3000F801F6CFEBECFFE384918F010F5F1F4F1A
:10AE4000882321F00E94DD77F801F6CF4091630757
:10AE500050916407609165077091660780E796E1FD
:10AE60000E9466D240916707509168076091690718
:10AE700070916A078DE696E10E9466D240916B0759
:10AE800050916C0760916D0770916E078AE696E1AC
:10AE90000E9466D240916F075091700760917107D0
:10AEA0007091720787E696E10E9466D28AE00E945E
:10AEB000DD77C11124C0EBECFFE384918F010F5FBC
:10AEC0001F4F882321F00E94DD77F801F6CFE5E4DB
:10AED000F6E184918F010F5F1F4F882321F00E94BC
:10AEE000DD77F801F6CFEBECFFE384918F010F5F84
:10AEF0001F4F882321F00E94DD77F801F6CF4091A3
:10AF0000E6105091E7106091E8107091E9108CE321
:10AF100096E10E9477D34091EA105091EB10609136
:10AF2000EC107091ED1089E396E10E9477D3409187
:10AF3000EE105091EF106091F0107091F11086E3D7
:10AF400096E10E9477D34091F2105091F3106091F6
:10AF5000F4107091F51083E396E10E9477D38AE0B4
:10AF60000E94DD77C11124C0EBECFFE384918F01D7
:10AF70000F5F1F4F882321F00E94DD77F801F6CF85
:10AF8000E9EEF5E184918F010F5F1F4F882321F0D7
:10AF90000E94DD77F801F6CFEBECFFE384918F019F
:10AFA0000F5F1F4F882321F00E94DD77F801F6CF55
:10AFB0004091FE105091FF106091001170910111AD
:10AFC00080EE95E10E9466D24091FA105091FB10FC
:10AFD0006091FC107091FD108DED95E10E9466D29C
:10AFE0004091F6105091F7106091F8107091F9109F
:10AFF0008AED95E10E9466D28AE00E94DD77C11158
:10B0000024C0EBECFFE384918F010F5F1F4F882377
:10B0100021F00E94DD77F801F6CFE6E6F5E18491B4
:10B020008F010F5F1F4F882321F00E94DD77F80109
:10B03000F6CFEBECFFE384918F010F5F1F4F882366
:10B0400021F00E94DD77F801F6CF40915F07509123
:10B05000600760916107709162078DE595E10E943C
:10B0600066D240915B0750915C0760915D077091DB
:10B070005E078AE595E10E9466D24091C70950912A
:10B08000C8096091C9097091CA0987E595E10E94D4
:10B0900077D34091910750919207609193077091F7
:10B0A000940784E595E10E9466D2409195075091FE
:10B0B0009607609197077091980781E595E10E9446
:10B0C00066D24091990750919A0760919B077091C1
:10B0D0009C078EE495E10E9466D240919D075091B5
:10B0E0009E0760919F077091A0078BE495E10E94F5
:10B0F00066D28AE00E94DD77C11124C0EBECFFE349
:10B1000084918F010F5F1F4F882321F00E94DD770C
:10B11000F801F6CFEDE3F5E184918F010F5F1F4F4A
:10B12000882321F00E94DD77F801F6CFEBECFFE3F6
:10B1300084918F010F5F1F4F882321F00E94DD77DC
:10B14000F801F6CF4091B4075091B5076091B6076A
:10B150007091B70784E395E10E9466D24091B807E9
:10B160005091B9076091BA077091BB0781E395E1EF
:10B170000E9466D24091BC075091BD076091BE0706
:10B180007091BF078EE295E10E9466D28AE00E942C
:10B19000DD77CC2379F089E5A82E86E0B82E91E5FD
:10B1A000C92E96E0D92E25E5E22E26E0F22E00E00B
:10B1B00010E024C0EBECFFE384918F010F5F1F4F81
:10B1C000882321F00E94DD77F801F6CFE1E1F5E177
:10B1D00084918F010F5F1F4F882321F00E94DD773C
:10B1E000F801F6CFEBECFFE384918F010F5F1F4F67
:10B1F000882389F20E94DD77F801F6CFB80188E054
:10B2000095E10E94EB67F501619171915F0185E025
:10B2100095E10E94EB67F601619171916F0182E007
:10B2200095E10E94EB67F701619171917F018FEFCA
:10B2300094E10E94EB678AE00E94DD770F5F1F4F69
:10B2400002301105D9F6C11124C0EBECFFE3849163
:10B250008F010F5F1F4F882321F00E94DD77F801D7
:10B26000F6CFE0EFF4E184918F010F5F1F4F882349
:10B2700021F00E94DD77F801F6CFEBECFFE384913B
:10B280008F010F5F1F4F882321F00E94DD77F801A7
:10B29000F6CF40918D0950918E0960918F09709180
:10B2A000900987EE94E10E9466D22CEA35EC47E2E1
:10B2B0005EE36091890970918A0980918B09909170
:10B2C0008C090E942EF8AB01BC0184EE94E10E942F
:10B2D0004AD22CEA35EC47E25EE360918509709131
:10B2E000860980918709909188090E9484F3AB01B7
:10B2F000BC0181EE94E10E944AD28AE00E94DD778F
:10B30000C1110CC0EBECFFE384918F010F5F1F4F65
:10B31000882321F00E94DD77F801F6CF409199094A
:10B3200050919A0960919B0970919C0988ED94E174
:10B330000E9466D22CEA35EC47E25EE36091950903
:10B340007091960980919709909198090E942EF822
:10B35000AB01BC0185ED94E10E944AD22CEA35ECA8
:10B3600047E25EE36091910970919209809193099F
:10B37000909194090E9484F3AB01BC0182ED94E1A9
:10B380000E944AD28AE0CF911F910F91FF90EF90D7
:10B39000DF90CF90BF90AF900C94DD77EBECFFE3A4
:10B3A00084918F010F5F1F4F882309F4A2CC0E9464
:10B3B000DD77F801F5CF83E50E94C179882319F084
:10B3C0000E942C7801C081E091E0892720CCCF93A6
:10B3D000DF9385E40E94867A811110C080E50E9487
:10B3E000C179882391F00E943B7860938D09709316
:10B3F0008E0980938F099093900907C00E941B7853
:10B40000882361F3E4E9FFE36DC089E40E94C17918
:10B41000882381F00E943B782CEA35EC47E25EE31A
:10B420000E9484F36093890970938A0980938B0941
:10B4300090938C0984E40E94C179882381F00E9452
:10B440003B782CEA35EC47E25EE30E942EF86093ED
:10B450008509709386098093870990938809EBEC9E
:10B46000FFE38491EF012196882321F00E94DD778C
:10B47000FE01F7CF40918D0950918E0960918F099F
:10B48000709190098EEC94E10E9466D22CEA35EC22
:10B4900047E25EE36091890970918A0980918B0986
:10B4A00090918C090E942EF8AB01BC018AEC94E1CA
:10B4B0000E944AD22CEA35EC47E25EE360918509AE
:10B4C0007091860980918709909188090E9484F380
:10B4D000AB01BC0186EC94E10E944AD210C00E94EC
:10B4E000DD77FE018491EF0121968111F8CFC9EF3C
:10B4F000D2E08991882319F00E94DD77FACF8AE0A3
:10B50000DF91CF910C94DD77CF93DF9380E50E949C
:10B51000C179882351F00E943B7860939909709318
:10B520009A0980939B0990939C0989E40E94C179B0
:10B53000882381F00E943B782CEA35EC47E25EE3F9
:10B540000E9484F3609395097093960980939709FC
:10B550009093980984E40E94C179882381F00E9425
:10B560003B782CEA35EC47E25EE30E942EF86093CC
:10B570009109709392098093930990939409EBEC4D
:10B58000FFE38491EF012196882321F00E94DD776B
:10B59000FE01F7CF4091990950919A0960919B095A
:10B5A00070919C0982EC94E10E9466D22CEA35EC01
:10B5B00047E25EE360919509709196098091970941
:10B5C000909198090E942EF8AB01BC018EEB94E19A
:10B5D0000E944AD22CEA35EC47E25EE36091910981
:10B5E0007091920980919309909194090E9484F33B
:10B5F000AB01BC018AEB94E10E944AD28AE0DF9160
:10B60000CF910C94DD77FB014081FC0120813181D9
:10B61000342768E0A901440F551F37FD07C09A0180
:10B620006150C1F7FC013183208308959A01F1E252
:10B630002F27F0E13F27F4CFEF92FF920F931F9354
:10B64000CF93DF93EC0189018C81833039F0E9E0FD
:10B65000440F551F661F771FEA95D1F79A01AB017A
:10B6600061E1CE010E94AD7C882331F084E08983C2
:10B67000CE010E94857C41C00E94897C7B010E9492
:10B68000D6778B838F3F49F40E94897C6E197F099E
:10B690006D327140A0F381E103C08E3F49F08FE02D
:10B6A0008983CE010E94857C8FEF0E94D17725C0CF
:10B6B0008FEF8EBDF80180E090E02FEF0DB407FE14
:10B6C000FDCF3EB531932EBD01968F3F31E09307FC
:10B6D000A9F70DB407FEFDCF8EB5F801E150FE4F7E
:10B6E00080830E94D6770E94D677CE010E94857C07
:10B6F0008FEF0E94D17781E001C080E0DF91CF9190
:10B700001F910F91FF90EF9008950F931F93CF9388
:10B71000DF93EC0189018C81833039F0F9E0440F2B
:10B72000551F661F771FFA95D1F79A01AB0168E1A3
:10B73000CE010E94AD7C882311F086E034C08EEFEC
:10B740008EBD80E090E00DB407FEFDCFF801E80F5C
:10B75000F91F20812EBD0DB407FEFDCF21812EBD26
:10B760000296811522E0920771F70DB407FEFDCF16
:10B770008FEF0E94D1778FEF0E94D1770E94D6770A
:10B780008B838F71853031F083E18983CE010E94F4
:10B79000857C0AC068E572E0CE010E94957C182F76
:10B7A000811107C087E18983CE010E94857C10E06A
:10B7B00012C020E030E0A9016DE0CE010E94AD7C16
:10B7C000811104C00E94D677882311F086E1EBCF67
:10B7D000CE010E94857C812FDF91CF911F910F9127
:10B7E0000895CF938091B3068823A9F14091B406C0
:10B7F0005091B5066091B6067091B7062DE334E01E
:10B800008091B1069091B20680DFC82F882321F184
:10B810004091B8065091B9066091BA067091BB0686
:10B82000411551056105710589F02DE334E08091E2
:10B83000B1069091B20669DF882359F01092B806DC
:10B840001092B9061092BA061092BB061092B30677
:10B850008C2FC82F01C0C1E08C2FCF910895CF92BB
:10B86000DF92EF92FF92CF936B017C01C42F809106
:10B87000B4069091B506A091B606B091B7068C15A6
:10B880009D05AE05BF05C1F0ACDF811102C080E0AF
:10B8900017C02DE334E0B701A6018091B106909165
:10B8A000B206CADE882399F3C092B406D092B506D8
:10B8B000E092B606F092B70681E0C1118093B3061C
:10B8C000CF91FF90EF90DF90CF9008958F929F924D
:10B8D000AF92BF92CF92DF92EF92FF920F931F939E
:10B8E000CF93DF93EC016A017B01890189859A85F9
:10B8F000AB85BC850196A11DB11D84179507A607D0
:10B90000B70710F480E054C08F89803129F499275B
:10B91000872F762F652F0BC08032A1F7CB01BA019C
:10B9200027E096958795779567952A95D1F78B8827
:10B930009C88AD88BE88680D791D8A1D9B1D8090EE
:10B94000B4069090B506A090B606B090B7066815FC
:10B9500079058A059B0581F48F89803191F4DD2476
:10B96000EE24FF24F601EE0FFF1FE35CFB4F808106
:10B970009181A0E0B0E016C040E071DF8111ECCF12
:10B98000C1CFE894C7F8DD24EE24FF24F601EE0FC2
:10B99000FF1FEE0FFF1FE35CFB4F80819181A281AF
:10B9A000B381BF70F80180839183A283B38381E068
:10B9B000DF91CF911F910F91FF90EF90DF90CF908B
:10B9C000BF90AF909F908F9008952F923F924F928B
:10B9D0005F926F927F928F929F92AF92BF92CF921F
:10B9E000DF92EF92FF920F931F93CF93DF93EC01BF
:10B9F0005B016A018B81811103C08FEF9FEFC6C08D
:10BA0000898180FFFACF49895A896B897C89888529
:10BA10009985AA85BB852601612C712C8A019B0121
:10BA2000081B190B2A0B3B0B0415150526053705BA
:10BA300018F46A01C81AD90A76013E0124E0620EA0
:10BA4000711CE114F10409F476C0488559856A85B2
:10BA50007B854A0181E098222B811A012B01E9E0C4
:10BA60005694479437942794EA95D1F7898D9A8D07
:10BA7000FC01223049F4628D738D848D958D620DA9
:10BA8000731D841D951D3CC0148111501221811419
:10BA90009104C1F4111116C0452B462B472B49F4D4
:10BAA0008D899E89AF89B88D8C839D83AE83BF833A
:10BAB00009C04C815D816E817F81930107DF8823FE
:10BAC00009F49BCFE98DFA8D6C817D818E819F81F8
:10BAD0006250710981099109058404C0660F771FBE
:10BAE000881F991F0A94D2F7268537854089518986
:10BAF000620F731F841F951F610F711D811D911DA2
:10BB000020E032E02819390987012E153F0508F495
:10BB100089010115F2E01F0761F52091B40630910B
:10BB2000B5064091B6065091B706621773078407B1
:10BB3000950719F41EC0C60129C09501AB01BC01CF
:10BB40008091B1069091B20677DD882309F455CF34
:10BB5000A00EB11E88859985AA85BB85800F911F8F
:10BB6000A11DB11D88879987AA87BB87E01AF10AB2
:10BB700068CF40E074DE882309F43FCFB401635CF2
:10BB80007B4FA801C5010E945CFAE2CFDF91CF9103
:10BB90001F910F91FF90EF90DF90CF90BF90AF90EB
:10BBA0009F908F907F906F905F904F903F902F90DD
:10BBB0000895AF92BF92CF92DF92EF92FF920F93D0
:10BBC0001F93CF93DF936C01EB017A01DC01139695
:10BBD0008C911397823070F018960D911D912D91D4
:10BBE0003C911B970F71112722273327012B022B22
:10BBF000032B11F08FEF58C04115510511F0F701DB
:10BC000010821DE040E250E0BE01C601DEDE9C0174
:10BC10008032910531F081E0232B09F480E0819599
:10BC200043C088818823C1F1853E61F38E3251F390
:10BC3000E114F10461F19B859F739F3041F54A8DBA
:10BC40005B8D452B21F58F719FEF980F9530F8F4A0
:10BC500090E00197189F9001199F300D1124FE016B
:10BC600080E090E05701A20EB31E8530B8F46181E8
:10BC7000A501480F591FDA016C93019632968D3059
:10BC8000910599F7888186FF02C0F50115868B859D
:10BC900083FDB8CF822F08C080E006C08B3010F43F
:10BCA0006481E6CF6681E4CFDF91CF911F910F9140
:10BCB000FF90EF90DF90CF90BF90AF9008954F929C
:10BCC0005F926F927F92AF92BF92CF92DF92EF928C
:10BCD000FF920F931F93CF93DF93EC016A017B01D7
:10BCE0002B81222349F089899A89AB89BC898417E1
:10BCF0009507A607B70710F480E06BC0223009F45F
:10BD000063C0C114D104E104F10449F41C821D8212
:10BD10001E821F82188619861A861B8659C088853E
:10BD20009985AA85BB85E98DFA8DE585F0E0399680
:10BD3000AC01BD0141505109610971090E2E04C0C9
:10BD400076956795579547950A94D2F7970186019E
:10BD5000015011092109310904C03695279517951D
:10BD60000795EA95D2F7041715072607370720F03D
:10BD7000892B8A2B8B2B49F48D899E89AF89B88DAD
:10BD80008C839D83AE83BF8304C0041B150B260BDD
:10BD9000370B280139015E0184E0A80EB11C411463
:10BDA00051046104710481F04C815D816E817F8159
:10BDB0009501898D9A8D8ADD91E0491A51086108B3
:10BDC00071088111ECCF05C0C886D986EA86FB864A
:10BDD00081E0DF91CF911F910F91FF90EF90DF9065
:10BDE000CF90BF90AF907F906F905F904F900895ED
:10BDF0004F925F926F927F92AF92BF92CF92DF92FB
:10BE0000EF92FF920F931F93CF93DF9300D01F9277
:10BE1000CDB7DEB78C0149835A836B837C8359018C
:10BE2000C12CD12C7601412CF2E05F2E612C712CBB
:10BE300049815A816B817C819E012F5F3F4FC801F0
:10BE400045DD882341F1D301C201F801058404C016
:10BE5000880F991FAA1FBB1F0A94D2F7C80ED91EBC
:10BE6000EA1EFB1E49815A816B817C818789803162
:10BE700039F481E0483F5F4F6105710538F4D8CF50
:10BE800081E0483F5F4F6F4F7F4090F2F501C082E5
:10BE9000D182E282F3820F900F900F900F90DF918A
:10BEA000CF911F910F91FF90EF90DF90CF90BF90B7
:10BEB000AF907F906F905F904F9008950F931F9376
:10BEC000CF93DF93EC018B018B81882311F080E00D
:10BED00041C0FB018789803131F18032C1F783E0B5
:10BEE0008B83F801428D538D648D758D4D8B5E8BE8
:10BEF0006F8B788F9E012F5E3F4FC80179DF8823BB
:10BF000031F31A8F098F81E089831C821D821E8282
:10BF10001F82188619861A861B861C861D861E8619
:10BF20001F86188A17C082E08B831D8A1E8A1F8A8B
:10BF3000188EFB01408D518D60E070E0A5E0440F4C
:10BF4000551F661F771FAA95D1F7498B5A8B6B8BAC
:10BF50007C8BD7CFDF91CF911F910F9108954F9296
:10BF60005F926F927F928F929F92AF92BF92CF9289
:10BF7000DF92EF92FF920F931F93CF93DF93EC0129
:10BF80004A015B0128013901423051056105710503
:10BF900008F462C049855A856B857C854F5F5F4F89
:10BFA0006F4F7F4F481559056A057B0508F454C04B
:10BFB0008F89803129F4FF24EB2CDA2CC92C0CC09A
:10BFC000803209F049C07501640107E0F694E794F6
:10BFD000D794C7940A95D1F74B895C896D897E897E
:10BFE000C40ED51EE61EF71E41E0C701B60137DCC0
:10BFF000882391F19F89903159F49924AA24BB2474
:10C00000F401EE0FFF1FE35CFB4F5182408210C032
:10C01000E89487F89924AA24BB24F401EE0FFF1FAB
:10C02000EE0FFF1FE35CFB4F4082518262827382FE
:10C030009A89923090F04D815E816F8178854C0DA8
:10C040005D1D6E1D7F1D4093B8065093B906609329
:10C05000BA067093BB0601C080E0DF91CF911F91BB
:10C060000F91FF90EF90DF90CF90BF90AF909F9097
:10C070008F907F906F905F904F900895AF92BF9296
:10C08000CF92DF92EF92FF920F931F93CF93DF93A4
:10C0900000D01F92CDB7DEB75C016A017B0182E060
:10C0A00090E0A0E0B0E0F50180839183A283B383A8
:10C0B0009E012F5F3F4FB701A601C50107DC81112B
:10C0C00002C080E023C000E010E09801B701A601A3
:10C0D000C50145DF8823A9F3C980DA80EB80FC80A5
:10C0E000F5018789803149F481E0F8EFCF16FFEF41
:10C0F000DF06E104F10450F4DBCF81E098EFC916CC
:10C100009FEFD906E9069FE0F90690F20F900F9095
:10C110000F900F90DF91CF911F910F91FF90EF90B3
:10C12000DF90CF90BF90AF900895CF93DF93CDB7BE
:10C13000DEB780918606811110C09E01275F3F4FB8
:10C140004F81588562E470E080E192E00E94E7F25E
:10C150000E94838883E080939E02DF91CF910895AF
:10C16000FF920F931F93CF93DF93C0917B0681E0E3
:10C17000C827D0917C06D827F0907D06F826C111FB
:10C1800002C0DD2319F0EBECFFE304C0F110FBCF9C
:10C1900080E077C084918F010F5F1F4F882321F0CB
:10C1A0000E94DD77F801F6CFE8E8F7E184918F018E
:10C1B0000F5F1F4F882321F00E94DD77F801F6CF33
:10C1C000CC2361F0E6E8F7E184918F010F5F1F4F08
:10C1D000882321F00E94DD77F801F6CFDD2361F09E
:10C1E000E4E8F7E184918F010F5F1F4F882321F06E
:10C1F0000E94DD77F801F6CFF11003C0EAE7F7E11E
:10C200000CC0E2E8F7E184918F010F5F1F4F882394
:10C21000A9F30E94DD77F801F6CF84918F010F5FBB
:10C220001F4F882321F00E94DD77F801F6CFFF2011
:10C2300019F04AE153E002C042E054E0DD2319F076
:10C240002CE133E002C022E034E0CC2319F08EE18F
:10C2500093E002C082E094E05F934F933F932F936B
:10C260009F938F9388E697E19F938F931F925DDF53
:10C270008DB79EB709960FB6F8949EBF0FBE8DBFBF
:10C2800081E0DF91CF911F910F91FF9008958091F0
:10C2900002128150823010F080E008951092021254
:10C2A0000E94897C60930B1270930C1280930D1284
:10C2B00090930E1281E008950F931F9380910212C4
:10C2C000813019F40E94897C08C060910B12709132
:10C2D0000C1280910D1290910E1200910712109184
:10C2E00008122091091230910A12601B710B820B07
:10C2F000930B28EE33E040E050E00E94F4F680918A
:10C30000031290910412A0910512B0910612280F09
:10C31000391F4A1F5B1FCA01B9011F910F91089570
:10C3200080910212813099F1823051F4C5DF60931F
:10C33000031270930412809305129093061218C092
:10C3400010920712109208121092091210920A12FB
:10C3500010920B1210920C1210920D1210920E12DB
:10C3600010920312109204121092051210920612EB
:10C3700081E0809302120E94897C6093071270937F
:10C3800008128093091290930A1281E0089580E0C8
:10C390000895CF92DF92EF92FF92C090CC07D09099
:10C3A000CD07E090CE07F090CF0720918007309125
:10C3B00081074091820750918307C701B6010E940F
:10C3C00084F30E9483F96093DE117093DF118093F0
:10C3D000E0119093E111C701B6010E9496F82FB7C2
:10C3E000F8946093510F7093520F8093530F909372
:10C3F000540F2FBF1092CE111092CF111092D01166
:10C400001092D111FF90EF90DF90CF90089580911E
:10C410000212813079F482E0809302120E94897CBA
:10C4200060930B1270930C1280930D1290930E1266
:10C4300081E0089580E00895E82FF0E0EC55FF4D8D
:10C44000849190E0FC013797EC30F105F8F4EE5858
:10C45000FF4F0C943DFA8091B100887F84608093F7
:10C46000B100089580919100887F8460809391004D
:10C4700008958091A100887F84608093A100089531
:10C4800080912101887F84608093210108958F929B
:10C490009F92AF92BF92CF92DF92EF92FF920F9353
:10C4A0001F93CF93DF931F921F92CDB7DEB77C010E
:10C4B00049018091C609811147C08B015B01A40E1F
:10C4C000B51E0A151B0509F43FC0F701C080D180D5
:10C4D000F80161918F016983C6016A830E94D5F5D5
:10C4E0006A81681729F1C6010E94DDF5C6010E9424
:10C4F000D5F599818917E1F0EBECFFE384918F0189
:10C500000F5F1F4F882321F00E94DD77F801F6CFDF
:10C51000EEE4F7E184918F010F5F1F4F882321F034
:10C520000E94DD77F801F6CF81E08093C6090CC048
:10C53000BE016F5F7F4FC40166D8F7018081918192
:10C54000019691838083BDCF0F900F90DF91CF91A3
:10C550001F910F91FF90EF90DF90CF90BF90AF9021
:10C560009F908F900895AF92BF92CF92DF92EF92FB
:10C57000FF920F931F93CF93DF931F92CDB7DEB738
:10C580008C016B017A0159018091C60981111BC090
:10C59000F801808191810E94D5F58983F60181930C
:10C5A0006F01BE016F5F7F4FC5012DD8F80140813B
:10C5B00051814F5F5F4F51834083F1E0EF1AF108E3
:10C5C000E114F10429F70F90DF91CF911F910F91A2
:10C5D000FF90EF90DF90CF90BF90AF900895CF92F3
:10C5E000DF92EF92FF920F931F93CF93DF937C0123
:10C5F0008B016A01E9010E943D8983E080939E02DC
:10C60000F0929007E0928F0710938E0700938D07AA
:10C610001092890710928A0710928B0710928C074C
:10C62000A601662757FD6095762F409385075093A6
:10C6300086076093870770938807F801808191814E
:10C64000AA2797FDA095BA2F809306119093071102
:10C65000A0930811B093091184E990E890936802BF
:10C6600080936702D093BE06C093BD061092BC06AD
:10C67000DF91CF911F910F91FF90EF90DF90CF90BE
:10C680000895CF92DF92EF92FF920F931F93CF9373
:10C69000DF9300D01F92CDB7DEB77C018B01CA01BA
:10C6A000B90129837A838B839C830E943D8923E08F
:10C6B00020939E02F0929007E0928F0710938E07CE
:10C6C00000938D072AE037ED43E25CE369817A81CC
:10C6D0008B819C810E9484F30E9496F86093890765
:10C6E00070938A0780938B0790938C070E9425F3A1
:10C6F0006B017C019B01AC0160E070E887E794E48A
:10C700000E9451F70E9496F8609385077093860700
:10C7100080938707909388072AE037ED43E25CE334
:10C72000F80160817181828193810E9484F3A70165
:10C7300096010E9451F70E949BF860930611709336
:10C74000071180930811909309118BED9EE7909348
:10C750006802809367020F900F900F900F90DF9107
:10C76000CF911F910F91FF90EF90DF90CF900895A0
:10C770000F931F93CF93DF938C01EB010E943D89B0
:10C7800083E080939E021093900700938F07D093CD
:10C790008E07C0938D0784EF91E0A0E0B0E0809316
:10C7A000890790938A07A0938B07B0938C0788EE34
:10C7B0009FE3AFE0B0E08093850790938607A09356
:10C7C0008707B093880720E030E048EC52E46881A6
:10C7D00079818A819B810E9484F320E030E04AEFD6
:10C7E00053E40E9451F70E949BF8609306117093E6
:10C7F0000711809308119093091187EA9CE69093A2
:10C800006802809367028BEA9FED9093BE06809347
:10C81000BD061092BC06DF91CF911F910F91089534
:10C82000CF92DF92EF92FF920F931F93CF93DF93FC
:10C8300000D01F92CDB7DEB77C018B0129833A83EC
:10C840004B835C830E943D8983E080939E02F0923B
:10C850009007E0928F0710938E0700938D07298130
:10C860003A814B815C81CA01B9010E9423F32AE01D
:10C8700037ED43E25CE30E9484F30E9496F86093F4
:10C88000890770938A0780938B0790938C070E9487
:10C8900025F36B017C019B01AC0160E070E887E748
:10C8A00094E40E9451F70E9496F860938507709374
:10C8B00086078093870790938807F80160817181CC
:10C8C000828193810E9423F32AE037ED43E25CE307
:10C8D0000E9484F3A70196010E9451F70E949BF8E1
:10C8E00060930611709307118093081190930911BA
:10C8F0008AEE9BE6909368028093670284EA96E84A
:10C900009093BE068093BD061092BC060F900F90C8
:10C910000F900F90DF91CF911F910F91FF90EF90AB
:10C92000DF90CF9008950F931F93CF93DF931F92C3
:10C930001F92CDB7DEB7FC0184918F010F5F1F4FAF
:10C94000811102C08B0108C069837A830E94DD7760
:10C95000F80169817A81F0CFD8018D918D0188230A
:10C9600019F00E94DD77F8CF0F900F90DF91CF91F3
:10C970001F910F9108950F931F93CF93DF938C0115
:10C98000EBECFFE38491EF012196882321F00E94D4
:10C99000DD77FE01F7CFB80181E497E1C4DF82E2E1
:10C9A0000E94DD778AE00E94DD7781E0DF91CF9100
:10C9B0001F910F9108958F929F92AF92BF92CF9245
:10C9C000DF92EF92FF92CF93FC01C080D180E28092
:10C9D000F38020E030E0A901C701B6010E941FF3F7
:10C9E00087FF08C0C701B601905820E030E048EC4E
:10C9F00052E406C020E030E048EC52E4C701B60142
:10CA00000E9484F30E9496F86B017C01603AF6E87C
:10CA10007F07F1E08F07910584F020EA36E841E0D6
:10CA200050E00E9416F7CA01B9012AE030E040E068
:10CA300050E00E9416F7605D01C060E260939706C7
:10CA400080E1C81687E2D806E104F10494F0C7013A
:10CA5000B60120E137E240E050E00E9416F7CA013B
:10CA6000B9012AE030E040E050E00E9416F7605D36
:10CA700001C060E260939806E8EECE16E3E0DE06C1
:10CA8000E104F10494F0C701B60128EE33E040E080
:10CA900050E00E9416F7CA01B9012AE030E040E0F8
:10CAA00050E00E9416F7605D01C060E26093990655
:10CAB000C701B60124E630E040E050E00E9416F7DE
:10CAC0009AE0892E912CA12CB12CCA01B901A501A3
:10CAD00094010E9416F7605D60939A068EE280933F
:10CAE0009B06C701B601A50194010E9416F7C62F47
:10CAF000CA01B901A50194010E9416F7605D609317
:10CB00009C06C05DC0939D0687E996E0CF91FF909B
:10CB1000EF90DF90CF90BF90AF909F908F9008954F
:10CB20008F929F92AF92BF92CF92DF92EF92FF923D
:10CB3000CF9320E030E048EC52E4FC016081718149
:10CB4000828193810E9484F30E9496F86B017C019C
:10CB500097FF0AC0F094E094D094C094C11CD11CFB
:10CB6000E11CF11C8DE201C08BE280939706C701A6
:10CB7000B60120E137E240E050E00E9416F76AE09B
:10CB8000862E912CA12CB12CCA01B901A5019401CA
:10CB90000E9416F7605D60939806C701B60128EE03
:10CBA00033E040E050E00E9416F7CA01B901A50148
:10CBB00094010E9416F7605D60939906C701B60163
:10CBC00024E630E040E050E00E9416F7CA01B901C7
:10CBD000A50194010E9416F7605D60939A068EE2AB
:10CBE00080939B06C701B601A50194010E9416F728
:10CBF000C62FCA01B901A50194010E9416F7605D14
:10CC000060939C06C05DC0939D0687E996E0CF9136
:10CC1000FF90EF90DF90CF90BF90AF909F908F905C
:10CC200008958F929F92AF92BF92CF92DF92EF9230
:10CC3000FF92FC01C080D180E280F38020E030E0F0
:10CC4000A901C701B6010E941FF387FF04C0C701F5
:10CC5000B601905802C0C701B6010E9496F86B0158
:10CC60007C016031F7E27F078105910584F020E1C6
:10CC700037E240E050E00E9416F7CA01B9012AE00D
:10CC800030E040E050E00E9416F7605D01C060E2D5
:10CC90006093990688EEC81683E0D806E104F10493
:10CCA00094F0C701B60128EE33E040E050E00E9466
:10CCB00016F7CA01B9012AE030E040E050E00E94D6
:10CCC00016F7605D01C060E260939A06E4E6CE1656
:10CCD000D104E104F10494F0C701B60124E630E088
:10CCE00040E050E00E9416F7CA01B9012AE030E0A6
:10CCF00040E050E00E9416F7605D01C060E2609382
:10CD00009B06FAE0CF16D104E104F1049CF07AE02E
:10CD1000872E912CA12CB12CC701B601A50194013D
:10CD20000E9416F7CA01B901A50194010E9416F7E5
:10CD3000605D01C060E260939C06C701B6012AE015
:10CD400030E040E050E00E9416F7605D60939D0681
:10CD500089E996E0FF90EF90DF90CF90BF90AF9081
:10CD60009F908F900895AF92BF92CF92DF92EF92F3
:10CD7000FF920F931F93CF93DF93CDB7DEB7A097AA
:10CD80000FB6F894DEBF0FBECDBF611571058105EA
:10CD90009105B1F1B12CC42ED12CE12CF12CAA2497
:10CDA000A394AB0C01E010E00C0F1D1F0B0D111D27
:10CDB000B7FC1A95A70196010E94F4F6F80160836A
:10CDC000B901CA01611571058105910511F41B2D89
:10CDD00012C0BA2CE4CFE1E0F0E0EC0FFD1FE10F50
:10CDE000F11D17FDFA9580818A3040F490E3890F98
:10CDF0000E94DD7711501F3F71F715C097E3F7CF01
:10CE000080E3A0960FB6F894DEBF0FBECDBFDF91D2
:10CE1000CF911F910F91FF90EF90DF90CF90BF9037
:10CE2000AF900C94DD77A0960FB6F894DEBF0FBEDE
:10CE3000CDBFDF91CF911F910F91FF90EF90DF90C9
:10CE4000CF90BF90AF900895CF92DF92EF92FF9274
:10CE50006B017C0197FF0BC08DE20E94DD77F0949F
:10CE6000E094D094C094C11CD11CE11CF11C4AE098
:10CE7000C701B601FF90EF90DF90CF9074CFCF93B2
:10CE8000DF93E8E2F1E28491EF012196882321F01B
:10CE90000E94DD77FE01F7CFE4E2F1E28491EF0139
:10CEA0002196882321F00E94DD77FE01F7CF62B33F
:10CEB0006695617070E080E090E0C6DF62B36170FB
:10CEC00070E080E090E0C0DF8AE00E94DD77E0E281
:10CED000F1E28491EF012196882321F00E94DD7711
:10CEE000FE01F7CF60910601772767FD7095872FC8
:10CEF000972F662797FD6395772788279927A4DFC3
:10CF000062B362FB662760F970E080E090E09CDF2E
:10CF10008AE00E94DD77ECE1F1E28491EF01219655
:10CF2000882321F00E94DD77FE01F7CF6091060192
:10CF300066FB662760F970E080E090E085DF609135
:10CF4000060165FB662760F970E080E090E07CDF19
:10CF50008AE00E94DD77E7E1F1E28491EF0121961A
:10CF6000882321F00E94DD77FE01F7CF6091060152
:10CF700063FB662760F970E080E090E065DF609118
:10CF800006016295617070E080E090E05DDF8AE00C
:10CF90000E94DD77E2E1F1E28491EF01219688239E
:10CFA00021F00E94DD77FE01F7CF609106016695C2
:10CFB000617070E080E090E047DF6091060162FB05
:10CFC000662760F970E080E090E03EDF8AE0DF9164
:10CFD000CF910C94DD770F931F93CF93DF938B0149
:10CFE000FC018491EF012196882321F00E94DD77D6
:10CFF000FE01F7CFB801882777FD8095982FDF9144
:10D00000CF911F910F9120CFCF93DF9383E50E94A3
:10D01000C179C82F882371F00E943B780E9496F84E
:10D0200070930B0260930A0221E0672B09F020E065
:10D030002093280480E50E94C179882369F08091BB
:10D040000A0290910B02892B19F00E942C7801C0E2
:10D0500081E0809328042BC0C11129C0EBECFFE3D1
:10D060008491EF012196882321F00E94DD77FE0153
:10D07000F7CF80912804882319F06CEE72E002C08B
:10D0800060E273E08FEF90E24EDC60910A027091F3
:10D090000B028EEE90E29FDFEAEEF0E28491EF0168
:10D0A0002196882321F00E94DD77FE01F7CFDF91E2
:10D0B000CF910895BC0180E090E04AE054DE8DE01D
:10D0C0000E94DD778AE00C94DD7790E0FC01E15965
:10D0D000F24C2491FC01EB54F24C8491882399F09A
:10D0E00090E0880F991FFC01EB5AF24CA591B49186
:10D0F00086579F4DFC01859194919FB7F8948C9130
:10D10000822B8C939FBF08951F93CF93DF93182F8B
:10D11000EB01DBDF209711F460E004C0CF3FD105C5
:10D1200039F461E0812FDF91CF911F910C94507CF5
:10D13000E12FF0E0EC55FF4D449150E0FA013197BA
:10D14000E231F10508F09BC0E258FF4F0C943DFA24
:10D1500084B5806884BDC7BD97C084B5806284BD36
:10D16000C8BD92C080918000806880938000D09379
:10D170008900C093880088C080918000806280937D
:10D180008000D0938B00C0938A007EC08091800085
:10D19000886080938000D0938D00C0938C0074C011
:10D1A0008091B00080688093B000C093B3006CC0E1
:10D1B0008091B00080628093B000C093B40064C0DE
:10D1C00080919000806880939000D0939900C093E4
:10D1D00098005AC080919000806280939000D09314
:10D1E0009B00C0939A0050C080919000886080930B
:10D1F0009000D0939D00C0939C0046C08091A000F9
:10D2000080688093A0008091A0008F7B8093A00015
:10D21000D093A900C093A80037C08091A00080627D
:10D220008093A000D093AB00C093AA002DC0809142
:10D23000A00088608093A000D093AD00C093AC00A4
:10D2400023C080912001806880932001D093290120
:10D25000C093280119C08091200180628093200131
:10D26000D0932B01C0932A010FC0809120018860C8
:10D2700080932001D0932D01C0932C0105C0C038AC
:10D28000D1050CF04ECF48CFDF91CF911F9108957B
:10D290001F93CF93DF93E0919211F0919311309708
:10D2A00019F084E891E11995C0918611D091871108
:10D2B000E091B511F091B61182E01995E091B511A8
:10D2C000F091B61181E0199520E030E045E1BE0112
:10D2D00084E891E10E94897B182F882341F027EB95
:10D2E00031E147E1BE0184E891E10E94897BE09150
:10D2F000B511F091B61180E01995812FDF91CF9192
:10D300001F910895209188113091891128173907AC
:10D3100009F444C09093891180938811009709F40F
:10D3200037C020919B11FC01211107C03596E49173
:10D33000E0939C11FC013C960FC0213039F43F96DC
:10D34000E491E0939C11FC01709606C03D96E49137
:10D35000E0939C11FC013E96849180939D118091F5
:10D360009C11992787FD909520919D11821B910911
:10D3700027FD939520919E11203441F0829FC0019A
:10D38000112446E0969587954A95E1F780939F1181
:10D390008EED95E790939A118093991108958EE8F8
:10D3A00097E1B0DF81E080939F060895CF93C82F67
:10D3B000823051F020F4813079F4CF91F0CF833076
:10D3C00031F0843021F008C08CE897E002C088E199
:10D3D00098E098DFC0939F06CF910895E091801167
:10D3E000F09181110190F081E02D682F80E891E1AA
:10D3F0001994CF93C82F8FEF8C0F893048F48CE8A5
:10D4000097E080DF8C2FEADF80919F06CFDF02C09C
:10D410008C2FE4DF81E0CF910895CF93C82F8FEF59
:10D420008C0F893048F48CE897E06CDF8C2FD6DFC6
:10D4300080919F06CF91BACF8C2FCF91CFCFCF9332
:10D44000DF93EC01FE018491882319F0E6DF219639
:10D45000F9CFDF91CF910895CF93DF93EC018991BC
:10D46000882311F0DADFFBCFDF91CF9108959CE0A4
:10D47000899F802D112441E0480F40935807845F15
:10D48000809359076091B81170E0282F30E02E5F2B
:10D490003F4F261737079CF150E02091BA1130E03A
:10D4A0004217530764F59EE39093BB118093BC1120
:10D4B00085E4B3DF809187068F5CAFDF80E2ADDF6C
:10D4C0006091460670914706809148069091490602
:10D4D0000E9496F8CB010E945787BEDF8FE29DDF46
:10D4E0000E94CF88811104C080918406811107C0F9
:10D4F0008091840F9091850F0E945787ADCF08953A
:10D50000CF93DF93C0E1D2E08991882329F066DFD1
:10D5100082E0C632D807C1F7DF91CF9108958F928C
:10D520009F92AF92BF92CF92DF92EF92FF921F93A2
:10D53000CF93DF93C82F2CED33E13093B2062093C5
:10D54000B1061092F81342E050E060E070E04093C2
:10D55000E1135093E2136093E3137093E41310927A
:10D56000B3061092B8061092B9061092BA0610923D
:10D57000BB064FEF5FEFBA014093B4065093B50678
:10D580006093B6067093B706882351F1853008F092
:10D59000F8C040E060E070E0CB010E942F5C88237F
:10D5A00009F4EFC020E1C29FF0011124E551FA4FC8
:10D5B00080818F7709F0E5C044855585668577853C
:10D5C000443651056105710508F4DBC0C084D1847F
:10D5D000E284F384C114D104E104F10421F4D1C044
:10D5E000C12CD12C760140E0C701B6010E942F5C0E
:10D5F000182F882309F4C5C08091480490914904EC
:10D600008115924009F0BDC0A0914D04AA2309F4F0
:10D61000B8C080914B0490914C04009709F4B1C0BC
:10D6200040914A04442309F4ACC0A093F3134093FF
:10D63000E513E0E050E061E070E0CE2F9B010E2E9C
:10D6400002C0220F331F0A94E2F74217530749F032
:10D6500021E02E0FE83018F02093EE1392C0E22F55
:10D66000ECCFE093EE132091530430915404211534
:10D67000310519F040E050E008C02091610430917C
:10D68000620440916304509164042093E613309344
:10D69000E7134093E8135093E91346015701880EAE
:10D6A000991EA11CB11C8092F4139092F513A092C4
:10D6B000F613B092F713E0914E04F0914F04F093FB
:10D6C000FA13E093F913B0E00E9432F7680D791D68
:10D6D0008A1D9B1D6093FB137093FC138093FD13B5
:10D6E0009093FE1355E0EE0FFF1F5A95E1F7E150BE
:10D6F000FE4FEF2FFF27E695DC01CB018E0F9F1F1A
:10D70000A11DB11D8093EF139093F013A093F1131B
:10D71000B093F213809050049090510481149104BE
:10D7200019F0A12CB12C08C080905D0490905E048B
:10D73000A0905F04B0906004A7019601281B390BEC
:10D740004A0B5B0BDA01C901880D991DAA1DBB1D8F
:10D750000C2E04C0B695A795979587950A94D2F795
:10D760008093EA139093EB13A093EC13B093ED1313
:10D77000853F4FE09407A105B10528F48CE0809324
:10D78000F81310E01AC0853F9F4FA105B10510F4B2
:10D7900080E111C08091690490916A04A0916B04AA
:10D7A000B0916C048093FB139093FC13A093FD1332
:10D7B000B093FE1380E28093F813812FDF91CF9115
:10D7C0001F91FF90EF90DF90CF90BF90AF909F9010
:10D7D0008F900895CF92DF92EF92FF921F93CF9395
:10D7E000DF9300D01F92CDB7DEB7809106119091E4
:10D7F0000711A0910811B0910911B7FF08C010924C
:10D8000006111092071110920811109209118091BF
:10D81000850790918607A0918707B091880740916E
:10D820000611509107116091081170910911841728
:10D830009507A607B70744F4809306119093071144
:10D84000A0930811B093091180919E02882351F191
:10D850006091061170910711809108119091091142
:10D86000C0908907D0908A07E0908B07F0908C07D2
:10D870006C0D7D1D8E1D9F1D0E9423F320E030E066
:10D8800048EC52E40E9484F369837A838B839C83FF
:10D89000CE010196C6D9BC0180918F079091900767
:10D8A0000E94507E809102111091BC06811106C029
:10D8B0001123C1F180919E028823A1F1609106118C
:10D8C000709107118091081190910911C0908907FA
:10D8D000D0908A07E0908B07F0908C076C0D7D1D2F
:10D8E0008E1D9F1D0E9423F320E030E048EC52E49F
:10D8F0000E9484F30E949BF8E0918D07F0918E07BF
:10D90000309721F06083718382839383112329F000
:10D91000E091BD06F091BE0619958091021181112A
:10D920000E94318A80910211882329F0E091BD067E
:10D93000F091BE0619950F900F900F900F90DF9108
:10D94000CF911F91FF90EF90DF90CF900895CF92ED
:10D95000DF92EF92FF921F93CF93DF9300D01F923D
:10D96000CDB7DEB78091061190910711A0910811F3
:10D97000B0910911B7FF08C010920611109207115B
:10D9800010920811109209118091850790918607D5
:10D99000A0918707B0918807409106115091071117
:10D9A000609108117091091184179507A607B707B0
:10D9B00044F48093061190930711A0930811B0933B
:10D9C000091180919E02882359F16091061170918E
:10D9D00007118091081190910911C0908907D0908A
:10D9E0008A07E0908B07F0908C076C0D7D1D8E1DD3
:10D9F0009F1D0E9425F32AE037ED43E25CE30E947D
:10DA000084F369837A838B839C83CE0101960E9481
:10DA1000DB64BC0180918F07909190070E94507E3B
:10DA2000809102111091BC06811106C01123B1F141
:10DA300080919E02882391F16091061170910711E7
:10DA40008091081190910911C0908907D0908A07A0
:10DA5000E0908B07F0908C076C0D7D1D8E1D9F1D37
:10DA60000E9425F32AE037ED43E25CE30E9484F351
:10DA7000E0918D07F0918E07309721F060837183DC
:10DA800082839383112329F0E091BD06F091BE06B5
:10DA900019958091021181110E94318A80910211A1
:10DAA000882329F0E091BD06F091BE0619950F90EC
:10DAB0000F900F900F90DF91CF911F91FF90EF90FB
:10DAC000DF90CF900895CF92DF92EF92FF921F9355
:10DAD000CF93DF9300D01F92CDB7DEB780910611B0
:10DAE00090910711A0910811B0910911B7FF08C0DA
:10DAF000109206111092071110920811109209113C
:10DB00008091850790918607A0918707B09188073B
:10DB100040910611509107116091081170910911FF
:10DB200084179507A607B70744F4809306119093CE
:10DB30000711A0930811B093091180919E028823C8
:10DB400059F160910611709107118091081190911F
:10DB50000911C0908907D0908A07E0908B07F09058
:10DB60008C076C0D7D1D8E1D9F1D0E9425F32AE0E4
:10DB700037ED43E25CE30E9484F369837A838B830D
:10DB80009C83CE0101960E949065BC0180918F0715
:10DB9000909190070E94507E809102111091BC06D6
:10DBA000811106C01123B1F180919E02882391F169
:10DBB00060910611709107118091081190910911DF
:10DBC000C0908907D0908A07E0908B07F0908C076F
:10DBD0006C0D7D1D8E1D9F1D0E9425F32AE037EDE3
:10DBE00043E25CE30E9484F3E0918D07F0918E079D
:10DBF000309721F06083718382839383112329F00E
:10DC0000E091BD06F091BE06199580910211811137
:10DC10000E94318A0F900F900F900F90DF91CF915B
:10DC20001F91FF90EF90DF90CF900895CF92DF92F9
:10DC3000FF920F931F93CF93DF931F921F92CDB745
:10DC4000DEB76901DB0112960D911C9113974233E7
:10DC500009F471C0B8F4453109F47AC0473109F4C8
:10DC60008BC0443109F0A1C0D80115962C911597AD
:10DC70001696ED91FC911797CF01820F911D820F9F
:10DC8000911D5EC0463409F487C0473409F488C04A
:10DC90004B3309F08AC0F90181819381913029F0D9
:10DCA000933031F4282F885004C028E0280F01C099
:10DCB000282F31E0D80113964C91481708F430E032
:10DCC00051E0F8014281241708F450E041E02817A0
:10DCD00008F040E0832F842B85233423832B09F421
:10DCE00064C0D6011296FC90913039F070F09230F9
:10DCF00039F0933041F020E001C021E030E007C06E
:10DD000020E03FEF04C02FEFF9CF20E031E0F7FE35
:10DD100008C0B601C8012A8339830E94267B398155
:10DD20002A81F6018081830F80838181820F818324
:10DD3000FF0C69F73AC0B901C8010E94267B35C0C3
:10DD40001192E817F907E1F7C8010E94517B2DC035
:10DD5000C8010E943B7B882351F1F8012581068090
:10DD6000F781E02DCF01820F911D820F911D11923D
:10DD7000E817F907E1F719C0D9011C92F80182816F
:10DD800011968C9311978581815012968C931297DE
:10DD9000838113968C9309C0D80115968C9103C08A
:10DDA000D80111968C91F601808381E001C080E05A
:10DDB0000F900F90DF91CF911F910F91FF90DF9007
:10DDC000CF900895EC01E4E9FFE384918F010F5FA8
:10DDD0001F4F882321F00E94DD77F801F6CFE2E59E
:10DDE000F1E284918F010F5F1F4F882321F00E9481
:10DDF000DD77F801F6CF0E944D520E946E780E94A6
:10DE00001B8361E0CE010E94B2880E942B8A0E948F
:10DE10009A5184E0CBDA809185118695869510928F
:10DE2000BB118093BC116CDB809185118695869522
:10DE3000880F1092BB118093BC1183E491E2FFDA4A
:10DE40008091851186958695982F990F980F10923D
:10DE5000BB119093BC1186E391E2F1DA19DA8111DA
:10DE6000D8CF2FEF8BE49DE1215080409040E1F727
:10DE700000C00000F8942FEF84E39CE02150804024
:10DE80009040E1F700C000000E944D52A895FECFDF
:10DE90006F927F928F929F92AF92BF92DF92EF929A
:10DEA000FF920F931F93CF93DF93CDB7DEB7AD975C
:10DEB0000FB6F894DEBF0FBECDBF7C01D62E809189
:10DEC0001212882309F4E9C180910614882309F409
:10DED0009CC0442309F4B9C180911E14882321F108
:10DEE000E4E9FFE384918F010F5F1F4F882321F046
:10DEF0000E94DD77F801F6CFE5EDF2E284918F0123
:10DF00000F5F1F4F882321F00E94DD77F801F6CFC5
:10DF100061E070E080E090E00E9424678AE00E9467
:10DF2000DD778CEC92E24EDF8FE280932314B12CEC
:10DF300021E004E214E19FE1A92E8091DB13B816E1
:10DF4000B8F4AB9CC0011124B80187559D4E2DA794
:10DF50000E945151C8012DA58C010196F801308114
:10DF6000332321F02D3810F42F5FF6CFB394E5CF93
:10DF700027FD06C0B80183E094E10E94515102C020
:10DF8000F8011082EBECFFE384918F010F5F1F4FCC
:10DF9000882321F00E94DD77F801F6CFB70183EBEB
:10DFA00092E20E94936460911E14FDE86F9FB0019D
:10DFB00011246D5D7B4E88EA92E20E949364409149
:10DFC000B4145091B5146091B6147091B71482EAEC
:10DFD00092E20E9477D38AE0F0D780911E1494E0F9
:10DFE000899FF0011124E15EFB4E4091B4145091E1
:10DFF000B5146091B6147091B71440835183628355
:10E0000073838F5F80931E140CC010921E1482E0E5
:10E01000B82E1DC1B70185E992E20E9493648AE09F
:10E02000CCD70E94304F1D8218861C821B828EE046
:10E0300093E09A83898385E692E190938512809399
:10E040008412F70180818F3209F069C087010F5F68
:10E050001F4FCE0101963C010115110509F465C061
:10E060006FE270E0C8010E9483FA5C01009709F436
:10E070005DC00817190708F059C04C01801A910AB1
:10E08000A401B801CE0180960E94A3FAE0E2F0E07C
:10E09000EC0FFD1FE80DF91D10828E01005E1F4F71
:10E0A000F80181918F01882311F087D7F9CF8AE099
:10E0B00084D760918412709185126115710519F0F1
:10E0C0006C5F7F4F02C060E070E021E0AE01405E17
:10E0D0005F4FCE0105960E944183811118C0E1E88F
:10E0E000F2E284918F010F5F1F4F811104C08E01F6
:10E0F000005E1F4F03C061D7F801F3CFF801819193
:10E100008F01882311F059D7F9CF8EE289C0709220
:10E1100085126092841285010F5F1F4F9DCF86E8A4
:10E1200092E190938512809384128701609184120A
:10E1300070918512DD2009F45BC06115710519F03D
:10E140006C5F7F4F02C060E070E021E0A80183E0D7
:10E1500094E10E944183882309F446C080911414FD
:10E1600090911514A0911614B09117148093B014C7
:10E170009093B114A093B214B093B314B80183E791
:10E1800092E20E9493644091B0145091B114609156
:10E19000B2147091B3148BE692E20E9477D38AE0B6
:10E1A0000CD71092B4141092B5141092B6141092A9
:10E1B000B714ECE5F2E284917F019FEFE91AF90AC6
:10E1C000882319F0FAD6F701F6CFB80180E090E085
:10E1D0000E94F88580912112811102C0C80102C0FD
:10E1E00081E292E160E02AC0B80188E492E213C0C3
:10E1F0006115710519F06C5F7F4F02C060E070E03F
:10E2000026E5A80183E094E10E94418381110AC0C0
:10E21000B80184E392E20E9493648EE2CED68AE053
:10E22000CCD60EC081E080930F12B70182E292E259
:10E230000E9493648AE0C1D660E0C8010E94A2886F
:10E24000CE0101960E94875028C0BB24B394EBEC0A
:10E25000FFE384918F010F5F1F4F882319F0ADD624
:10E26000F801F7CFEDE9F2E284918F010F5F1F4FC4
:10E27000882319F0A2D6F801F7CFE1E0BE1203C05F
:10E280000AE213E002C004E213E0F80181918F0179
:10E29000882309F4BFCE91D6F8CFAD960FB6F89487
:10E2A000DEBF0FBECDBFDF91CF911F910F91FF90C9
:10E2B000EF90DF90BF90AF909F908F907F906F9086
:10E2C000089560E08091860F9091870F0E94F28EF2
:10E2D00060934606709347068093480690934906DC
:10E2E0008091820F9091830F0E94B08B60934A06B9
:10E2F00070934B0680934C0690934D06A8958FB76C
:10E30000F8941092880F8FBF0895CF92DF92FF92FA
:10E310000F931F93CF93DF931F921F92CDB7DEB75A
:10E32000F82E6A0180916302882309F43CC0E4E975
:10E33000FFE384918F010F5F1F4F882339F06983BA
:10E340007A833BD6F80169817A81F3CFFB0184910E
:10E350008F010F5F1F4F882319F02FD6F801F7CFD9
:10E36000E7E7F1E284918F010F5F1F4F882319F0D7
:10E3700024D6F801F7CFF7FC0BC06F2D772767FD88
:10E380007095872F972F0E9424678AE016D60BC0BE
:10E39000E2E7F1E284918F010F5F1F4F882319F0AC
:10E3A0000CD6F801F7CF8091BF06811107C01092FB
:10E3B000630281E08093BF06C60104DD0F900F90D9
:10E3C000DF91CF911F910F91FF90DF90CF900C9430
:10E3D0004D522F923F924F925F926F927F928F9207
:10E3E0009F92AF92BF92CF92DF92EF92FF920F93E4
:10E3F0001F93CF93DF9300D01F92CDB7DEB74C01B0
:10E400001B0129833A834B835C8327013801D7FEA4
:10E4100012C080919606882309F4A7C0F4011082E7
:10E420001092C4061092C5061092C6061092C70636
:10E4300001E010E015C0F601EC57F94F8081882308
:10E4400009F4BEC0F4011082F601EE0FFF1FEE0FBB
:10E45000FF1FE054F94F108211821282138286014D
:10E46000F40180818230E1F0833009F455C08130BD
:10E4700009F0A8C0F801EE0FFF1FEE0FFF1FE054D8
:10E48000F94F208131814281538169817A818B8169
:10E490009C810E941FF387FD95C082E0F401808378
:10E4A000000F111F000F111F0054194FB5018827CD
:10E4B00077FD8095982F0E9425F39B01AC01F80110
:10E4C00060817181828193810E9451F79B01AC012F
:10E4D00069817A818B819C810E9478F987FD0CC0CB
:10E4E0000E94897C6856754C8F4F9F4FF101608365
:10E4F00071838283938366C00E94897CF1010081CD
:10E50000118122813381601B710B820B930B97FD6C
:10E5100059C083E0F4018083FFEFCF16DF0631F0AE
:10E52000C114D10431F44CEC51E205C045E951E28B
:10E5300002C049EB51E269EA71E28C2D0F900F9015
:10E540000F900F90DF91CF911F910F91FF90EF905F
:10E55000DF90CF90BF90AF909F908F907F906F9003
:10E560005F904F903F902F90D0CE01E010E0780167
:10E57000EE0CFF1CEE0CFF1CC7018054994F7C0170
:10E58000A3019201FC0160817181828193810E94CB
:10E590001FF3882309F464CFF7014082518262821D
:10E5A0007382FF24F39420E030E0A901C301B2019B
:10E5B0000E9478F918160CF0F12CF401F08250CF7B
:10E5C0008601D5CF0F900F900F900F90DF91CF91D4
:10E5D0001F910F91FF90EF90DF90CF90BF90AF9081
:10E5E0009F908F907F906F905F904F903F902F9073
:10E5F00008958F3F29F0811106C04AE85AE405C00A
:10E6000047E55AE402C04AE75AE468E67AE47DCE78
:10E610008F3F29F0811106C04DEC5AE405C04AE94C
:10E620005AE402C04DEB5AE46BEA7AE46ECE4F92A4
:10E630005F926F927F92AF92BF92CF92DF92EF92F2
:10E64000FF920F931F93CF93DF9300D01F92CDB70C
:10E65000DEB78091880F811113C00F900F900F903B
:10E660000F90DF91CF911F910F91FF90EF90DF906E
:10E67000CF90BF90AF907F906F905F904F90089534
:10E6800020DE0E94897C69837A838B839C838091BE
:10E69000640290916502181619060CF026C10197C4
:10E6A000909365028093640240904606509047061E
:10E6B000609048067090490680918406811119C0C7
:10E6C0008091800690918106A0918206B091830688
:10E6D0000097A105B10569F029813A814B815C81E0
:10E6E000281B390B4A0B5B0B57FD03C081E080935D
:10E6F00084066091840F7091850F882777FD80953F
:10E70000982F0E9425F31EE1A12EB12CC12CD12CF3
:10E710007B018C01A30192016AED76E089ED96E020
:10E7200058DE40904606509047066090480670902C
:10E7300049066091AD077091AE07882777FD8095F7
:10E74000982F0E9425F39B01AC01C301B2010E94E6
:10E7500078F91816D4F460916E0270916F028827D0
:10E7600077FD8095982F0E9425F39B01AC01C30192
:10E77000B2010E941FF387FF08C080E00E948D8DC8
:10E780000E9496F87595679501C060E060939A0FB6
:10E790008091D5069091D606A091D706B091D80663
:10E7A0000097A105B10521F129813A814B815C8156
:10E7B000281B390B4A0B5B0B57FD1AC00E94928F26
:10E7C0002B013C016091D3067091D40680E090E06B
:10E7D0000E9423F39B01AC01C301B2010E941FF30D
:10E7E00087FFA5C040E152E261E072E280E08DDD8A
:10E7F0008091CF069091D006A091D106B091D2061B
:10E800000097A105B10521F129813A814B815C81F5
:10E81000281B390B4A0B5B0B57FD1AC00E94E98E6F
:10E820002B013C016091CD067091CE0680E090E016
:10E830000E9423F39B01AC01C301B2010E941FF3AC
:10E8400087FF72C04FED51E262EF71E28FEF5DDD45
:10E850006091800F7091810F882777FD8095982FA8
:10E860000E9425F320914A0630914B0640914C06B8
:10E8700050914D06FAE0AF2EB12CCC24CA94DC2C7A
:10E880007B018C0168EC76E08CEC96E0A2DD809157
:10E890009606811127C040904A0650904B06609022
:10E8A0004C0670904D0620E030E040EA50E4C30191
:10E8B000B2010E9478F987FF04C060E06093980F6E
:10E8C000CCCE20E030E046E153E4C301B2010E9427
:10E8D0001FF3181694F30E94508C0E9496F87595B9
:10E8E0006795ECCF1092980FB8CE409046065090A6
:10E8F0004706609048067090490620E030E848E9F5
:10E9000053E4C301B2010E9478F91816A4F020E084
:10E9100030E040EA50E4C301B2010E941FF387FFD8
:10E92000CBCE80E066DEC0CE0E94198B91CF80E016
:10E930000E94648B5DCF80E06BDE40904606509075
:10E9400047066090480670904906E1CF0F931F93E9
:10E95000CF93DF93EC018B016091F0114091F111A5
:10E96000641306C084EE91E10E94F85160DEF4CF9A
:10E9700028813981F801808191815091EF1174E0F3
:10E98000579FF0011124E851FE4E33872287958767
:10E9900084876F5F6093F01181E0850F841719F011
:10E9A0008093EF1102C01092EF11DF91CF911F9170
:10E9B0000F9108950F931F93CF93DF93CDB7DEB7D9
:10E9C00028970FB6F894DEBF0FBECDBF8823C1F0E5
:10E9D00083E992E098878F8304E610E01A83098325
:10E9E000BE01695F7F4FCE010196B0DF8AEB92E0F6
:10E9F0009E838D831A830983BE016B5F7F4F0BC09B
:10EA000088EB91E09C838B8384E190E09A838983F7
:10EA1000BE016D5F7F4FCE01019698DF28960FB63D
:10EA2000F894DEBF0FBECDBFDF91CF911F910F9144
:10EA300008950E9494D3BECFAF92BF92CF92DF923F
:10EA4000FF920F931F93CF93DF9300D01F92CDB708
:10EA5000DEB7F82E662351F01092E2061092DE0621
:10EA60001092DF061092E0061092E10652D7009154
:10EA7000DE061091DF062091E0063091E1065B0191
:10EA80006C01A01AB10AC20AD30AD7FC3DC0F7FE36
:10EA900005C004EC19E020E030E015C0E091E2068A
:10EAA0002F2D332727FD30952C5F3F4F4E2F5527B5
:10EAB00047FD5095241735073CF1EF1554F300E955
:10EAC00011E020E030E0DC01CB01800F911FA21F9C
:10EAD000B31F8093DE069093DF06A093E006B09309
:10EAE000E10680ED97E09C838B838CE291E09A8332
:10EAF0008983BE016D5F7F4FCE01019627DF809134
:10EB0000E2068F5F8093E2060F900F900F900F90B8
:10EB1000DF91CF911F910F91FF90DF90CF90BF9029
:10EB2000AF900895CF92DF92EF92FF926B017C013C
:10EB300083E3C816D104E104F10460F082E3C81A4B
:10EB4000D108E108F10862E370E080E090E04AD685
:10EB50006EDDEECFC701B60145D6FF90EF90DF9096
:10EB6000CF9065CDCF92DF92EF92FF920F931F93DC
:10EB7000CF93DF937C016A01EB0100E010E00C15FC
:10EB80001D0571F06991D701ED91FC910190F08123
:10EB9000E02DC7011995892B19F00F5F1F4FEFCF9B
:10EBA000C801DF91CF911F910F91FF90EF90DF90FF
:10EBB000CF900895089580E090E0089580E0089552
:10EBC000FC01E60FF11D849190E0982F8827319683
:10EBD000E4918E0F911D08950895DC011696ED9134
:10EBE000FC91179712968C911297481B15968C9151
:10EBF000483018F0E80FF11D477086958695869588
:10EC0000489F402D1124E40FF11D362F377080E806
:10EC100090E002C0959587953A95E2F766956695DE
:10EC20006695E60FF11D3081222311F0832B02C07F
:10EC3000809583238083089581E00895089590E06E
:10EC4000FC013197E231F10508F04CC0E057FF4F6D
:10EC50000C943DFA809180008F7703C080918000F2
:10EC60008F7D80938000089580918000877FF9CF09
:10EC700084B58F7702C084B58F7D84BD089580915F
:10EC8000B0008F7703C08091B0008F7D8093B0007B
:10EC90000895809190008F7707C0809190008F7DBC
:10ECA00003C080919000877F8093900008958091A9
:10ECB000A0008F7707C08091A0008F7D03C0809156
:10ECC000A000877F8093A0000895809120018F7716
:10ECD00007C0809120018F7D03C080912001877F34
:10ECE0008093200108953FB7F89480910B11909183
:10ECF0000C11A0910D11B0910E1126B5A89B05C065
:10ED00002F3F19F00196A11DB11D3FBF6627782F37
:10ED1000892F9A2F620F711D811D911D42E0660F90
:10ED2000771F881F991F4A95D1F708958091770F13
:10ED30009FB780FF09C0F89480910B018D7F80936D
:10ED40000B019FBF8FEF08C0F89480910B01826088
:10ED500080930B019FBF81E0809384028091770FA5
:10ED60009FB781FF09C0F89480910B018160809367
:10ED70000B019FBF8FEF08C0F89480910B018E7F2D
:10ED800080930B019FBF81E0809385028091770F74
:10ED90009FB782FF09C0F89480910B018B7F80930D
:10EDA0000B019FBF8FEF08C0F89480910B01846026
:10EDB00080930B019FBF81E0809386028091770F43
:10EDC0009FB783FF09C0F89480910B018064809302
:10EDD0000B019FBF8FEF08C0F89480910B018F7BD0
:10EDE00080930B019FBF81E08093870208954F922B
:10EDF0005F926F927F92AF92BF92CF92DF92EF922B
:10EE0000FF920F931F93CF93DF938C01EB01FC01D3
:10EE100047A050A461A472A4AFA0B8A4C9A4DAA466
:10EE20009501A601C301B2010E941FF387FF40C0F4
:10EE3000A3019201C301B2010E9484F32B013C01A2
:10EE4000F80183A994A9A5A9B6A9BC01CD01905840
:10EE50009B01AC010E9452F7F80127A530A941A9F6
:10EE600052A90E9484F39B01AC01C301B2010E942C
:10EE700051F70E94BDF97B018C019B01AC01B501EA
:10EE8000C6010E941FF387FF02C07501860197012A
:10EE9000A801B501C6010E941FF3882349F0A7010C
:10EEA000B8014FA358A769A77AA788818160888392
:10EEB000DF91CF911F910F91FF90EF90DF90CF9056
:10EEC000BF90AF907F906F905F904F9008958F921A
:10EED0009F92AF92BF92CF92DF92EF92FF920F93E9
:10EEE0001F93CF93DF9300D01F92CDB7DEB756EEBE
:10EEF000852E50E1952E64E7A62E67E0B62E06EB30
:10EF000019E0C12CD12C7601C394F4016191719167
:10EF1000819191914F01F50121913191419151914F
:10EF20005F0129833A834B835C830E9423F3298109
:10EF30003A814B815C810E9484F30E949BF8F80126
:10EF400061937193819391938F01C616D706E8065A
:10EF5000F90610F46B017C01F6EF8F16F0E19F06C5
:10EF6000A1F66FEF7FEFCB01A70196010E94F4F6A7
:10EF70002093B60F3093B70F4093B80F5093B90F4B
:10EF80000F900F900F900F90DF91CF911F910F91E5
:10EF9000FF90EF90DF90CF90BF90AF909F908F90B9
:10EFA00008958EBD0DB407FEFDCF08958FEF8EBD81
:10EFB0000DB407FEFDCF8EB508959091C00095FF6A
:10EFC000FCCF8093C60008953FB7F89420914E0A75
:10EFD00080914D0A821759F0E22FF0E0E353F64F8B
:10EFE000808190E02F5F2F7720934E0A02C08FEF31
:10EFF0009FEF3FBF08958091E3069091E40600974C
:10F0000031F04AE050E060E070E00C945FF160E0C5
:10F0100070E0CB0108958091E3069091E40600979B
:10F0200031F04AE050E060E070E00C942EF060E0D7
:10F0300070E0CB010895EFDF97FD0CC0ECDF6F3F70
:10F0400071058105910509F014F4E5DF01C06FEF4A
:10F05000862F089580E008958091E3069091E4065C
:10F06000892B39F0E8DF91E0811101C090E0892F10
:10F07000089581E008951F93CF93DF938091E30675
:10F080009091E4060097E1F0FC01EF011191212F2E
:10F090002F7D79F0153411F01536B9F7188260E03C
:10F0A00070E00E94C6EE1883562F472F382F292F65
:10F0B0000BC060E070E0DF91CF911F910C94C6EE21
:10F0C00050E040E030E020E0652F742F832F922F36
:10F0D000DF91CF911F910895149A0895179A109275
:10F0E000B107169A1092B207159A1092B307F4CF8F
:10F0F000CF92DF92EF92FF92C0905D06D0905E06B5
:10F10000E0905F06F090600680916206882321F10E
:10F1100020E030E0A901C701B6010E941FF3882357
:10F12000D9F020E030E040E05FE3C701B6010E9483
:10F1300084F39B01AC010E9484F32BED3FE049E492
:10F1400050E40E9484F39B01AC0160E070E080E831
:10F150009FE30E942EF804C060E070E080E89FE327
:10F160006093BB0F7093BC0F8093BD0F9093BE0F45
:10F17000FF90EF90DF90CF900895CF92DF92EF92C3
:10F18000FF92CF93DF93EC0180916602882309F40C
:10F1900042C0C0905702D0905802E0905902F090BF
:10F1A0005A02A7019601688179818A819B810E9418
:10F1B00078F9181624F4C882D982EA82FB82C090BA
:10F1C0005B02D0905C02E0905D02F0905E02A701CD
:10F1D00096016C817D818E819F810E9478F918163D
:10F1E00024F4CC82DD82EE82FF82C0905F02D09058
:10F1F0006002E0906102F0906202A70196016885CA
:10F2000079858A859B850E9478F9181624F4C8862A
:10F21000D986EA86FB86DF91CF91FF90EF90DF9051
:10F22000CF90089580E1E0ECF7E0A9E2B4E001902E
:10F230000D928A95E1F7089580E1E9E2F4E0A0EC0F
:10F24000B7E001900D928A95E1F70895AF92BF92D1
:10F25000CF92DF92EF92FF920F931F93CF93DF93A2
:10F26000C82FDD27C7FDD0958E01000F111F000F9D
:10F27000111FF801EC54F84F20E030E0A901608143
:10F280007181828193810E9452F7F801EF52FF4E03
:10F2900020813181428153810E9452F76B017C01B0
:10F2A000F801ED59F94F60837183828393830E5C7B
:10F2B0001C4DF80165917591859194918E01000F17
:10F2C000111F000F111F98012159394F5901A70132
:10F2D00096010E9452F7F5016083718382839383C4
:10F2E000025C1C4DF8016591759185919491CC0F4C
:10F2F000DD1FCC0FDD1FC95ADD4FA70196010E940B
:10F3000052F7688379838A839B83DF91CF911F9122
:10F310000F91FF90EF90DF90CF90BF90AF90089546
:10F320009091CF10E92FF0E0E053F84F80839F5F7A
:10F33000943018F49093CF1002C01092CF108091A7
:10F3400073098F5F809373090895CF93FC01C62FD3
:10F3500080818B3399F080917309843078F4209107
:10F36000CF1030E6239FC0011124BF018E50984F6B
:10F370000E948EFA8C2FD4DF81E001C080E0CF9113
:10F38000089581548A3148F5482F50E0FA01B3E0DE
:10F39000F595E795BA95E1F7EC5DFB4F208130E0FC
:10F3A000877002C0359527958A95E2F720FF15C032
:10F3B000FA01E65FFB4F2081222339F08091880615
:10F3C00090918906820F911D02C080E090E0909399
:10F3D000E4068093E30681E0089580E0089583E5E4
:10F3E000D0DF882349F047DE60935F0770936007A2
:10F3F000809361079093620784E5C3DF882349F017
:10F400003ADE60935B0770935C0780935D0790938F
:10F410005E0782E4B6DF882349F0EDDD6093C7091B
:10F420007093C8098093C9099093CA0988E5A9DF38
:10F43000882349F020DE60939107709392078093B0
:10F4400093079093940789E59CDF882349F013DEA6
:10F45000609395077093960780939707909398070A
:10F460008AE58FDF882349F006DE60939907709361
:10F470009A0780939B0790939C0785E482DF8823FB
:10F4800049F0F9DD60939D0770939E0780939F0775
:10F490009093A007089583E574DF882319F0DCDDDD
:10F4A0008093D40708950F931F93CF93DF93C6E102
:10F4B000D3E003E617E0899164DF882331F0DBDDD8
:10F4C000F80160837183828393830C5F1F4FF3E0A5
:10F4D000CA31DF0781F7DF91CF911F910F91089516
:10F4E00083E54FDF882389F0C6DD20E030E04AE77E
:10F4F00054E40E9484F30E949BF86093AE0F7093D3
:10F50000AF0F8093B00F9093B10F08953ADF882327
:10F5100039F081E02091E3063091E406232B09F4D1
:10F5200080E0089583E5F2DF882329F074DD70938D
:10F530009D0260939C020895CF92DF92EF92FF921A
:10F540000F931F93CF93DF93C6E1EC2EC3E0FC2E05
:10F5500009E214E0C0ECD7E08AE8C82E86E0D82E95
:10F56000F70181917F010DDF8823C9F084DDF60169
:10F570002081211104C020918E06222329F02881A8
:10F5800039814A815B8103C020E030E0A9010E94FB
:10F5900052F7F801608371838283938309C0888165
:10F5A0009981AA81BB81F80180839183A283B3836F
:10F5B0000C5F1F4F2496FFEFCF1ADF0A8AE1E8168F
:10F5C00083E0F80669F686E4A1DF8823B9F053DD0D
:10F5D00020E030E0A9010E9478F918167CF44BDD98
:10F5E00020E030E040E752E40E942EF860930C02E5
:10F5F00070930D0280930E0290930F02DF91CF91D2
:10F600001F910F91FF90EF90DF90CF900895809120
:10F61000E2119091E311891B8F7008950B96FC0104
:10F62000849108950A96FC018491089568E0C8CAFF
:10F6300066E0C6CAFC0184910895FCDF882311F0BE
:10F64000823011F486E0089583E00895FB01418142
:10F65000DC0112962C911297421760F013962C91B0
:10F660001397241738F0608115962C91621710F4C7
:10F670002481B3CA0895FC0120818281820F828394
:10F680009181891760F484818F5F84838381820FE5
:10F69000891710F08FEF890F838381E0089580E050
:10F6A0000895FC0112828081815083831482089521
:10F6B00088E290E00197F1F708952EE93FE0009786
:10F6C00029F0F9013197F1F70197F9CF08950F93D8
:10F6D000FC010150040F84A996A9941718F008178B
:10F6E00028F402C0081750F0041740F42150260FE8
:10F6F00083A995A9961720F4281720F480E007C065
:10F70000281720F481E0261710F0F8CF81E00F9140
:10F710000895DB01ED91FC911994EF92FF920F9304
:10F720001F93CF93DF931F92CDB7DEB78C01DC011F
:10F730001296ED90FC901397D196ED91FC91D29793
:10F7400082E0199520E030E04AE0B701C801E1DF2E
:10F75000F82ED801D196ED91FC91D29783E01995BE
:10F76000D801D196ED91FC91D29780E01995FF20B8
:10F7700081F1F801628173819E012F5F3F4F46E462
:10F78000C801C7DF8981D8018C9312966D917C9155
:10F7900013979E012F5F3F4F47E4C801BADF89816D
:10F7A000F80181836281738120E030E048E4C80180
:10F7B000B0DFD8011B968C931B9798012D5C3F4FAF
:10F7C00012966D917C91139747E1C801A2DF81E009
:10F7D00001C080E00F90DF91CF911F910F91FF90BA
:10F7E000EF9008958F929F92AF92BF92CF92DF9247
:10F7F000EF92FF926B017C0176DA4B015C01C11440
:10F80000D104E104F104D9F06EDA681979098A09A2
:10F810009B09683E73408105910588F321E0C21A77
:10F82000D108E108F10888EE880E83E0981EA11C3B
:10F83000B11CC114D104E104F10431F7E0CFFF9011
:10F84000EF90DF90CF90BF90AF909F908F900895F2
:10F85000CF93DF93282F30E0F901EC55FF4D8491D1
:10F86000F901E159F24CD491F901EB54F24CC491F5
:10F87000CC2389F08111E3D9EC2FF0E0EE0FFF1FCC
:10F88000E85EFC4DA591B4912C912D2381E090E090
:10F8900021F480E002C080E090E0DF91CF910895F4
:10F8A0000F931F93CF93DF931F92CDB7DEB7282F0F
:10F8B00030E0F901EC55FF4D8491F901E159F24C2A
:10F8C0001491F901EB54F24C04910023C1F0882308
:10F8D00019F06983B4D96981E02FF0E0EE0FFF1FC2
:10F8E000E657FF4DA591B4919FB7F8948C916111A3
:10F8F00003C01095812301C0812B8C939FBF0F9073
:10F90000DF91CF911F910F91089561E0FC018081FB
:10F91000C7CF2FB7F8946091101170911111809199
:10F920001211909113112FBF08950F931F93CF932E
:10F93000DF93EB01EEDF8B0139DB8F3F41F0E9DF35
:10F94000601B710B6C177D07B8F380E001C081E08C
:10F95000DF91CF911F910F910895CF92DF92FF9287
:10F960000F931F93CF93DF9300D01F92CDB7DEB7D5
:10F970006C01F62EFC018281982F906A96959CBDB1
:10F9800080FD06C091E0863009F490E0892F01C027
:10F9900080E08DBD60E0F601808129833A834B834E
:10F9A0005C837EDF6CE271E0C601BFDF8F2D806477
:10F9B000F8DA08E110E05C814B813A812981DA01B3
:10F9C000C901002E04C0B695A795979587950A940E
:10F9D000D2F729833A834B835C83E3DA0850110919
:10F9E00029813A814B815C81083FFFEF1F0739F77E
:10F9F000FF2029F088E0F81621F08FEF03C085E999
:10FA000001C087E8CEDAECE0FE1201C0CFDA10E0E8
:10FA1000CDDAF601838387FF04C01F3F11F01F5F1B
:10FA2000F7CF0F900F900F900F90DF91CF911F9114
:10FA30000F91FF90DF90CF9008956BDF60933904B2
:10FA400070933A0480933B0490933C0408955F9232
:10FA50006F927F928F929F92AF92BF92CF92DF92DE
:10FA6000EF92FF920F931F93CF93DF93EC01C62E7B
:10FA7000D42EB22EEC80FD80C701DCDD182F8C81E6
:10FA80009D81DBDD982E113011F00FEF01C00FE0EA
:10FA90008C819D81C7DD182F8C819D81BFDDA82EB3
:10FAA0008C819D81C3DD20E62B1530F4009721F079
:10FAB000E80EF91E11E60FC08C819D81B9DDE0E4EE
:10FAC000EB1530F4009721F0E80EF91E11E403C0A5
:10FAD000F1E1EF0EF11CAB1430F4188A1B8A1C8A7A
:10FAE000198A1A8A95C0A116C0F3A92DB0E0F701B2
:10FAF00084918F3F21F4FFEFEF1AFF0A3EC01B11E4
:10FB000034C08C819D8196DD97012F5F3F4FF701B7
:10FB1000882311F0823091F484918B8BF901249128
:10FB20002C8BF7013396E491E88BF7013496E4913E
:10FB3000E98BF7013596E491EA8B24C09491892FE3
:10FB40008F7082508A8B92959F70998BF9012491C6
:10FB5000822F8F708C8B22952F702B8BF701329612
:10FB6000E491E295EF70E88B0DC0F7013296E491D5
:10FB7000E023EE0EF11CEA0EFB1E1A1509F4ADCFC0
:10FB80001F5FB5CFE114F10409F442C08C819D815F
:10FB900054DDA82E6B88BC8879887C0C9A899B0DD3
:10FBA0001D2D191B0B2D262D412F672DCE018FDD0D
:10FBB000882361F1EA0CF11CF7E06F0E66946694FD
:10FBC0006694512E5B0C5E012CE1A20EB11C862CBA
:10FBD000912C1515D9F0072D67018C2D8E198615DE
:10FBE00088F4F60184916A817B810C8F1D8F1F8EB2
:10FBF0008E8F95014BE3CE018CDDFFEFCF1ADF0A2C
:10FC0000085FEBCFE80CF91C1F5FE3CF888901C0C8
:10FC100080E0DF91CF911F910F91FF90EF90DF90E7
:10FC2000CF90BF90AF909F908F907F906F905F909C
:10FC30000895CF92DF92EF92FF920F931F93CF938D
:10FC4000DF931F92CDB7DEB76C01DC01DC96EC9040
:10FC5000DC97DB96FC90DB978C010C5F1F4F59966D
:10FC6000ED91FC915A97C80169831995482F4E0D63
:10FC700029816F2DC801EBDEF60123AD992787FDA1
:10FC80009095820F911D83AF81E090E00F90DF91FE
:10FC9000CF911F910F91FF90EF90DF90CF9008953B
:10FCA000BF92CF92DF92EF92FF920F931F93CF9369
:10FCB000DF937C018B0120E030E0F701E20FF31FBE
:10FCC000E491EE2319F02F5F3F4FF7CFF801CF01FA
:10FCD000801B910B41914111FACFC4E1D0E0C81BC8
:10FCE000D1093327C217D3071CF492E0C92E02C0F2
:10FCF000CC24C3948091851190E06C2D70E06F5FEF
:10FD00007F4F0E942AFAB62E86E0D82ED60E80911A
:10FD1000B811D81650F08091BA1190E02D2D30E036
:10FD20002B5031098217930794F5F12C0115110519
:10FD3000C1F18AE30E94EE6982E0C8120FC0DB0CB9
:10FD40008091B811D81668F12091BA1130E08D2D4C
:10FD500090E00B97281739071CF423C0FF2009F106
:10FD60008C2F880F8C0F880F8093BB11D092BC1101
:10FD700080E20E94EE69C801DF91CF911F910F913F
:10FD8000FF90EF90DF90CF90BF900C942C6A109270
:10FD9000BB11D092BC11C7010E941F6AFF24F394CB
:10FDA000C5CFDF91CF911F910F91FF90EF90DF9022
:10FDB000CF90BF900895CF92DF92EF92FF921F9362
:10FDC000CF93DF9300D01F92CDB7DEB7809106119D
:10FDD00090910711A0910811B0910911B7FF08C0C7
:10FDE0001092061110920711109208111092091129
:10FDF0008091850790918607A0918707B091880729
:10FE000040910611509107116091081170910911EC
:10FE100084179507A607B70744F4809306119093BB
:10FE20000711A0930811B093091180919E028823B5
:10FE300051F1609106117091071180910811909114
:10FE40000911C0908907D0908A07E0908B07F09045
:10FE50008C076C0D7D1D8E1D9F1D0E9425F320E0DB
:10FE600030E048EC52E40E9484F369837A838B8308
:10FE70009C83CE0101960E941166BC0180918F0780
:10FE8000909190070DDF809102111091BC068111B5
:10FE900006C01123B1F180919E02882391F16091F7
:10FEA0000611709107118091081190910911C0906D
:10FEB0008907D0908A07E0908B07F0908C076C0D33
:10FEC0007D1D8E1D9F1D0E9425F320E030E048EC33
:10FED00052E40E9484F3E0918D07F0918E073097F1
:10FEE00021F06083718382839383112329F0E09151
:10FEF000BD06F091BE0619958091021181110E94F4
:10FF0000318A0F900F900F900F90DF91CF911F913A
:10FF1000FF90EF90DF90CF9008950F931F93CF93B2
:10FF20008091061190910711A0910811B0910911CB
:10FF3000B7FF08C010920611109207111092081115
:10FF4000109209118091850790918607A0918707EB
:10FF5000B0918807409106115091071160910811E6
:10FF60007091091184179507A607B70744F4809389
:10FF7000061190930711A0930811B0930911809175
:10FF80009E02882301F16091061170910711809102
:10FF90000811909109110091890710918A07209109
:10FFA0008B0730918C07600F711F821F931F0E9477
:10FFB00025F30E9496F8CB017AD7BC0180918F0778
:10FFC000909190076DDE80910211C091BC06811165
:10FFD00006C0CC23A1F180919E02882381F160911B
:10FFE00006117091071180910811909109110091EB
:10FFF000890710918A0720918B0730918C07600F39
:020000021000EC
:10000000711F821F931F0E9425F3E0918D07F091CD
:100010008E07309721F06083718382839383CC2392
:1000200029F0E091BD06F091BE061995809102116C
:10003000882329F0CF911F910F910C94318ACF9191
:100040001F910F9108958091061190910711A09131
:100050000811B0910911B7FF08C010920611109253
:100060000711109208111092091180918507909143
:100070008607A0918707B09188074091061150919B
:100080000711609108117091091184179507A6074F
:10009000B70744F48093061190930711A0930811B9
:1000A000B093091180919E02882389F020918907DD
:1000B00030918A078091061190910711820F931F4A
:1000C000F6D6BC0180918F0790919007E9DD809171
:1000D00002114091BC06811106C0442311F18091A8
:1000E0009E028823F1F08091890790918A072091E0
:1000F000061130910711820F931FE0918D07F09147
:100100008E07309711F091838083442329F0E0918A
:10011000BD06F091BE0619958091021181110E94D1
:10012000318A8091021108958EDF882329F0E091B1
:10013000BD06F091BE061994089585CF80910211F5
:1001400081110C94318A6091061170910711809190
:10015000081190910911611571058105910571F1E1
:100160000E9425F32091E5063091E6064091E706CE
:100170005091E8060E9484F39B01AC016091CC078A
:100180007091CD078091CE079091CF070E9452F7D2
:100190006093CC077093CD078093CE079093CF07E1
:1001A0001092061110920711109208111092091165
:1001B00083E00E94078981E080939E0280919E02E5
:1001C000882339F08CEC97E0C1D5BC0189E298E333
:1001D00067CD08953F924F925F926F927F928F9278
:1001E0009F92AF92BF92CF92DF92EF92FF920F93C6
:1001F0001F93CF93DF9300D000D0CDB7DEB78C0133
:10020000362E809102118823C9F026960FB6F894F5
:10021000DEBF0FBECDBFDF91CF911F910F91FF9039
:10022000EF90DF90CF90BF90AF909F908F907F9096
:100230006F905F904F903F900C94318A809106119F
:1002400090910711A0910811B0910911892B8A2B67
:100250008B2B09F490C0F1DB932DA4E09A02C0012E
:1002600011249E838D83FC01E054F84F408051801F
:10027000628073808091660281110BC020E030E0C3
:100280004AE754E4C301B2010E9452F76B017C01BA
:1002900008C0ED81FE81E95AFD4FC080D180E28027
:1002A000F3808091061190910711A0910811B091EF
:1002B000091189839A83AB83BC83BC01CD010E9461
:1002C00025F32091E5063091E6064091E70650912E
:1002D000E8060E9484F39B01AC01C301B2010E94B5
:1002E00052F74B015C01AD81BE81A054B84FBE8373
:1002F000AD83FD01608371838283938389819A81B9
:10030000AB81BC81B7FF13C020E030E04AE754E482
:10031000C301B2010E9451F76B017C019B01AC014A
:10032000C501B4010E941FF387FF18C010C0898166
:100330009A81AB81BC81892B8A2B8B2B79F0A70109
:100340009601C501B4010E9478F918163CF4AD81FC
:10035000BE81CD92DD92ED92FC921397832D57D7FB
:1003600010920611109207111092081110920911A3
:1003700081E080939E0280919E02882309F49FC0B1
:100380002DEC3CEC4CEC5DE36091E5067091E606EB
:100390008091E7069091E8060E9478F9E32DFF2707
:1003A000E7FDF09587FD09C0CF01880F991F880FE1
:1003B000991F8054984FCAD468C0EE0FFF1FEE0FEC
:1003C000FF1FE054F84F20E030E04AE754E460813A
:1003D0007181828193810E9484F30E9496F86B015F
:1003E0007C01611571058105910561F097FF0AC0D7
:1003F000F094E094D094C094C11CD11CE11CF11C79
:100400008DE201C080E280939806C701B60128EE14
:1004100033E040E050E00E9416F76AE0862E912C0F
:10042000A12CB12CCA01B901A50194010E9416F7B3
:10043000605D609399068EE280939A06C701B601CB
:1004400024E630E040E050E00E9416F7CA01B9010E
:10045000A50194010E9416F7605D60939B06C70199
:10046000B601A50194010E9416F7F62ECA01B90142
:10047000A50194010E9416F7605D60939C0680E3DD
:100480008F0D80939D0688E996E0BC01C8012696F1
:100490000FB6F894DEBF0FBECDBFDF91CF911F9195
:1004A0000F91FF90EF90DF90CF90BF90AF909F9013
:1004B0008F907F906F905F904F903F90F1CB2696FA
:1004C0000FB6F894DEBF0FBECDBFDF91CF911F9165
:1004D0000F91FF90EF90DF90CF90BF90AF909F90E3
:1004E0008F907F906F905F904F903F90089562E063
:1004F00082E298E36FCE61E08BE198E36BCE60E03F
:1005000084E198E367CECF92DF92FF920F931F931F
:10051000CF93DF931F921F92CDB7DEB7082F162F10
:10052000E0919911F0919A1184E891E149835A83FD
:100530001995180F4981C42E5A81D52EF12CD60158
:100540002D916D01222341F0412F602F84E891E12C
:100550007EDA080FF80EF3CF8F2D0F900F90DF91FA
:10056000CF911F910F91FF90DF90CF9008950F933F
:100570001F930E949A5106ED15E320E448E060E0E5
:1005800080E00E94E65086E69DE20E94826940E398
:1005900053E061E18DE3B7DF8BE09AE20E9482696C
:1005A00046E353E06CE18EE3AEDF8EE693E20E9419
:1005B000826946E453E069E28FE3A5DF8EE693E2C9
:1005C0000E94826942E553E06EE38EE39CDF44E5DE
:1005D00053E06EE383E497DF0E9448698111CBCF3B
:1005E0001F910F91089580910211882319F01092A4
:1005F0007F0637C7BCCFCF93DF931F92CDB7DEB74F
:100600008091BD11811106C081E08093BD1184E805
:1006100091E183D8609186117091871119829E01B2
:100620002F5F3F4F4FE084E891E173D8A0DF0F9038
:10063000DF91CF910895DFDFE4E0F1E080818F7DED
:1006400080839FB7F894E5E0F1E080818062808349
:100650009FBFE4E0F1E080818F7B80839FB7F894B7
:10066000E5E0F1E08081806480839FBF6A98729AA0
:1006700054985C9A82E08093B309F0D41092AD094B
:1006800008952F923F924F925F926F927F928F9236
:100690009F92AF92BF92CF92DF92EF92FF920F9311
:1006A0001F93CF93DF93CDB7DEB7C454D1090FB6F4
:1006B000F894DEBF0FBECDBF4C015B017A01322E34
:1006C0001C8E1F8E19821C826115710511F410E0B9
:1006D000AFC0FC0183818111FACFFA0180818F3292
:1006E00061F4CA017C010196F70120812F32D1F318
:1006F000F50183818250823010F465010BC0618D59
:10070000728DCE0101960E945E5F882301F3CE01B7
:1007100001966C018E01045E1F4F2801F7E36F2ED6
:10072000712C6C0E7D1E9BE0690E711CFE013196D2
:100730002496FFAFEEAF249725960FAF2597212E75
:1007400037C080E28193E615F705D9F7D70120E09D
:1007500097E04A2F3B2F8D9181112DC08FA98032B8
:1007600009F4B5CF842F932F7C01FC0120810196E1
:100770002F32D1F3222309F452C021E0AE01495CAB
:100780005F4FB601C8010E94A34B882309F49FCF95
:10079000CA14DB0419F0C6010E94284F0415150580
:1007A000B9F125969FAD2597822D6801092F182F45
:1007B000FE01F796C6CF8F3289F28E3219F0EAE445
:1007C000F3E20AC09A3009F482CF28E09AE0C1CF60
:1007D0003196381709F47BCF34913111F9CF921744
:1007E00008F475CF813208F472CF8F3709F46FCFD8
:1007F00031E0320FE7E3F0E0EC0FFD1FE20FF11DF7
:100800002FE9280F2A3108F480528083232FA1CFAB
:1008100023969FAD239724968FAD2497C6CF232D83
:10082000AE01495C5F4FB601C4010E94A34B182F73
:10083000CE0101960E948250CE014C960E948250B9
:10084000812FCC5BDF4F0FB6F894DEBF0FBECDBF5C
:10085000DF91CF911F910F91FF90EF90DF90CF909C
:10086000BF90AF909F908F907F906F905F904F90D0
:100870003F902F9008952F923F924F925F926F92E8
:100880007F928F929F92AF92BF92CF92DF92EF9220
:10089000FF920F931F93CF93DF93CDB7DEB7C0576F
:1008A000D1090FB6F894DEBF0FBECDBF7C016B013E
:1008B0004A012DB73EB7AF963FAF2EAFAF97AD967B
:1008C0001FAEAD9734E0C30ED11C8E01015A1F4FED
:1008D000BEE06B2EB3E07B2E80E4282E312C2C0E54
:1008E0003D1E84E0280E311C41E252E1BE016F5FE3
:1008F0007F4FC6010E94D95D18160CF056C12C8599
:10090000922F9871903109F0CEC08091BD14815022
:10091000823008F4C8C04DB65EB6BE016F5F7F4F2F
:10092000C80171D681E0F70190819111B4C0E1E076
:10093000F0E0D8010D900020E9F7E01BF10BEA0F81
:10094000FB1F31962DB73EB72E1B3F0B0FB6F89409
:100950003EBF0FBE2DBFEDB7FEB731965F018823B6
:1009600019F06DE573E001C0B701C5010E948EFA70
:10097000B801C5010E9478FA6DE573E0C5010E94D7
:1009800078FA25961FAE259728961FAE28972496AD
:100990001FAE1EAE249722967FAE6EAE229721E048
:1009A000A801B601C1016DDE81114DC08091BD1459
:1009B000811149C0EBECFFE384919F012F5F3F4F12
:1009C000882381F0E0962FAFE097E1963FAFE19763
:1009D0000E94DD77E0962FADE097E1963FADE1977D
:1009E000F901EACFEAE5F3E284919F012F5F3F4FDF
:1009F000811102C0980110C0E0962FAFE097E196F8
:100A00003FAFE1970E94DD77E0962FADE097E1964A
:100A10003FADE197F901E8CFF90181919F0188236A
:100A200079F0E0962FAFE097E1963FAFE1970E9413
:100A3000DD77E1963FADE197E0962FADE097ECCF03
:100A40008AE00E94DD778BE1FE01EC5BFF4FDE0167
:100A5000959601900D928A95E1F724968EAD9FAD03
:100A600024979CA38BA37AA269A240E050E0BE0128
:100A70006F5D7F4FC501FFDECE0181960E948750DA
:100A8000CE01805C9F4F0E9487500FB6F8945EBEE7
:100A90000FBE4DBE29CF80E001900020E9F73197CD
:100AA000EE19FF0946CF8981882309F47EC0853E6F
:100AB00009F41ACF8E3209F417CF809121128E32A9
:100AC00009F412CF2A7009F00FCF81E0903109F0BC
:100AD00080E080931312811108C08985873409F062
:100AE00003CF8A858E3709F4FFCE8091BD14813003
:100AF00021F068F08230A1F1F7CE8091BE14909180
:100B0000BF1401969093BF148093BE14EDCEBE0126
:100B10006F5F7F4F84E192E176D55701F5018191B6
:100B20005F01882319F00E94DD77F8CFA4E1AA2E97
:100B3000A2E1BA2EF50181915F01882319F00E948C
:100B4000DD77F8CF80E20E94DD776D8D7E8D8F8D11
:100B500098A14AE00E94B3668AE00E94DD77C4CE85
:100B6000BE016F5F7F4F84E192E14DD58114910406
:100B700041F064E172E1C4010E9465FA892B69F4D5
:100B800014C0AD96FFADAD972F2F30E08091BE140D
:100B90009091BF142817390741F0AD963FADAD973E
:100BA0003F5FAD963FAFAD979FCEAF962EAD3FADB9
:100BB000AF970FB6F8943EBF0FBE2DBFC059DF4FA1
:100BC0000FB6F894DEBF0FBECDBFDF91CF911F915E
:100BD0000F91FF90EF90DF90CF90BF90AF909F90DC
:100BE0008F907F906F905F904F903F902F900895DF
:100BF000EF92FF920F931F93CF93DF93CDB7DEB7A2
:100C00006F970FB6F894DEBF0FBECDBF7B0104E82F
:100C100012E126E832E1F8013183208322E02093BB
:100C2000BD149093BF148093BE1440E050E0BA010D
:100C30008AE892E10E945F5EF801808191812BE158
:100C4000FC013496DE01159601900D922A95E1F78C
:100C5000FC01828193819C838B838EE093E09A8355
:100C60008983A701BE016F5F7F4F82E094E003DEBE
:100C7000CE0101960E9487506F960FB6F894DEBFA2
:100C80000FBECDBFDF91CF911F910F91FF90EF90DD
:100C9000089524E08202C0011124FC01EB5BF04FB7
:100CA0004081518162817381FC01EB51F84F408397
:100CB000518362837383E091780FF091790F828979
:100CC0009389A489B5898093550F9093560FA0936B
:100CD000570FB093580F0895FC01138212828FE6CC
:100CE00093E09183808313AE14AE15AECF010496CA
:100CF0001186108613861286158621E0248722E24B
:100D00002687138A128A20E030E04FEFDC01A20F21
:100D1000B31F93964C932F5F3F4F2E303105B1F7A1
:100D200041E044A32EED35E7328F218F438F148E9F
:100D3000158E20E4268F178E2CEE35E736AB25ABCB
:100D4000778366830C948D7B0C94677720E030E08A
:100D500040E251E4FC0160817181828193810E94B3
:100D600084F30E9496F89B0177FF06C02227332761
:100D7000261B370B8DE201C08BE280939806C901D8
:100D800068EE73E00E942AFACB01EAE0F0E0BF01CE
:100D90000E942AFA805D80939906C90164E670E09A
:100DA0000E942AFACB01BF010E942AFA805D80933B
:100DB0009A06C901BF010E942AFA282FCB01BF0160
:100DC0000E942AFA805D80939B068EE280939C06A7
:100DD000205D20939D0688E996E00895492F441FE1
:100DE0004427441F29F022273327281B390B01C031
:100DF0009C01883E9340ACF0C90168EE73E00E940C
:100E00002AFACB01EAE0F0E0BF010E942AFA805DF5
:100E100080939A06C90164E670E00E942AFACB0129
:100E200012C024363105B4F0442311F08DE201C024
:100E300080E280939A06C90164E670E00E942AFA73
:100E4000CB01EAE0F0E0BF010E942AFA805D8093C6
:100E50009B0611C080E280939A0680939B062A30FD
:100E600031059CF0442311F08DE201C080E28093B3
:100E70009B06EAE0F0E0C901BF010E942AFACB011B
:100E8000BF010E942AFA805D05C0442311F08DE263
:100E900001C080E280939C06C9016AE070E00E9474
:100EA0002AFA805D80939D068AE996E008959C0168
:100EB00097FD0EC08436910584F064E670E00E94D0
:100EC0002AFACB016AE070E00E942AFA805D06C02F
:100ED0003195219531098DE201C080E280939B0616
:100EE0002A30310564F0EAE0F0E0C901BF010E9458
:100EF0002AFACB01BF010E942AFA805D01C080E27C
:100F000080939C06C9016AE070E00E942AFA805D25
:100F100080939D068BE996E008950F931F93CF93DE
:100F2000DF93E091780FF091790F82819381A48112
:100F3000B581181619061A061B06FCF48091770F66
:100F400080FF1BC083B19091460782958695869558
:100F5000837041E08427282F21709E7F292B2093C6
:100F60004607809145078170822339F08091F1070F
:100F700081608093F10780E08CDEE091780FF09142
:100F8000790F86819781A085B185181619061A06F2
:100F90001B063CF58091770F81FF23C023B1809120
:100FA000460790E022952695277031E02327022FEF
:100FB000017010E011950195110908271927027099
:100FC000112708271927009346078091450782704B
:100FD000802339F08091F10782608093F10781E0EE
:100FE00058DEE091780FF091790F82859385A48582
:100FF000B585181619061A061B063CF58091770F61
:1010000082FF23C023B18091460790E022952F7084
:1010100031E023272170C22F20E0D22FD195C19536
:10102000D109C827D927C470DD27C827D927C0937D
:1010300046078091450784708C2339F08091F10731
:1010400084608093F10782E024DE809146078093DC
:101050004507DF91CF911F910F9108950F931F9333
:101060000E94897C0091A1091091A2092091A309F5
:101070003091A409601B710B820B930B97FD0FC07D
:101080008091030185FB882780F991E08927909161
:10109000030196FF8260629B84608093B509809112
:1010A000B50981709091B50991FD826090914407D6
:1010B000891731F18130A9F028F0823041F0833076
:1010C00059F01CC0913089F0923099F017C09923E3
:1010D00061F0933071F012C0913059F0923071F498
:1010E00004C0992331F0933049F49091AD099F5F8A
:1010F00003C09091AD0991509093AD09809344073E
:101100001F910F910895E0E1F2E080E0919191113B
:1011100005C0282F482F421B50E204C0863181F4BD
:1011200026E1F8CF822F90E0342F320FFC01E05FF0
:10113000FD4F363118F450832F5FF4CF108208959D
:101140008F5FE4CF2091860621110BC042E450E06E
:10115000BC0180E192E00E94A3FAD5DF83E0809396
:101160009E02089567FF03C01092860660E02091FA
:10117000860630E0462F552747FD50954217530706
:101180006CF06093860642E450E0BC0180E192E09E
:101190000E9490F2B8DF83E080939E020895CF9280
:1011A000DF92EF92FF920F931F930E94897C009130
:1011B00040071091410720914207309143076B018E
:1011C0007C01C01AD10AE20AF30AF7FC13C020918D
:1011D0003F07209520933F07DC01CB018A549C4FA9
:1011E000AF4FBF4F8093400790934107A0934207B2
:1011F000B093430781E090913F07911101C080E0D7
:101200001F910F91FF90EF90DF90CF900895CF92B4
:10121000DF92EF92FF92CF93C82F0E94897C6B01DF
:101220007C0124EA30E74DE75FE36091E5067091C9
:10123000E6068091E7069091E8060E941FF387FF7B
:1012400004C040E050E0BA0104C04AEF50E060E062
:1012500070E04C0D5D1D6E1D7F1D40939D095093E8
:101260009E0960939F097093A009C0937102CF916A
:10127000FF90EF90DF90CF90089520913E072630A9
:10128000D8F486E0289FF0011124E65EF84F8091A3
:1012900067029091680291838083809106119091FA
:1012A0000711A0910811B091091182839383A4833F
:1012B000B5832F5F20933E0708956F927F928F92A0
:1012C0009F92AF92BF92CF92DF92EF92FF920F93D5
:1012D0001F93CF93DF9300D01F92CDB7DEB76C0181
:1012E0003B014701580129833A834B835C83C5DF67
:1012F00083E080939E02D0929007C0928F077092F5
:101300008E0760928D0729813A814B815C81CA01E9
:10131000B9010E9496F86093890770938A078093B9
:101320008B0790938C070E9425F36B017C019B0136
:10133000AC01C501B4010E9451F70E9496F8609378
:101340008507709386078093870790938807A70186
:101350009601F30160817181828193810E9451F72E
:101360000E949BF8609306117093071180930811F7
:10137000909309118DE89FE790936802809367022C
:101380000F900F900F900F90DF91CF911F910F91C1
:10139000FF90EF90DF90CF90BF90AF909F908F9095
:1013A0007F906F900895209167023091680228170E
:1013B0003907D9F090936802809367024093061131
:1013C000509307116093081170930911835193444E
:1013D00021F410927F0610923E0782E080939E02D5
:1013E00081E0809304111092AE090895CF93DF93AA
:1013F0001F921F92CDB7DEB789839A833EDF40E00C
:1014000050E0BA0189819A810F900F90DF91CF91BE
:10141000CACF21E020937F066093E5067093E6062D
:101420008093E7069093E80640E050E0BA0180918F
:10143000490790914A07B7CF6DEC7CEC8CEC9DE3AB
:10144000E8CF60E070E080E89FE3E3CF60E070E029
:1014500080E291E4DECF40E050E0BA0183E193E422
:10146000A2CFE0913E07EE2381F0E150E0933E07EA
:1014700086E0E89FF0011124E65EF84F4281538137
:1014800064817581808191818ECFE5CFCF93DF9389
:10149000EC0164E972E020DC83E693E099838883C1
:1014A000DF91CF9108952FB7F894909105019B7F1C
:1014B000909305012FBF87FD96C0A3982FB7F8948E
:1014C000909105019460909305012FBF880F2FB76D
:1014D000F894909105019B7F909305012FBF87FDA4
:1014E0008EC0A3982FB7F8949091050194609093C3
:1014F00005012FBF880F2FB7F894909105019B7FAE
:10150000909305012FBF87FD78C0A3982FB7F8945B
:10151000909105019460909305012FBF880F2FB71C
:10152000F894909105019B7F909305012FBF87FD53
:1015300062C0A3982FB7F89490910501946090939E
:1015400005012FBF880F2FB7F894909105019B7F5D
:10155000909305012FBF87FD4CC0A3982FB7F89437
:10156000909105019460909305012FBF880F2FB7CC
:10157000F894909105019B7F909305012FBF87FD03
:1015800036C0A3982FB7F89490910501946090937A
:1015900005012FBF982F990F2FB7F894809105015F
:1015A0008B7F809305012FBF97FD1FC0A3982FB796
:1015B000F894809105018460809305012FBF2FB7B7
:1015C000F894809105018B7F809305012FBF96FDD4
:1015D00018C0A3989FB7F894809105018460809308
:1015E00005019FBF0895A39A69CFA39AE0CFA39A5C
:1015F000C9CFA39AB3CFA39A9DCFA39A87CFA39A1B
:1016000071CFA39AE7CFFC0120E03EE2DB014C91D1
:10161000403241F0283011F430833196DB014C9197
:10162000408331962F5F6F5F7F4F2B3079F71082A9
:101630000895CF92DF92EF92FF92C0904A06D09029
:101640004B06E0904C06F0904D066091800F709133
:10165000810F68507109882777FD8095982F0E9427
:1016600025F39B01AC01C701B6010E941FF387FF60
:101670001DC020E030E040E050E4C701B6010E9408
:1016800052F70E949BF87093CE066093CD060E949D
:10169000897C605A75418F4F9F4F6093CF0670933E
:1016A000D0068093D1069093D20608C01092CF0640
:1016B0001092D0061092D1061092D206FF90EF90B1
:1016C000DF90CF900895B5CFCF92DF92EF92FF9247
:1016D000C0904606D0904706E0904806F090490634
:1016E0006091840F7091850F65517109882777FD8E
:1016F0008095982F0E9425F39B01AC01C701B6018C
:101700000E941FF387FF1DC020E030E040E251E45B
:10171000C701B6010E9452F70E949BF87093D4064D
:101720006093D3060E94897C605C73468F4F9F4F05
:101730006093D5067093D6068093D7069093D8060B
:1017400008C01092D5061092D6061092D7061092B5
:10175000D806FF90EF90DF90CF90089580E0B4CF4F
:101760004F925F926F927F928F929F92AF92BF92B1
:10177000CF92DF92EF92FF920F931F93CF93DF935D
:101780002C0126EB38E381E090E0F901459154917A
:10179000441655060CF062C0AC0141505109DA0103
:1017A000AA0FBB1FAA0FBB1FAC54B74CFD0165911C
:1017B0007491440F551F440F551F4E54574CFA0156
:1017C00065907490FC01EE0FFF1FEE0FFF1FEC54AD
:1017D000F74CA590B490FD0105911491F901C591C4
:1017E000D491FA0185909490882777FD8095982F61
:1017F0000E9425F36B017C01B201661977098827E5
:1018000077FD8095982F0E9425F32B013C01B501AF
:10181000601B710B882777FD8095982F0E9425F318
:101820009B01AC01C301B2010E9484F32B013C0176
:10183000BE0168197909882777FD8095982F0E9445
:1018400025F39B01AC01C301B2010E942EF89B015C
:10185000AC01C701B6010E9452F711C001962C5F7E
:101860003F4F8A33910509F090CFE8E9F9E365919C
:101870007491882777FD8095982F0E9425F3DF913A
:10188000CF911F910F91FF90EF90DF90CF90BF907D
:10189000AF909F908F907F906F905F904F90089542
:1018A0004F925F926F927F928F929F92AF92BF9270
:1018B000CF92DF92EF92FF92CF93DF93CDB7DEB757
:1018C0002C970FB6F894DEBF0FBECDBF80914A06AD
:1018D00090914B06A0914C06B0914D0689839A8356
:1018E000AB83BC836091800F7091810F882777FD57
:1018F0008095982F0E9425F329813A814B815C8144
:101900000E9451F76B017C016093160770931707D3
:1019100080931807909319072091990930919A099B
:1019200040919B0950919C090E9484F36D837E83B2
:101930008F8398876093120770931307809314071F
:101940009093150720910E0730910F0740911007D3
:1019500050911107C701B6010E9452F74B015C017B
:1019600060930E0770930F078093100790931107F1
:1019700020919509309196094091970950919809C5
:101980000E9484F369877A878B879C8760930A0714
:1019900070930B0780930C0790930D0720ED3CECA0
:1019A0004CE45DE3609191097091920980919309F3
:1019B000909194090E9484F32B013C012091060729
:1019C00030910707409108075091090769817A8192
:1019D0008B819C810E9451F79B01AC01C301B20134
:1019E0000E9484F32B013C0123E333E343E75FE3ED
:1019F0006091020770910307809104079091050799
:101A00000E9484F39B01AC01C301B2010E9452F712
:101A10002B013C0160930207709303078093040736
:101A20009093050789819A81AB81BC8180930607D9
:101A300090930707A0930807B093090729853A8573
:101A40004B855C856D817E818F8198850E9452F7E0
:101A5000A30192010E9451F72B013C0120E030E0EC
:101A60004EE453E40E9478F920E030E0A901181612
:101A7000ACF4C701B6010E9478F918166CF5A701FD
:101A80009601C501B4010E9451F760930E0770934F
:101A90000F0780931007909311071EC0C301B20176
:101AA0000E941FF387FF22C020E030E0A901C70198
:101AB000B6010E941FF387FF16C0A7019601C5015A
:101AC000B4010E9451F760930E0770930F07809343
:101AD00010079093110707C0412C512C8EE4682EFB
:101AE00083E4782E03C0412C512C3201C301B20192
:101AF0002C960FB6F894DEBF0FBECDBFDF91CF910D
:101B0000FF90EF90DF90CF90BF90AF909F908F901D
:101B10007F906F905F904F9008954F925F926F9279
:101B20007F928F929F92AF92BF92CF92DF92EF926D
:101B3000FF920F931F93CF93DF9300D01F92CDB7E7
:101B4000DEB70091840F1091850F8090460690902B
:101B50004706A0904806B0904906B801882777FD4F
:101B60008095982F0E9425F3A50194010E9451F7BA
:101B70006B017C016093FE067093FF068093000763
:101B80009093010720ED3CEC4CE45DE36091850906
:101B90007091860980918709909188090E9484F349
:101BA0002B013C012091FA063091FB064091FC0686
:101BB0005091FD06C501B4010E9451F79B01AC0193
:101BC000C301B2010E9484F32B013C0123E333E300
:101BD00043E75FE36091F6067091F7068091F8069F
:101BE0009091F9060E9484F39B01AC01C301B201FC
:101BF0000E9452F769837A838B839C836093F606F5
:101C00007093F7068093F8069093F9068092FA068F
